:020000040002F8
:1070000050900020C5730200CD730200CF730200C0
:10701000D1730200D3730200D57302000000000098
:10702000000000000000000000000000D773020014
:10703000D973020000000000DB730200DD73020060
:1070400029820200DF730200B98B0200E58702008B
:10705000F9870200DF730200698102008D8502005A
:10706000898B0200A18B0200DF730200DF73020034
:10707000DF730200DF730200DF730200DF730200C0
:10708000C98B020085820200DF730200DF730200F9
:10709000DF730200DF73020021880200DF73020049
:1070A000DF730200DF730200DF730200DF73020090
:1070B00071820200DF730200000000000000000087
:1070C000DF730200DF730200DF7302000D8802002D
:1070D0009D820200DF730200DF730200DF73020093
:1070E000DF7302000000000000000000000000004C
:1070F00000000000DF73020000000000DF730200E8
:10710000000000000000000000000000000000007F
:10711000000000000000000000000000000000006F
:10712000000000000000000000000000000000005F
:10713000000000000000000000000000000000004F
:10714000000000000000000000000000000000003F
:10715000000000000000000000000000000000002F
:10716000000000000000000000000000000000001F
:10717000000000000000000000000000000000000F
:1071800000000000000000000000000000000000FF
:1071900000000000000000000000000000000000EF
:1071A00000000000000000000000000000000000DF
:1071B00000000000000000000000000000000000CF
:1071C00000000000000000000000000000000000BF
:1071D00000000000000000000000000000000000AF
:1071E000000000000000000000000000000000009F
:1071F000000000000000000000000000000000008F
:10720000DFF810D000F042FA0048004755D50200E0
:10721000AFF300805090002030B450E8012F93B2BB
:10722000C48923448489A34228BF1B1B0489A34229
:1072300002BFBFF32F8F002007E0C3EA020340E83C
:107240000134002CE9D14FF001000A6030BC7047D6
:1072500050E8012FC2EA024240E801210029F7D19B
:10726000704730B450E8022F1FFAA2F3C488A3423B
:1072700002BFBFF32F8F00200DE0C489234484890F
:10728000A34228BF1B1BC2EA034340E80234002C80
:10729000E8D14FF001000A6030BC704750E8022F7F
:1072A000C2EA224240E802210029F7D17047034692
:1072B00053E8022FD988B2EB324F4FF0000017BFCE
:1072C00092B241EA014142EA014104E05A68B2EB5C
:1072D000324F08BF012043E80212002AE8D170476C
:1072E00030B4044654E8000F0D4644E80053002B28
:1072F000F8D1156030BC704730B4044654E8000F34
:1073000040EA010544E80053002BF7D1156030BC7A
:10731000704730B4044654E8000F00EA010544E821
:107320000053002BF7D1156030BC704730B40446D1
:1073300054E8000F80EA010544E80053002BF7D120
:10734000156030BC704730B4044654E8000F00EBC1
:10735000010544E80053002BF7D1156030BC70479D
:1073600030B4044654E8000FA0EB010544E8005394
:10737000002BF7D1156030BC704770B404464FF055
:10738000000054E8006F0D68AE4207BF44E80023D8
:10739000012044E800630E60002B1CBF0020F0E7D2
:1073A00070BC704730B4044654E8000F88422CBFCC
:1073B000451A054644E80053002BF5D1156030BC52
:1073C000704700000648804706480047FEE7FEE792
:1073D000FEE7FEE7FEE7FEE7FEE7FEE7FEE7FEE785
:1073E000CD8902000172020000487047B44D0300CD
:1073F00010B50446FFF7F8FF0068005D00F00100DB
:1074000010BD40EA01039B0703D009E008C9121F21
:1074100008C0042AFAD203E011F8013B00F8013B4E
:10742000521EF9D27047D2B201E000F8012B491E7A
:10743000FBD270470022F6E710B513460A46044611
:107440001946FFF7F0FF204610BD421C10F8011B43
:107450000029FBD1801A704730B50446002003464E
:1074600000E05B1C934203D2E05CCD5C401BF8D093
:1074700030BD034611F8012B00F8012B002AF9D189
:10748000184670470FB400B58DB010A909900B9045
:1074900000914FF0FF300A9000200C9005480690B4
:1074A000054807906A4609A80F9900F0C1F80DB089
:1074B0005DF814FB4D7602006B7602002DE9FF5F4C
:1074C0001D464FF0FF3BD5E9014691465F464FF020
:1074D0000008A9697F1C01988847296A8246884765
:1074E0000028F6D1BAF1FF3F0CD024F4C064002E7E
:1074F00019DD600614D5BAF12B0F09D0BAF12D0FA2
:107500000ED103E0584604B0BDE8F09F44F4806417
:10751000A9697F1C01988847761E8246002E02DDED
:10752000BAF1300F03D0B9F1000F26D032E0A969CB
:10753000761E44F400747F1C019888478246002E12
:1075400005DDBAF1780F06D0BAF1580F03D0B9F1C2
:10755000000F10D01EE0B9F1000F02D0B9F1100FEA
:1075600018D1A969761E24F400747F1C01988847FD
:107570008246102002E0082000E00A20814609E04F
:1075800008FB0908A969761E44F400747F1C019861
:1075900088478246002E05DD4946504600F034F803
:1075A0000028EDDAE96901988847A00502D46FF058
:1075B0000100A8E7E00725D1600613D5600502D5D4
:1075C000C8F1000000E0404629680A1D2A600968E9
:1075D000220501D5087015E0220701D5088011E0C9
:1075E00008600FE02868011D29600068210502D5A8
:1075F00080F8008006E0210702D5A0F8008001E0B5
:10760000C0F8008038467EE73A2800D2303820F0B3
:107610002002412A01D3A2F13700884201D34FF062
:10762000FF307047026811441378016018467047B4
:10763000D160044951610449116200211161114670
:1076400000F036B825760200F1730200426842B1BC
:10765000016811F8013B23B1521EC0E9001218461F
:1076600070470121C160881E704742685AB1C368E3
:10767000016843B983688B4205D0491E521CC0E99A
:107680000012002070474FF0FF307047064C074D46
:1076900006E0E06840F0010394E8070098471034E2
:1076A000AC42F6D3FFF7B0FDD0580300F05803000A
:1076B0002DE9F34F8BB04FF0000801F10C000C46A0
:1076C0004FF0010B46460DF1080A01906269012155
:1076D00001989047051E2DD0252D2CD0216A884772
:1076E000C0B16269012101989047216A884700284A
:1076F000F7D1411E62690198904700E0761CA169AC
:107700000B988847216A88470028F7D1E1690B98D0
:107710008847DBE7A1690B9888470746A84201D153
:10772000761CD3E7E1690B9888477F1C02D1B8F13A
:10773000000F6FD047E1002762693D463946019846
:1077400090472A2804D162690121019890470125B8
:10775000DFF888926269012101989047A0F1300119
:107760000A290AD24F45E5DC07EB870100EB410708
:10777000303FDFD445F01005ECE7E90601D46FF0A7
:1077800000476C280AD04C2814D0682815D06A28E5
:107790000DD074281CD07A281AD01DE0626901210E
:1077A000019890476C2802D045F0040514E045F09C
:1077B00002050DE045F020050AE06269012101980B
:1077C0009047682802D045F0080505E045F40065BB
:1077D0006269012101989047C4E9015765283DD0AD
:1077E00019DC58287AD00CDC452837D004DC252851
:1077F00026D0412831D131E046282FD047282CD13E
:107800002CE05B2877D0612828D063287CD06428BE
:1078100023D15AE0D1E06F2848D008DC66281DD07B
:1078200067281BD0692821D06E2816D127E0702840
:1078300045D0732868D0752847D078280DD14DE001
:10784000A1690B988847054625283FF469AFE1698F
:107850000B9888476D1C3FF46AAFB4E023466A4634
:107860006FF001000B99AFF300809FE045F04000FE
:107870006060A80723464FF0000236D43EE0E807D8
:107880007FF447AF2068011D21600068290501D5FC
:1078900006701BE7290701D5068017E7A90703D55E
:1078A000F117C0E9006111E706600FE745F04000FD
:1078B0006060A80723464FF0080216D41EE040F689
:1078C0000E0125EA0100606016E045F040006060AE
:1078D000A80723464FF00A0207D40FE045F0400006
:1078E0006060A80708D5234610226FF001000B99AD
:1078F000AFF300805AE007E0234610226FF001004A
:107900000B99FFF7DBFD51E04FF000094F464B4666
:10791000632802D05B2807D041E02079C00601D45B
:107920000120A06001273AE0626901210198904797
:107930005E2805D14FF001096269494601989047D8
:10794000216939B900210A46534643F82120491CD0
:107950000829FADBB0B3216969B9C11700EBD1621C
:1079600053110AEB830122F01F02821A01200B68D7
:10797000904003430B6062690121019890475D28A4
:10798000E8D1B9F1000F09D00020514651F820206C
:10799000D24341F82020401C0828F7DB02AB2246E6
:1079A00000976FF001000B99AFF3008000280CDA0C
:1079B000401C08D1BBF1000F05D04FF0FF300DB0D7
:1079C000BDE8F08FFFE74046F9E7E90701D108F18C
:1079D000010806444FF0000B78E60000CCCCCC0C3C
:1079E00070B58C1810F8015B15F0070301D110F881
:1079F000013B2A1106D110F8012B03E010F8016BAE
:107A000001F8016B5B1EF9D12B0705D40023521E30
:107A10000DD401F8013BFAE710F8013BCB1A921C98
:107A200003E013F8015B01F8015B521EF9D5A14296
:107A3000D8D3002070BD00002CB5294800F080F894
:107A400028480078002847D100BF274A012127484D
:107A500002F078F80546D5B125482649264A891A04
:107A6000C9080322CDE9000542EA014040F215238E
:107A700022A228A107F040F906F078FF00BF00BF5E
:107A800024B100BF204601F08FFD00BF00BF00BF42
:107A900000BF284A0021284802F054F80546D5B115
:107AA00026481449144A891AC9080322CDE9000559
:107AB00042EA014040F2162310A216A107F01CF979
:107AC00006F054FF00BF00BF24B100BF204601F004
:107AD0006BFD00BF00BF00BF0120024908702CBD34
:107AE000C5950200652D0020098302001C49030092
:107AF000044E030098590300005903007372635C3D
:107B00006170705F626C655F736572766963652E24
:107B10006300000025733A2564205A4552524F52A3
:107B20005F434845434B28257329206661696C3AB9
:107B300025640000CD820200204903005C4E030052
:107B400004490A680968491C024B1960024941F856
:107B500022007047D02D00201456002010B5034A93
:107B60000121034801F0EEFF10BD0000619D0200FD
:107B70002449030010B500BF00220649064808F05A
:107B8000F1F8044624B100BF204601F00DFD00BF0E
:107B900000BF10BD38490300F82D002010B5044681
:107BA0006CB10949088900EBD0714910074A11806E
:107BB000022301220649074808F076F903E0012173
:107BC000044808F0B3F910BD38490300002E002026
:107BD00028490300F82D002010B504460B48047016
:107BE0000B48006802F027F800200A49086007489F
:107BF000007818B90020FFF7D1FF06E0002240F618
:107C00009A110348006801F0E7FF10BD082E00201C
:107C1000244903000C2E00202CB5002109200CF073
:107C20004DFE00BF114A0121114801F08BFF0546AE
:107C3000CDB110481049114A891AC9080322CDE96B
:107C4000000542EA01402B230DA215A107F054F8CC
:107C500006F08CFE00BF00BF24B100BF204601F03B
:107C6000A3FC00BF00BF00BF2CBD0000C17C020010
:107C700044490300544F030098590300005903007E
:107C80007372635C626F6172645C626F6172645F85
:107C90006C696768745F6374726C2E630000000027
:107CA00025733A2564205A4552524F525F43484546
:107CB000434B28257329206661696C3A25640000CE
:107CC00010B504462348007830B92348007808B33B
:107CD000002000F075F836E01E480078012806D133
:107CE0001D480078B0B9012000F06AF82BE019486F
:107CF0000078022827D119480068022818DA1749A5
:107D0000086800EBD0714910A0EB410119B90120BE
:107D100000F056F817E01149086800EBD0714910DF
:107D2000A0EB410101290ED1002000F049F80AE042
:107D30000A48006864214843B0F57A7F03DB0020DD
:107D40000649086010BD05480068401C03490860EA
:107D500000BFF7E7102E0020112E0020142E002067
:107D60000148007870470000102E002010B504462E
:107D70001148047024B1012C0AD0022C18D10FE054
:107D80000E48006801F057FF002000F019F810E0DD
:107D90000A48006801F04FFF012000F011F808E0E8
:107DA000002240F266610548006801F015FF00E01E
:107DB00000BF00BF10BD0000102E0020444903008A
:107DC00038B504468CB109200090684606F0F2FBF5
:107DD00005460121009A01FA02F0C5F8080500BF26
:107DE00000BF01200A49087010E009200090684691
:107DF00006F0E0FB05460121009A01FA02F0C5F801
:107E00000C0500BF00BF00200149087038BD00000C
:107E1000112E002010B520480078022800D110BD96
:107E200001221EA1002004F027FB002004F00EF820
:107E300000221146052006F03FFB002211460B20D0
:107E400006F03AFB00221146112006F035FB002215
:107E50001146042006F030FB01211E2006F056FCDE
:107E6000642005F0FDFF00211E2006F04FFC0021DC
:107E7000012006F04BFC00211C2006F047FC1E20D0
:107E800005F0EEFF01211C2006F040FC0220024913
:107E9000087000BFC3E70000382E0020000000007B
:107EA0002DE9F84357480078012801D1BDE8F8834F
:107EB00001211E2006F02AFC0121084606F026FCBE
:107EC0001E2005F0CDFF00211E2006F01FFC01241E
:107ED0004FF00A0805E0002003F054FE0446A8F124
:107EE0000108B8F1000F01D0002CF4D1002C25D0EE
:107EF0004549464A891AC908032242EA01402246F6
:107F000043A106F0C9FE00BF49A03F493F4A891A74
:107F1000C9080322009042EA01409A2345A24DA1DC
:107F200006F0D6FE06F022FD00BF4FF0000800BFAD
:107F3000002001F039FB00BF00BF00BF3249334AC7
:107F4000891AC908032242EA014048A106F09AFEB4
:107F500001224EA14E4804F08FFA0546002D24D090
:107F600029492A4A891AC908032242EA014049A13B
:107F700006F088FE00BF2EA02349244A891AC908AA
:107F80000322009042EA0140A1232AA231A106F077
:107F90009FFE06F0EBFC00BF4FF0000800BF002082
:107FA00001F002FB00BF00BF00BF3E48006841690E
:107FB0003C48884740684FF48011B1FBF0F63948DF
:107FC00000684169374888470068B0FBF6F70E49FA
:107FD0000E4A891AC908032242EA014032A106F07A
:107FE00051FE0949094A891AC908032242EA014097
:107FF0003A4631A106F050FE01200249087000BF48
:1080000054E70000382E002098590300005903005F
:108010004469736B20696E697469616C697A617413
:10802000696F6E206661696C65642E2025640000AE
:10803000300000007372635C626F6172645C626F37
:108040006172645F7364636172645F6472697665B0
:10805000722E630025733A2564205A4153534552CA
:108060005428257329206661696C00004469736B8C
:1080700020696E697469616C697A6174696F6E20D8
:108080007375636365656465642E0000000000001D
:108090003C5600204D6F756E74206661696C656496
:1080A0002E000000504903004D6F756E74207375EB
:1080B0006363657373000000436170616369747981
:1080C0003A202564204D42000148007870470000A6
:1080D000382E002010B51E48007800B110BD0022D7
:1080E0001146052006F0E8F9002211460B2006F0A3
:1080F000E3F900221146112006F0DEF900221146B4
:10810000042006F0D9F903211C200CF0D7FB012133
:108110001C2006F0FBFA032101200CF0CFFB00210C
:10812000012006F0F3FA03211E200CF0C7FB00210A
:108130001E2006F0EBFA00200649087001210648CF
:1081400003F06EFF01200249087000BFC6E700007F
:10815000392E0020382E00203C2E002001480078C7
:1081600070470000B82D00202DE9FC4700260020B4
:10817000009001904FF480770125002410E03846EC
:1081800006F0FAFA40B100BF25480068284018B14F
:10819000384606F0E3FA2E436D00381D87B2641CA2
:1081A000082CECD34FF4BE7006F0E6FA50B14FF451
:1081B000BE7006F0D3FA46F000466A46022100205F
:1081C00006F0B4F9F0B210B3012500241DE005EA71
:1081D0000600C0B100BF134850F82400C0F30520CA
:1081E000814600BF0F4850F82400C0F3014082468A
:1081F000204602F0B3FE8046B8F1000F02D051468F
:108200004846C04700BF6D00641C082CDFD306F051
:10821000004010B1684608F07DFEBDE8FC87000014
:10822000046300401065004010B54FF4807005F005
:10823000FBFD50B14FF4807005F0FFFD012005F00B
:1082400005FE0A480168002088474FF4827005F057
:10825000EBFD50B14FF4827005F0EFFD022005F008
:10826000F5FD024801680120884710BD582E002006
:1082700010B50249024804F09BFF10BD682E002093
:1082800000C0014010B5034A1068034A11688847CE
:1082900010BD0000B82E0020B42E002010B504221E
:1082A0000021024804F0D6FF10BD0000004002404B
:1082B00010B50020034908700348006801F0BBFCBA
:1082C000002010BD642D00201C49030010B5044699
:1082D0000248006800F004F810BD0000602D002086
:1082E00070B50546074C07266A20A0700020607014
:1082F00003202070C4F80350314620460CF00DF9DD
:1083000070BD00000C5000202DE9FC4E81466548F0
:10831000007808B9BDE8FC8E6348006800284AD19F
:108320004FF480716148FFF785F84FF480725F4920
:108330005F48006800F0C2FA8246BAF1000F36DCEE
:108340005C495D4A891AC908032242EA01405BA1DF
:1083500006F098FC00BF60484FF4F67102685F4871
:10836000006801F039FC8346BBF1000F1BD05C486C
:108370005049514A891AC9080322CDE9000B42EA43
:108380000140C42357A25DA106F0B6FC06F0EEFA48
:1083900000BF00BFB8F1000F04D000BF404601F09D
:1083A00003F900BF00BF00BFFFF782FFB2E73E48FE
:1083B000C0F800A000BF3C48006800B9AAE70BF075
:1083C00089FE0546802D01DA284600E0802005461A
:1083D00035480068C0F58070344946183248006856
:1083E000A84201DD284601E02F48006807463149D0
:1083F000314A891AC908032242EA01402A490095F4
:108400003A460B6845A106F063FC0CF051F960B9DF
:108410002849294A891AC908032242EA014043A18E
:1084200006F030FCFFF744FF74E7B8B2019001A9F1
:1084300030460CF019F8044600BF0CB3082C0CD1E0
:108440001C491D4A891AC908032242EA01403FA17A
:1084500006F018FCFFF72CFF5CE7112C01D0132C61
:1084600000D157E71349144A891AC908032242EA7E
:10847000014022463DA106F00FFCFFF719FF49E736
:10848000002006E0315C144A12681144124A11605F
:10849000401CB842F6D304480068C01B024908607B
:1084A00000BF37E7642D00205C2D002030520020F3
:1084B000582D00209859030000590300726561642B
:1084C0002066696C6520656E642C73746F7020750E
:1084D000706C6F6164000000602D00202049030073
:1084E000E04E03007372635C6170705F626C655F85
:1084F000736572766963652E6300000025733A2503
:1085000064205A4552524F525F434845434B2825F9
:108510007329206661696C3A2564000075706C6F80
:10852000616420256420256420256400626C652038
:10853000697320646973636F6E6E65637465642C20
:1085400073746F702075706C6F616400626C65206D
:10855000756E656E61626C65206E6F746966792CEC
:1085600073746F702075706C6F616400626C65204D
:1085700073656E64206572726F722C73746F7020F5
:1085800075706C6F6164202578000000FEB54FF4B3
:10859000827006F071FE002837D04FF4827006F02A
:1085A00075FE6C4890F82E0018B16A4890F82F00BC
:1085B00058B300208DF80000664840680190654877
:1085C0000189ADF80810C06818B900206149087425
:1085D00012E06048008B5F4948830846C0684860E5
:1085E0000846008B08810020C860084690F82E00DD
:1085F00010B9002006F056FE5648016868468847C4
:108600000020544981F82F0000BF524890F82E00F6
:10861000002852D04FF4807006F02EFE00284CD077
:108620004FF4807006F032FE4A48408B494991F879
:108630002D10884216DD4748408B464991F82D1091
:10864000401A444948830A4612890B465B8BD21A6A
:108650000B465B6803EB42000A4692F82D1006F0C9
:1086600003FE23E03B48408B3A4991F82D108842A5
:108670000FD13848C06860B10120364981F82F0019
:10868000002048830A4692F82D10D06806F0ECFDD1
:108690000CE03048408B2F4991F82D10884205D1CD
:1086A00001202C4981F82F00002048834FF482706C
:1086B00006F0ECFD042006F0F5FD4FF4887006F09E
:1086C000DBFD70B14FF4887006F0E0FD0020214919
:1086D000087402208DF80000084601686846884743
:1086E00000BF4FF48A7006F0C7FD38B14FF48A70AE
:1086F00006F0CCFD0020174908742AE015484569AA
:1087000024E0B5FA85F64FF00040F0408543B00014
:1087100000F58C74204606F0AFFDB8B1204606F097
:10872000B5FD01208DF80000A4F58C70C0F3C700E2
:108730008DF80400A4F58C70012121EA90018DF8D8
:108740000510044801686846884700BF002DD8D14D
:1087500000BFFEBDE059002010B500F055FA10BD75
:108760002DE9F047074688461646C24607EB470103
:108770001B4800EBC109D9F8140020B1012811D021
:10878000022826D11EE0484600F076FA0546B5429A
:1087900001D2002405E0344632465146484600F0F6
:1087A000B2FA18E0484600F067FA0546B54201D231
:1087B000284600E03046044622465146484600F02E
:1087C000A2FA08E032465146484600F063FA0446F1
:1087D00001E0002400BF00BF2046BDE8F087000094
:1087E0005079002010B50249024804F0CFFC10BDBA
:1087F000105A00200030004010B503494FF04020CF
:108800000BF07EF810BD0000785A002010B5024928
:10881000024804F0BBFC10BD345A00200030024076
:1088200010B506F043FF10BD10B50949094A891A71
:10883000C908032242EA014007A106F023FAFFF724
:1088400043FC012801D108F0A5FDFFF7E3FA10BDB4
:1088500098590300005903006368616E67652074CE
:108860006F20657874206D6F6465000010B507494E
:10887000074A891AC908032242EA014005A106F005
:1088800001FAFFF70DFB08F085FD10BD98590300B4
:10889000005903006368616E676520746F206C6F18
:1088A00063616C206D6F64650000000010B5FFF718
:1088B00011FCFFF7DBFFFFF7B7FF10BD2DE9FC410F
:1088C00080460D46164600BF21480078002817D183
:1088D00020A02349234A891AC9080322009042EAAA
:1088E00001408F2320A229A106F0F2F906F03EF8FC
:1088F00000BF002700BF002000F056FE00BF00BFF1
:1089000000BF01AB32462946264803F0DAFE044692
:1089100000BF002C17D024A01149124A891AC90897
:108920000322009042EA014092230FA217A106F011
:10893000CFF906F01BF800BF002700BF002000F0B1
:1089400033FE00BF00BF00BF0198BDE8FC810000FE
:10895000882D00206D5F69735F6F70656E00000089
:1089600098590300005903007372635C73616D7062
:108970006C655F646174615F6D616E616765725F94
:10898000736572766963652E6300000025733A256E
:1089900064205A4153534552542825732920666157
:1089A000696C0000DC53002066665F726573756C4D
:1089B00074203D3D2046525F4F4B00000148024964
:1089C000086070470090D003602F002010B504F0BD
:1089D000E5FF40B10020644908604FF08041C1F8D4
:1089E00010016249086004F0F3FF002855D0604888
:1089F0000068604908605E48001D0068091D086045
:108A00005B4808300068091D086059480C30006850
:108A1000091D0860564810300068091D0860544858
:108A200014300068091D0860514818300068514929
:108A3000203108604E481C300068091D08604C4811
:108A400020300068091D0860494824300068091D6D
:108A50000860474828300068091D086044482C30E9
:108A60000068091D086042483030006841494031C3
:108A700008603F4834300068091D08603C483830C1
:108A80000068091D08603A483C300068091D08600C
:108A9000374840300068091D086004F04BFF40B1C2
:108AA0003548006800F0010018B16FF0010032494C
:108AB00008603248006840F470003049086000BF28
:108AC00000BF00BFBFF34F8F00BF00BF00BF00BF9C
:108AD00000BF00BFBFF36F8F00BF00BF00BF00BF6C
:108AE00004F042FF20B12648006820492031086088
:108AF00000BF2348001D006800F0010080B3012082
:108B000007F044FC1E48001D006820F001004FF0F3
:108B10001021C1F80C0207F043FC002007F036FCDE
:108B200000BF00BF00BF00BF00BFBFF34F8F00BF3B
:108B300000BF00BF11487C38006800F4E0601149B4
:108B40000843001D0D497C39086000BF00BF00BF0D
:108B5000BFF34F8F00BF00BF00BF00BF00BFFDE7E6
:108B6000FFE7FFF72BFF10BD0C0100403805004068
:108B70000404001020C500400004004088ED00E01F
:108B8000081200100000FA0510B50422024903483B
:108B900004F0BCFB10BD0000B45A0020008000406F
:108BA00010B504220249034804F0B0FB10BD0000D8
:108BB000C05A00200090004010B502490868804764
:108BC00010BD0000602E002008B500BF4FF480707B
:108BD0000B49405808B1012000E0002078B1094855
:108BE0000068804700BF00204FF48071044A88501D
:108BF000084611464058009000BF00BF00BF08BDA6
:108C000000000140742E002010B5124C022020619B
:108C1000606111A0A0611349E1614FF4007121620C
:108C20000021A1626162E1620BA0A0640E49E164CF
:108C3000102121650021A1656165E1650BA1E01DA1
:108C4000FEF717FC0AA12046FEF713FC2020A071B6
:108C500010BD0000387900205465726D696E616C3A
:108C600000000000B0790020B07B00205254540076
:108C7000534547474552000010B501460A69CB6885
:108C80009A4204D88C68641EE41AA01801E0D41A31
:108C9000601E10BD2DE9F0470446894617464FF087
:108CA000000AE56800BFD4F81080A84503D9A8EBF6
:108CB0000500461E04E0A5EB0800401CA1680E1A42
:108CC000A068401BB04201D9304601E0A068401BBB
:108CD0000646BE4201D2304600E03846064661688C
:108CE000481932464946FEF78CFBB244B144BF1BDB
:108CF0003544A068A84200D10025E560002FD2D1FC
:108D00005046BDE8F0872DE9F047044689461546F0
:108D1000E668A068871BAF4208D9616888192A46AF
:108D20004946FEF76EFB7019E06010E0B8466168D6
:108D3000881942464946FEF764FBA5EB070809EB94
:108D4000070142466068FEF75CFBC4F80C80BDE892
:108D5000F08702E008C8121F08C1002AFAD1704744
:108D60007047002001E001C1121F002AFBD17047AB
:108D70000146202908DA012088400A4A104008B13B
:108D8000012070470020FCE7402909DAA1F120000A
:108D9000012202FA00F008B10120F2E70020F0E71A
:108DA0000120EEE7FC06FFBD00BFEFF3108108468F
:108DB00072B670470246002104E0505C08B1012001
:108DC0007047491C0629F8D30020F9E7FEB5FF20BB
:108DD0008D49C870142088700F20487029200870B1
:108DE000C00788600320087300BF00231A46874825
:108DF00005F05AF90546002D19D085A09049914AF1
:108E0000891AC9080322CDE9000542EA01408623F8
:108E10008DA294A105F070FF05F0A8FD00BF00BF72
:108E200024B100BF204600F0BFFB00BF00BF00BF61
:108E3000002103200BF042FD00211D200BF03EFD20
:108E4000032005F03CFC1D2005F039FC8D488E49BF
:108E50000860002048608D488D4908600120486006
:108E60008849894800F010FA8849894800F00CFACE
:108E70004021854800F00AFA06467149714A891A6C
:108E8000C908032242EA0140324682A105F004FFEC
:108E900040217F4800F0FAF906466949694A891A73
:108EA000C908032242EA0140324680A105F0F4FEDF
:108EB00000221146744800F023FA0020029002AB11
:108EC0004122804980A00AF0A9FCBDF808000028D2
:108ED00037DD5B495B4A891AC908032242EA01402F
:108EE0007BA105F0CFFE82227F497648FEF7B4FAD7
:108EF00050B15349534A891AC908032242EA014032
:108F00007AA105F0BFFE09E04D494E4A891AC90809
:108F1000032242EA01407EA105F0B4FE00240BE0EA
:108F2000684800EB44004278664810F81410564830
:108F300000F0F6F9601C84B2BDF808008442EFDB53
:108F40000FE000240BE0684800EB440042786648DC
:108F500010F814104C4800F0E3F9601C84B2412C66
:108F6000F1D302AB4122714971A00AF057FCBDF860
:108F70000800002837DD3249324A891AC90803221D
:108F800042EA01406CA105F07DFE822270496748EB
:108F9000FEF762FA50B12A492A4A891AC9080322FF
:108FA00042EA01406BA105F06DFE09E02449254A23
:108FB000891AC908032242EA01406FA105F062FE46
:108FC00000240BE0594800EB44004278574810F861
:108FD00014102F4800F0A4F9601C84B2BDF80800FA
:108FE0008442EFDB0FE000240BE0594800EB440023
:108FF0004278574810F81410254800F091F9601C89
:1090000084B2412CF1D3FEBDE82C002008490300B6
:109010006E72665F6472765F7370695F696E6974A1
:1090200028267370692C20267370695F636F6E66E3
:1090300069672C204E554C4C2C204E554C4C290029
:1090400098590300005903007372635C61647331C3
:109050003239335F73696D706C655F746573746505
:10906000722E630025733A2564205A4552524F529E
:109070005F434845434B28257329206661696C3A54
:1090800025640000B1920200B82B0020D9920200A2
:10909000C02B0020616473313239335F3020726538
:1090A0007669643A2025640A000000006164733127
:1090B0003239335F312072657669643A2025640A5B
:1090C0000000000088310020302E63666700000039
:1090D0006C6F616420302E6366672066726F6D204E
:1090E00066617466730A0000C82B0020302E636628
:1090F0006720697320646966666572656E742066B0
:10910000726F6D2064656661756C740A0000000002
:10911000302E6366672069732073616D652061730B
:109120002064656661756C740A0000000A320020D4
:10913000312E6366670000006C6F616420312E631E
:1091400066672066726F6D2066617466730A000040
:109150004A2C0020312E636667206973206469669B
:10916000666572656E742066726F6D2064656661F7
:10917000756C740A00000000312E63666720697305
:109180002073616D652061732064656661756C7420
:109190000A000000FEB505460C46002637260020D2
:1091A00000900190029009236A463146284600F05B
:1091B00043F89DF8000000049DF8011000EB012029
:1091C0009DF80210084420609DF8030000049DF8FB
:1091D000041000EB01209DF80510084460609DF824
:1091E000060000049DF8071000EB01209DF8081010
:1091F0000844A060FEBD70B505460C4600202070F6
:109200006070A070E07020716071A0710723224629
:109210001821284600F010F870BD000070B5044613
:109220000D4604480068401C024908600AF088FAAC
:1092300070BD0000E02C00202DE9F04105460E46EF
:1092400017461C46FF2C01DDFF2000E020460446A7
:1092500046F080080A4880F800802146401CFEF74E
:10926000E9F8601CC2B2074905482B6898472246B6
:109270000449491C3846FEF7C4F8BDE8F0810000F7
:10928000642F002064300020016070477CB50446E4
:109290000D4645F080008DF8040000208DF8050093
:1092A0000222694601A8236898479DF801007CBD09
:1092B000F8B504460D461646032005F051F92B4635
:1092C000324621460348009604F032FF032005F0A1
:1092D000F6F9F8BD08490300F8B504460D461646F0
:1092E0001D2005F03DF92B463246214603480096E5
:1092F00004F01EFF1D2005F0E2F9F8BD0849030047
:10930000F8B504460D46164605F07F008DF80000BE
:109310008DF8016002220021684623689847F8BD55
:10932000FEB506460C461546002002900295182C04
:1093300002DB1E2C00DCFEBD302C02DB3F2C00DCEF
:10934000F9E7402C00D1F6E7502C00D1F3E702AB4F
:109350002A462146304600F02FF89DF80800A84222
:109360000FD09DF80800CDE900500749074BC91AF6
:10937000C908012343EA0140234605A1726805F0AC
:10938000BBFC00BFD7E70000985903000059030059
:109390006164735F25642077726974652025782085
:1093A0006661696C65642C773A2578207265616422
:1093B00062616B3A25780A002DE9F04105460E46B8
:1093C00017461C463A4631462846FFF799FF314674
:1093D0002846FFF75BFF2070BDE8F0811CB5032035
:1093E00005F0BEF81D2005F0BBF800208DF8040044
:1093F00001208DF8050000200346022201A90090FB
:10940000044804F095FE032005F059F91D2005F0ED
:1094100056F91CBD0849030070B504460D4604F218
:109420002740FFF7C7FC0646012D06D0022D0DD0C0
:10943000032D11D0042D19D113E0A07928B194F88F
:10944000240010B90EB1012070BD00BFE07910B149
:109450000EB10220F8E700BF207A08B10320F3E73D
:1094600000BF607A08B10420EEE700BF0020EBE700
:109470000146481C052290FBF2F302FB1300C0B228
:109480007047014691F82420012A01D1EE2000E026
:109490001F20704710B501220221002001F064FC5A
:1094A000044600BF1CB1072C01D0204610BD00BFF0
:1094B00007220221012001F057FC044600BF1CB125
:1094C000072C01D02046F1E700BF0A220021084600
:1094D00001F04AFC044600BF1CB1072C01D0204615
:1094E000E4E700BF0020E1E710B572B600BF05F069
:1094F000B7FC00BF00BF05F039FA0028FBD100BF60
:1095000000BF1E491E4A891AC908012242EA0140C9
:109510001CA105F0B7FB00BF1D48006800F001006A
:1095200000B100BE00BF1549154A891AC9080222B8
:1095300042EA014017A105F0A5FB00BF00BF00BF34
:1095400000BF00BFBFF34F8F00BF00BF00BF104878
:10955000E438006800F4E06012490843001D0C493B
:10956000E439086000BF00BF00BFBFF34F8F00BFEA
:1095700000BF00BF00BF00BFFDE700009859030017
:1095800000590300466174616C206572726F72004D
:10959000F0ED00E053797374656D20726573657446
:1095A000000000000000FA053EB5044600200090CF
:1095B0000190029002946A46002144F20100FFF7F4
:1095C00093FF3EBD70B505460E462C46207820B967
:1095D0006179207907F024FE1CE02078012807D16A
:1095E0000D480068401C0C490860FEF7B7FD11E00B
:1095F0002078092802D107F003FE0BE02078032829
:1096000008D10648007828B1042204F108016068F6
:1096100007F074FD70BD00007C2D0020112D00208E
:109620002DE9F84307460C469046264800888442B8
:1096300044DC4FF6FF7500200090684600F01EFBEA
:1096400000BF214890F800902048007804F04AF9C3
:10965000484501D1012000E0002030B91B480578C1
:10966000007804F03FF9194908709DF8000000F0F7
:109670000BFB4FF6FF7085421ED01548006840F87E
:1096800035808FB1002C0FDD124909680D4A128810
:1096900005FB021022463946FDF7B3FE0C48006870
:1096A00000EBC500848005E000200949096801EB52
:1096B000C5018880002600E0042600E00926304627
:1096C000BDE8F8838A2E0020882E0020892E0020F5
:1096D000802E0020842E00202DE9F0411AE016484B
:1096E0000478164800681649098804FB01051548E6
:1096F000006800EBC40086881248006850F8347097
:1097000031462846B8470C48007804F0EBF80A497F
:10971000087000BF00BF002058B900BF0649087894
:1097200009490978814201D1012100E00021002985
:10973000D5D0BDE8F0810000882E0020842E0020C6
:109740008A2E0020802E0020892E002030B503466E
:10975000481C4FF6FF7505EAC004104600F00305EB
:109760000DB9012500E000250DB9072030BD0848DE
:1097700002601019074D28600020074D2870074D22
:10978000287007480380074801800020EEE70000AA
:10979000802E0020842E0020892E0020882E00207C
:1097A0008A2E00208C2E00202DE9F04707460E4619
:1097B00014461F4890F8220010B90820BDE8F08731
:1097C0001B4890F82200032801D01120F6E70CB9BD
:1097D0000720F3E70421164880F82210807AC0F3AE
:1097E000C00018B971021248016101E01048066119
:1097F0000F48C7608482C48200218183012C01DD6F
:10980000522000E051208146094801220169484662
:1098100008F0BAF8054600BFA846B8F1000F04D01A
:1098200000BF4046FFF7C0FE00BF00BF0020C5E7F5
:109830009C5B00202DE9F04107460E4615462D4859
:1098400090F8220010B90820BDE8F081294890F86E
:109850002200032801D01120F6E70DB90720F3E715
:109860000521244880F82210807AC0F3C00018B97E
:1098700071022048016101E01E4806611D48C76071
:109880008582C58200218183012D12D101220169C7
:10989000582008F079F8044600BFA046B8F1000F40
:1098A00004D000BF4046FFF77FFE00BF00BF00208E
:1098B000CAE71048807A00F00700012807D10D4858
:1098C00001220169592008F05FF8044605E00122F1
:1098D0002946D72008F058F8044600BFA046B8F142
:1098E000000F04D000BF4046FFF75EFE00BF00BF80
:1098F0000020A9E79C5B0020064890F8220003287E
:1099000005D0044890F8220008B1012070470020DB
:10991000FCE700009C5B0020044890F8220003282C
:1099200002DB0248001D70470020FCE79C5B002022
:10993000F0B587B004460E463A4890F8220010B1C0
:10994000082007B0F0BD5EB1E078FF2808D060784D
:10995000FF2805D02078FF2802D0A078FF2801D169
:109960000720EEE7E0782F4981F85800084690F884
:10997000587000200090034601221146019038469D
:1099800004F057FD00BF00BF264991F8580004F0CD
:10999000B0FE00BF244B0FCB03AD0FC5A0788DF8F0
:1099A0000C0020788DF80D0060788DF80E000023F3
:1099B0001E4A03A91E4804F077FB054600BF2F4648
:1099C00027B100BF3846FFF7EFFD00BF00BF1548C5
:1099D0000660012180F82210807A20F007011148EA
:1099E0008172807A20F008010E488172002180F88F
:1099F0002310FF200B4981F828000A2001F13803C9
:109A00000122283100900A4804F0ABFB054600BF54
:109A10002F4627B100BF3846FFF7C6FD00BF00BF85
:109A200000208EE79C5B0020184C0300C12E030031
:109A3000084C03007CB5144890F8220008B90820AF
:109A40007CBD114890F82200032801D01120F7E7CF
:109A50000E4C201D06F0FCFB00BF0B4890F8584050
:109A60000025002000902B4602460146019020462A
:109A700004F0DFFC00BF0021034880F8231080F8C9
:109A800022100020DCE700009C5B0020084C030053
:109A900010B50446022C0AD10C490D4A891AC9088E
:109AA000032242EA01400BA105F0ECF801E001209D
:109AB00010BD00BF0549064A891AC908032242EAB7
:109AC000014010A105F0DEF80120F1E798590300EC
:109AD00000590300506F776572206D616E61676594
:109AE0006D656E742077616E747320746F2072657B
:109AF00073657420746F20444655206D6F64652E25
:109B000000000000506F776572206D616E616765BF
:109B10006D656E7420616C6C6F77656420746F2066
:109B2000726573657420746F20444655206D6F64B0
:109B3000652E000010B5024802F0CEFA10BD0000FC
:109B4000902E002030B503460C460AB9072030BDE0
:109B500019684FF0FF358D60CD604A61012C01D14D
:109B6000012000E0002008610020F0E738B513482C
:109B7000006800900823A82211491248006803F0E9
:109B800041FF04460CB1204638BD0F4A69460F48D4
:109B900002F0A8FA04460CB12046F5E701210B4873
:109BA00002F046FB01230A4A1946084802F066FA09
:109BB0000120084908702046E6E70000284A030013
:109BC000CC5A0020184A0300F1150300902E002003
:109BD000FFFF7F009C2E00202DE9F84306460D462E
:109BE0009046344600200090684600F047F84FF059
:109BF000FF33D4E9021059405840014308D103F023
:109C0000FFF9401941F10001C4E90201012700E018
:109C100000279DF8000000F037F817B90020BDE8D4
:109C2000F883C4F81880206900B12561214600201E
:109C300009F064FDF3E7F8B50446254600200090DE
:109C4000684600F01BF84FF0FF33D5E90210594089
:109C50005840014301D1002604E04FF0FF31A960D4
:109C6000E96001269DF8000000F00EF80EB9002012
:109C7000F8BD2946012009F041FDF9E710B5044679
:109C8000204607F0D1FD10BD70B5044625460E48AC
:109C90008068B0B1ADB9FFF787F806460A4800689A
:109CA0000A490860084840684FF0E021C1F8040103
:109CB0000020054988601EB900BF62B600BF00BF22
:109CC00000BF00BF70BD0000845B002000E100E029
:109CD000F8B505460C4617462088001DB84201D944
:109CE0000C20F8BD684679DF064600BF304600B15B
:109CF000F7E700BF0320218868542088401C20809B
:109D00001920218868542088401C2080208841190F
:109D1000BDF800000AF06BF821880844208000207C
:109D2000DFE70000002113E00C480269012308E08E
:109D300000BFD0680079884201D1002303E0D068D9
:109D40000268002AF4D100BF0BB108467047491CD5
:109D50000A29E9DB4FF0FF30F8E70000187900200E
:109D600010B504463948007818B90020FDF716FFF1
:109D700064E036480078012815D13548006818B9E4
:109D80000120FDF70BFF59E031480068002855D04D
:109D90000020FDF703FF2F480068FFF74CFF00206D
:109DA0002A4908704AE029480078022820D128482A
:109DB0000068062811D22648007800F0010018B982
:109DC0000120FDF7EBFE39E02148007800F00100AA
:109DD00038B30020FDF7E2FE30E00020FDF7DEFEA4
:109DE0001C480068FFF727FF00201849087025E08D
:109DF00016480078032821D115480068062811D29A
:109E00001348007800F0010018B90120FDF7C6FEE4
:109E100014E00F48007800F0010010B10020FDF7B9
:109E2000BDFE0BE00A4800689621484342F21071DB
:109E3000884203D300200649086010BD044800682A
:109E4000401C0349086000BFF7E70000082E00200F
:109E50000C2E0020244903002DE9FC4105468846CC
:109E60001646002437880020308095F82D0058B120
:109E70003A463146404600F095FA044600BF204677
:109E800008B1BDE8FC8100BFA87850B13A46314620
:109E90004046FFF71DFF044600BF204600B1F0E733
:109EA00000BFE87860B1E97848B23B4632464146A7
:109EB00002F0E6FE044600BF204600B1E1E700BF25
:109EC000686868B1696891F900003B4632464146CE
:109ED00009F06CFF044600BF204600B1D1E700BF87
:109EE000288900280EDD43460622022105F10800DC
:109EF000CDE900670AF027F8044600BF204600B10C
:109F0000BFE700BF288A00280EDD43460722032151
:109F100005F11000CDE900670AF015F8044600BF0E
:109F2000204600B1ADE700BF288B00280EDD434678
:109F30001522142105F11800CDE900670AF003F895
:109F4000044600BF204600B19BE700BF286A58B115
:109F50003B4632464146286A01F091FA044600BF6A
:109F6000204600B18DE700BF686A58B13B463246D3
:109F70004146686A03F054FB044600BF204600B126
:109F80007FE700BF95F82C0000280BDD3B463246EA
:109F90004146284608F0B6FC044600BF204600B102
:109FA0006FE700BF287858B13B4632464146284605
:109FB00003F034FC044600BF204600B161E700BF57
:109FC00020465EE7F8B504460E4615460020009090
:109FD0002B466A463146204600F008F807460FB97E
:109FE0000020F8BDBDF800002044FAE7F0B50446B3
:109FF0000D461E4604B10AB90020F0BD002103E061
:10A00000605C401C084481B2481CA84206DA1088F3
:10A010008842F5DC481C205CB042F1D1A94201DB4A
:10A020000020EAE7881C87B2605C10B1605C401ECB
:10A0300000E0002083B213B1F818A84201DD00202F
:10A04000DBE717801846D8E780F83010704770B506
:10A0500004460D4605B10CB90E2070BD05F178001F
:10A0600001F042F908B90720F7E70020A0702C2280
:10A0700005F17801201DFDF7C4F9002084F83000B7
:10A08000D5F8A4006063D5F8A800A0634FF6FF7070
:10A09000A4F8240404F58260C4F82004002140F2EE
:10A0A0002C40C4F82614A4F82A140155207810B9BD
:10A0B000FF2084F8540004F15500C4F81004204631
:10A0C000FFF7DFF940F21441085304F2144204F19F
:10A0D00055012846FFF7C0FE064600BF304600B1D6
:10A0E000BBE700BF04F231204FF4836108512046E2
:10A0F000FFF7C7F9A4F81C044FF48360015904F278
:10A100001C4205F13C00FFF7A7FE064600BF3046A3
:10A1100000B1A2E700BF012151200155208B81B27F
:10A1200048200153012084F83C0000212164502084
:10A1300001556169616404F13C02002104F154009D
:10A1400072DF064600BF304600B186E700BF01203F
:10A150002070304681E770B504460D462E462088B3
:10A16000102804D0112807D026280FD109E0214655
:10A17000304606F06DFA0AE02146304606F064FCEF
:10A1800005E02146304606F0E7FD00E000BF00BFD5
:10A1900070BD70B504460E46207808B9082070BD21
:10A1A000A670002140F22C40C4F82614A4F82A140A
:10A1B0000155A07910B1A078012809D0E07910B13B
:10A1C000A078012804D0E07970B1A07802280BD1E2
:10A1D000606B30B1012084F82D040820616B884742
:10A1E00002E0002084F82D0431462046FFF714F9E0
:10A1F000A070606BA0B1A078032802D0A0780428DA
:10A200000ED1607960B194F82E0448B9002084F82A
:10A210003004012084F82F040720616B884702E096
:10A22000002084F82F04182104F13C00FDF702F906
:10A23000012084F83C0004F12C0006F01CFE20B143
:10A2400094F82C105120015502E0012151200155B4
:10A2500094F8240060B104F1280006F00CFE20B14F
:10A2600094F828105220015502E001215220015596
:10A27000002150200155A078052824D2DFE800F005
:10A280001F030A11180004F13C01204608F09DFB51
:10A29000054619E004F13C01204608F07EFB054626
:10A2A00012E004F13C01204608F0A1FB05460BE05A
:10A2B00004F13C01204608F0C8FB054604E00020FC
:10A2C00084F8310000E000BF00BFA07898B104F12D
:10A2D0003C0204F15400D4F8201472DF05460DB19D
:10A2E00028465CE794F8301094F8540073DF054674
:10A2F0000DB1284653E7606B18B194F83100616BDB
:10A30000884700204BE700002DE9F041044600BFDC
:10A3100014B90E20BDE8F08100BF1C2221461C4864
:10A32000FDF76FF81B481A490860206860B1206883
:10A330007ADF05460DB12846ECE7164821680A6821
:10A3400002604968416005E012487BDF05460DB1B7
:10A350002846DFE7002617E006EB86000E4901EBF2
:10A36000800700BF4FF6FF70388000BF0B4800EB3E
:10A37000461078600A4A0021381DFFF7E3FB0546C6
:10A380000DB10320C6E7761C002EE5D00020C1E702
:10A39000CC580020502E0020B8580020985800209B
:10A3A000B53E03002DE9FC4105460C4617462088C2
:10A3B0000930B84202D90C20BDE8FC8168466DDF47
:10A3C000064600BF304600B1F6E700BF08202188EE
:10A3D00068542088401C20801B20218868542088D5
:10A3E000401C208020882844DDF801100160BDF861
:10A3F000051081802088801D20809DF80000400885
:10A4000018B900202188685402E00120218868548E
:10A410002088401C20800020CEE7000070B503F0AB
:10A4200037FD044600BF204600B170BD00BF00BF2D
:10A43000084D28464FF0030C00DF00BF044600BF64
:10A44000204600B1F1E700BF03F09CFD0446204622
:10A45000EBE700002480002010B51349134A891A45
:10A46000C908042242EA014011A104F00BFC4FF09C
:10A47000FF3100203DDF044600BF204600B110BD83
:10A4800000BFB12100203CDF044600BF204600B1E0
:10A49000F5E700BF1348416901208847022004F016
:10A4A0005FFE0020EBE7000098590300005903000D
:10A4B000496E20626C655F6466755F627574746F67
:10A4C0006E6C6573735F626F6F746C6F61646572DD
:10A4D0005F73746172745F66696E616C697A650D31
:10A4E0000A0000000880002010B505480068416996
:10A4F00000208847FFF7B0FF0446204610BD00004B
:10A500005C2F002070B504460D4600BF04B970BD35
:10A5100000BF2088102806D0112808D051280AD062
:10A52000532810D10BE0204606F08CF80CE02046B2
:10A5300006F07CFA08E0204606F0ECFB04E020463A
:10A5400006F0C4FB00E000BF00BF00BFDFE7000073
:10A5500070B504460426207B012802D0022822D1AF
:10A5600009E001F003FF05460DB9012602E0112DB7
:10A5700000D1062619E0607B142801DC607B08B955
:10A5800005260FE0627B04F10E011248FCF739FF4B
:10A59000607B1049091F8861084608F085FA054666
:10A5A00005B9012601E0022600BF00BF012E0FD031
:10A5B000207B314600F058F8054625B10648006872
:10A5C00041690320884704480068416902208847A0
:10A5D00070BD0000348000205C2F002070B505465F
:10A5E0000E4600BF1E48006820B11D48406808B1F3
:10A5F000012000E0002000B970BD00BF184800F144
:10A600000801426828469047044600BF082C24D021
:10A610007CB900201349096848760121022000F026
:10A6200023F80446CCB10F480068416903208847ED
:10A6300013E000200B49096848760621022000F04B
:10A6400013F8044624B1074800684169032088478D
:10A650000448006841690220884700BFCCE7000039
:10A66000248000205C2F0020F0B587B004460D4602
:10A67000032700200190029003900490032006908D
:10A6800020208DF814008DF815408DF816500E48D6
:10A69000C088ADF8040002208DF806000020ADF857
:10A6A000080006A8039005A804900749888801A916
:10A6B000AEDF064626B9BDF81800032800D00C26E8
:10A6C000304607B0F0BD00000880002070B5054698
:10A6D0000E462888102802D011282CD115E01748E2
:10A6E000006860B900F032FF044600BF34B114487E
:10A6F000006818B1204612490968884700BF0F4812
:10A700000068401C0D49086016E00C480068401EB7
:10A710000A4908600846006860B9FEF7BBFE0446B7
:10A7200000BF34B10648006818B1204604490968E2
:10A73000884700BF00E000BF00BF70BD4C2E002066
:10A74000482E002070B504460D462088102806D0FB
:10A75000112808D012280ED0502810D107E020462A
:10A7600005F038FF0CE0204606F046F908E02046E8
:10A7700006F012FB04E0204605F014FF00E000BFE5
:10A7800000BF70BD2DE9F04104460F46A688208821
:10A79000102806D0112817D019283DD01A2848D1E2
:10A7A00016E006F09FFE304606F078FE20B900BFA6
:10A7B0000420FEF7F9FE06E0E07B022803D13146D3
:10A7C0001D4803F089F934E0304606F0AFFE30E072
:10A7D000207A0509042D01DB012000E0002002465B
:10A7E000314615480C3002F03CFA032D01DB012004
:10A7F00000E00020024631460F48083002F031FAEE
:10A80000022D01DB012000E00020024631460A480B
:10A81000001D02F026FA0CE0207A48B9607AC0F3F5
:10A82000C0052A46314604480C3002F01AFA00BF2F
:10A8300000BF00BFBDE8F081F45800202DE9BE4103
:10A8400005460F46288821282BD006DC10280BD07F
:10A85000112817D013287DD154E03B287BD05228F3
:10A860007BD05628F7D1C5E0A88877490880012019
:10A87000764908707648006818B108467449096836
:10A880008847DDE04FF6FF706F49088002206F496E
:10A8900008706F48006818B108466D490968884714
:10A8A000CEE06C496C4A891AC908042242EA014088
:10A8B0006AA104F0E7F900200290A88802A98FDFBE
:10A8C000044600BFA046B8F1000F19D068A0614946
:10A8D000614A891AC9080322CDE9000842EA014009
:10A8E000462366A26DA104F007FA04F03FF800BF0A
:10A8F00000BF26B100BF3046FEF756FE00BF00BFC6
:10A9000000BF9DE000231A4685214F4800887FDF65
:10A91000044600BFA046B8F1000F19D054A04D491D
:10A920004D4A891AC9080322CDE9000842EA0140CC
:10A930004C2352A259A104F0DFF904F017F800BF2C
:10A9400000BF26B100BF3046FEF72EFE00BF00BF9D
:10A9500000BF75E073E028E0FFE700231A461946C0
:10A9600039480088B1DF044600BFA046B8F1000FA7
:10A9700019D03FA03749384A891AC9080322CDE9BE
:10A98000000842EA014052233CA244A104F0B4F979
:10A9900003F0ECFF00BF00BF26B100BF3046FEF75A
:10A9A00003FE00BF00BF00BF4AE0A888132176DF86
:10A9B000044600BFA046B8F1000F19D02CA02549CD
:10A9C000254A891AC9080322CDE9000842EA014054
:10A9D00058232AA231A104F08FF903F0C7FF00BF6A
:10A9E00000BF26B100BF3046FEF7DEFD00BF00BF4E
:10A9F00000BF25E0A888132176DF044600BFA046EB
:10AA0000B8F1000F19D01AA01249134A891AC908BF
:10AA10000322CDE9000842EA01405E2317A21FA1EC
:10AA200004F06AF903F0A2FF00BF00BF26B100BF27
:10AA30003046FEF7B9FD00BF00BF00BF00E000BF19
:10AA400000BFBDE8BE8100003C2F0020442F002045
:10AA5000402F002098590300005903005048592006
:10AA600075706461746520726571756573742E000C
:10AA70006572725F636F6465000000002E2E5C6C6F
:10AA800069627A6E6F726469635C7372635C7A6226
:10AA90006C655F6D6F64756C652E630025733A2578
:10AAA00064205A4552524F525F434845434B282534
:10AAB0007329206661696C3A2564000070B504460C
:10AAC000204609F08EF90546C5F3400070BD70B50B
:10AAD0000446204609F085F9054605F0010070BDE1
:10AAE00030B50246087A0B7833B1012B05D0022B22
:10AAF00005D0032B14D101E000BF00BF00BF4B788D
:10AB000000EB4004084D2D6805EB840423720023FC
:10AB100000EB4004044D2D6805EB8404A37200E0B3
:10AB200000BF00BF30BD00004C2F002001460A4688
:10AB3000906970472DE9FE4380460C469146454694
:10AB4000AE692869B0F5007F02D00620BDE8FE831B
:10AB50001648006808B11120F8E7C6F81890B460EC
:10AB6000124805600027124905F11400FEF7E0FEC7
:10AB700007464FB944B907F005FE0E48007808B9FA
:10AB8000002000E00D20074677B10020074908604B
:10AB900054B1094A07CA8DE80700B06902906946B6
:10ABA0004046B268904700BF3846CFE7D02E00201D
:10ABB000811A0300CC2E0020D84B030030B5034689
:10ABC0001D4611B101290ED105E014460CB100203B
:10ABD0002070002030BD0AB90720FBE71446281D6D
:10ABE00020600020F6E700BF00BF0620F2E700006B
:10ABF0002DE9FE4307460D46B846D8F81840002612
:10AC00001B480068404502D01120BDE8FE83FEF7D6
:10AC100073FE08B11120F8E795E80700C4E90412B3
:10AC2000E060AB889AB22968A868FEF7BDFD0646C9
:10AC300056B9A06840B907F0A5FD0E48007808B9DC
:10AC4000002000E00D200646A06870B16EB10A4AEF
:10AC500007CA8DE8070004F10C000190A06902907A
:10AC600069463846A268904700BF3046CDE70000ED
:10AC7000D02E0020CC2E0020F04B0300FEB506465F
:10AC80003746BD6913480068B84201D01120FEBDA7
:10AC9000FEF732FE08B11120F9E7FEF7CBFE0446BD
:10ACA00014B900200B490860A86880B10A4A07CA95
:10ACB0008DE807000CB1012000E000208DF80100B4
:10ACC000A869029069463046AA68904700BF2046AE
:10ACD000DDE70000D02E0020E44B03002DE9FE4309
:10ACE00007460D46B846D8F8184000261B480068AD
:10ACF000404502D01120BDE8FE83FEF7FDFD08B1FE
:10AD00001120F8E795E80700C4E90412E060AB8879
:10AD10009AB22968A868FEF78DFD064656B9A06864
:10AD200040B907F02FFD0E48007808B9002000E078
:10AD30000D200646A06870B16EB10A4A07CA8DE8B8
:10AD4000070004F10C000190A069029069463846A2
:10AD5000A268904700BF3046CDE70000D02E00200B
:10AD6000CC2E0020FC4B030030B503460020042B02
:10AD700023D2012A07D1012903D103F10E04E4B241
:10AD800000E00024224679B1012902D0022911D124
:10AD900004E003EB43040A4D2A550DE003EB4304A2
:10ADA000074D2C44627007E003EB4304044D2C4430
:10ADB000A27001E0072000BF00E0072030BD0000C6
:10ADC000885800202DE9FC4704460D461646A71C6E
:10ADD0004FF001080020019001A8FEF74FFF304816
:10ADE000406828602E4840682D498968411A2D48DE
:10ADF0000068401CA0EB010915E001212A4802F07F
:10AE000088FE02F041FB82465146274802F081FE4F
:10AE10002348406822498968411A22480068401C3A
:10AE2000A0EB010900BF4F45E7D8B8F1000F30D0C3
:10AE30000021009176B1009921F00301491C009195
:10AE4000009921F00401091D0091009964F3891112
:10AE500000910DE0009921F00301891C00910099F7
:10AE600021F00401091D0091009964F39F510091A4
:10AE70000B4949680B4A12681140094A0C3202EB2F
:10AE80008100009901600649496839440C3A5160D3
:10AE900000BF9DF80400FEF7F7FE4046BDE8FC87C2
:10AEA00018690020E82E00203479002070B504468F
:10AEB0000D460A2D03D10D212046FFF7F7FFA168AB
:10AEC000481CA06020684554D4E90110884202D390
:10AED000204603F074F970BD04488068034949684E
:10AEE000884201D1012070470020FCE7186900204A
:10AEF00070B504460D46032C06D1A920034908600D
:10AF000000BF002004F02CF970BD000020050040B7
:10AF100010B506490648FEF76EF906490648FEF7E1
:10AF20006AF90449014807F06FFC10BDCC2C0020E1
:10AF3000B82B0020D32C0020C02B00204FF0FF3175
:10AF4000054A42F82010082804DBFF23A0F108017D
:10AF50005A32535470470000785900200146024885
:10AF600050F8210070470000785900202DE9F04F7B
:10AF700003460C464FF0FF390AB1002000E00820DC
:10AF800084460AB1082000E00C208046614624E097
:10AF9000154850F82100401CF0B91D4608462746C8
:10AFA00016464FFA80FBDFF840A00AF1300A0AF893
:10AFB00005B0DFF834A04AF820704EB94FFA85FB8F
:10AFC000A0F1080ADFF820E00EF15A0E0EF80AB0E0
:10AFD00000BF4FFA81F902E0491C4145D8D300BFB8
:10AFE0004846BDE8F08F000078590020014601482E
:10AFF00040567047A859002070B590B006460C46E0
:10B000001546A07818B901208DF80E0002E0A0784E
:10B010008DF80E002088ADF80C0000200290607CB6
:10B0200002A907F071FDA07C0DF1090107F06CFD8C
:10B03000E07B08B1012000E000209DF80A1060F3D9
:10B04000C3018DF80A10207C08B1012000E0002027
:10B050009DF80A1060F304118DF80A10207B08B1E6
:10B06000012000E000209DF80A1060F300018DF837
:10B070000A10207D08B1022000E001209DF80A108E
:10B0800060F342018DF80A101C2109A8FCF7D2F9DF
:10B09000607BC0F3001018B9607BC0F34010F8B1BA
:10B0A00000200090E07C0DF1010107F02DFD00BFB4
:10B0B0009DF8000020F00F00401C8DF800009DF866
:10B0C000000020F0F00010308DF8000000BF9DF867
:10B0D000020020F00600801C8DF80200CDF838D068
:10B0E000607B8DF82400A07B8DF82500142104A836
:10B0F000FCF7A0F903A8049002A80590A088ADF879
:10B100001C00A06820B1E088ADF81800A068089085
:10B11000A069002849D000200190A0690088ADF8FE
:10B120002C00A0694088ADF82E00A06940680A9004
:10B1300001A80D90A169087B01A907F0E5FCA169B0
:10B14000487B0DF1050107F0DFFCA069807A08B1AA
:10B15000012000E000209DF8061060F3C3018DF887
:10B160000610A069C07A08B1012000E000209DF817
:10B17000061060F304118DF80610A069007A08B17A
:10B18000012000E000209DF8061060F300018DF81A
:10B190000610A069807B08B1022000E001209DF824
:10B1A000061060F342018DF80610E06908B1E0690D
:10B1B0000C902B4604AA09A93046AADF10B070BD36
:10B1C00070B504460D460020E070401EE06229463E
:10B1D000204602F009FB08B1042070BD04F22E20C5
:10B1E00002F033F94AF65521884201D00320F4E7F2
:10B1F00094F83000E92807D094F83000EB2817D1F4
:10B200003220005D902813D104F1660002F011F99C
:10B2100020F07F400749884201D10020DDE704F19A
:10B22000820002F006F90449884201D10020D4E7E7
:10B230000220D2E74641540046415433024600E022
:10B24000521C107810B110788842F9D110787047EC
:10B2500070B505460DB9094C01E0084C083409E009
:10B26000204602F0BAF8064606B904E0284671689E
:10B27000884700BFF4E700BF70BD00006C59002094
:10B2800010B504462CB90120064948700020FFF78C
:10B29000DFFF012C04D1012002498870FFF7D8FF9D
:10B2A00010BD0000645900200246891E5069801EAE
:10B2B000884201D8002070475389906A01FB03003F
:10B2C000F9E72DE9F047024613468C46D3E90245DB
:10B2D000DCE90267B6EB040877EB050002D3012036
:10B2E000BDE8F0870020FBE701468878012805D1FA
:10B2F00091F82000012801D1002070470120FCE7CF
:10B300002DE9F04F89B006460F46002458E03D5D18
:10B31000FF2D4ED0C5F3C010049025F0800005A984
:10B3200041F82400049880B105A850F82400039047
:10B3300003A803F07FF980460121039A01FA02F085
:10B34000C8F8080500BF00BF10E005A850F82400A9
:10B35000039003A803F06EF980460121039A01FAD5
:10B3600002F0C8F80C0500BF00BF00BF05A850F8E8
:10B3700024804FF00109CA464FF0000BCDE9018B44
:10B38000CDF80CB001A803F055F9009049EA4A0045
:10B3900040EA8B01029841EA0021039841EA00410A
:10B3A000009800F5E060019A40F8221000BF00BF4D
:10B3B00004E04FF0FF3005A941F82400601CC4B23E
:10B3C000042CA4DB05AA3168002007E052F82050C5
:10B3D00001F5AC6343F82050431CD8B20428F5DBD8
:10B3E00000BF09B0BDE8F08F33B58BB00546002033
:10B3F00000900C9878B100240BE021460CA802F0D4
:10B400005CFB28B1009A501C009001A820F8124063
:10B41000641C142CF1D32C2269462846FBF7F1FF5B
:10B420000DB030BD01460888062808DB0888B0F555
:10B43000486F06DD08884FF6FF72904201D0072062
:10B4400070474888062808DB4888B0F5486F06DD55
:10B4500048884FF6FF72904201D00720F0E7088835
:10B460004FF6FF72904208D04888904205D0088875
:10B470004A88904201DD0720E2E70020E0E72DE95D
:10B48000F04107460D46144698462088801D4045E9
:10B4900002D90C20BDE8F0813846FFF7C3FF06460D
:10B4A00000BF304600B1F5E700BF05202188685491
:10B4B0002088401C20801220218868542088401C4D
:10B4C000208022885119388808F091FC218808448E
:10B4D000208022885119788808F089FC2188084446
:10B4E00020800020D6E710B5044600BF2046FEF7B6
:10B4F0005BF800BF10BD0000F8B505460C46607A49
:10B5000088B9207A10B91048476801E00E4887686A
:10B510002A4639466068FEF75FFB064616B130469C
:10B5200007F090F90EE0002020720748406948B10A
:10B5300001208DF80000ADF80250034841696846CB
:10B54000884700BFF8BD0000CC58002010B501228C
:10B5500000210846FFF708FC044600BF1CB1072C79
:10B5600001D0204610BD00BF072202210120FFF7B5
:10B57000FBFB044600BF1CB1072C01D02046F1E7BD
:10B5800000BF042202210020FFF7EEFB044600BFAB
:10B590001CB1072C01D02046E4E700BF0020E1E702
:10B5A0002DE9F04782468946DAF80040B9F1000FEC
:10B5B00006D1E76817B16069B84215D8012713E0D2
:10B5C0004946504601F020FC0646022E02D20120D8
:10B5D000BDE8F087701C08B93046F9E76069B042F1
:10B5E00001D93046F4E74F463D4600BF6D1C606907
:10B5F000A84204D80225BD4201D90020E8E7294627
:10B60000504601F001FC064606B909E0012E01D0C2
:10B61000701C08B93046DBE7BD42E7D10020D7E710
:10B6200000BF00BF4FF0FF322946204605F00EFE56
:10B630008046B8F1000F08D1B9F1000F05D02A46B5
:10B640004946204605F002FE8046B8F1000F0DD1B4
:10B65000E560D4E90410801E814202D22069401EB8
:10B660002061207940F00100207107E0B8F1010F5E
:10B6700002D14FF0FF3000E0012005462846A7E741
:10B680002DE9F35F8A46DAF80090009800F1200572
:10B690000B222021284602F01DF800208046074694
:10B6A0004FF0080B00BF38467F1C19F80040202CD3
:10B6B00000DC55E02F2C01D05C2C0AD100E07F1C6F
:10B6C00019F807002F28FAD019F807005C28F6D0DF
:10B6D00046E02E2C01D0D8450CD3BBF10B0F01D086
:10B6E0002E2C02D00620BDE8FC9F4FF008084FF03A
:10B6F0000B0BD8E7812C01DB9F2C03DDE02C1CDB3E
:10B70000FC2C1ADC38467F1C19F80060402E01DB47
:10B710007E2E03DD802E05DBFC2E03DCABF1010069
:10B72000404501D80620DEE7404608F101082C54C8
:10B73000404608F101082E5411E0214614A0FFF7FD
:10B740007DFD08B10620CEE7612C04DB7A2C02DCFB
:10B75000A4F12000C4B2404608F101082C54A2E72D
:10B7600000BF09EB0700CAF80000B8F1000F01D1D3
:10B770000620B8E72878E52801D105202870202C7C
:10B7800001DC042000E00020E8720020ABE70000AC
:10B79000222A2B2C3A3B3C3D3E3F5B5D7C7F0000E8
:10B7A0002DE9FF4105460C4629492A4A891AC9084C
:10B7B000042242EA01402B46224627A103F078FAF0
:10B7C000002002900390ADF80840ADF80A400090C8
:10B7D00001906A4602A9284690DF0646002E32D024
:10B7E000304604F051F8074619491A4A891AC9081F
:10B7F000012242EA01403B462A46234903F058FA17
:10B80000BDF8000010B9BDF8020068B1BDF8023003
:10B81000BDF800200E490F4FC91BC908012747EA90
:10B8200001401AA103F044FABDF8040058B1BDF874
:10B8300004200749074BC91AC908012343EA0140FC
:10B84000224903F029FA304604B0BDE8F081000037
:10B8500000590300005903005570646174696E67F4
:10B860002064617461206C656E67746820746F2059
:10B870002575206F6E20636F6E6E656374696F6EE1
:10B8800020307825782E000014500300546865207D
:10B890007265717565737465642054582F52582011
:10B8A0007061636B6574206C656E67746820697382
:10B8B00020746F6F206C6F6E672062792025752F62
:10B8C0002575206F63746574732E0000605003004B
:10B8D00020BF70472DE9F04104460E46D4F80080A1
:10B8E0000021204600F000F90546EDB9002700BF11
:10B8F0004046A16901F078FF054605B113E0E06913
:10B900000078E52802D0E069007820B9781C074665
:10B91000B04201D107E000270121204600F040F8A5
:10B920000546002DE4D000BF042D00D10725284690
:10B93000BDE8F0812DE9F04104462768002120464A
:10B9400000F0D2F8054615B12846BDE8F08100BFE9
:10B950003846A16901F048FF054605B11DE0E069E0
:10B9600006780EB9042518E0E069C07A00F03F00BF
:10B97000A071E069C07A00F0080038B90B2204F128
:10B980002001E06901F087FE00B906E000212046B1
:10B9900000F006F80546002DDAD000BF2846D4E7AF
:10B9A0002DE9F047044689462568206900F1200703
:10B9B000A06910B1B7F5001F02D30420BDE8F087DD
:10B9C000C7F30800002868D1A069401CA061606925
:10B9D00038B92889B0EB571F5FD80020A061042038
:10B9E000ECE76889401E00EA5720002855D1204620
:10B9F000616901F009FA0646012E01D80220DDE74F
:10BA0000701C08B90120D9E76869B0423FD8B9F184
:10BA1000000F03D10020A0610420CFE72046616918
:10BA2000FFF7BEFD06460EB90720C7E7012E01D17C
:10BA30000220C3E7701C08B90120BFE7284607F0C1
:10BA400071FD08B10120B9E74FF40072002105F142
:10BA5000300001F03FFE4FF0000831462846FFF766
:10BA600023FCE8620CE00120E870284607F05AFD4C
:10BA700008B10120A2E708F10108E86A401CE86269
:10BA800068894045EFD8E86AA0EB0800E862666183
:10BA900031462846FFF708FCA0612761C7F308017B
:10BAA00005F130000844E061002087E770B50446E6
:10BAB000266801212046FFF70DFF054695B930465F
:10BAC000A16901F091FE054665B920220021E069D7
:10BAD00001F000FE0B2204F12001E06901F0EDFD10
:10BAE0000120F070284670BD2DE9F04104460D4656
:10BAF0002668B5F5001F02D205F01F0010B1022024
:10BB0000BDE8F0812561A7681FB93078032800DB04
:10BB1000776A47B93089B0EB551F01D80220EFE7AB
:10BB2000706AA0611CE070894FEA402811E0394634
:10BB3000204601F069F90746781C08B90120DFE7C3
:10BB4000022F02D37069B84201D80220D8E7A5EBD2
:10BB500008054545EBD239463046FFF7A5FBA06105
:10BB60006761A06908B90220CAE7A06900EB552007
:10BB7000A061C5F3080106F130000844E06100202F
:10BB8000BEE700002DE9F04104463E4800788442BB
:10BB900002DB0320BDE8F08104EB44003A49096868
:10BBA00051F8200008B90320F4E704EB44003649BB
:10BBB000096801EB8000407A00F0010038B904EB1D
:10BBC00044003149096801EB8000407AE2E704EB68
:10BBD00044002D49096801EB8000406838B92B48C2
:10BBE00004EB4401284A126802EB810148600120FD
:10BBF00004EB4401244A126802EB8101887204EBD1
:10BC000044002149096851F82060214F30682246DC
:10BC10003946036830469847054600BF4DBB07E0EC
:10BC200004EB4401184A126802EB8101486880471E
:10BC300004EB44001449096801EB8000807A002875
:10BC4000EED104EB44001049096801EB8000007A52
:10BC500078B904EB44000C49096801EB8000407A94
:10BC600020F0010004EB4401074A126802EB810155
:10BC7000487204EB44000449096801EB8000407AF3
:10BC800088E70000502F00204C2F0020D1B8020080
:10BC9000E1AA0200F8B504460E4615462A48007887
:10BCA000844201DB0420F8BD26B1012E1BD0022EF8
:10BCB00045D12EE00120009000BF04EB4401234A4F
:10BCC000126852F821006A46002102F0A2F80746E5
:10BCD00017B1112F00D003E09DF800000028ECD12F
:10BCE00000BF0020DFE704EB44001849096851F861
:10BCF000200008B90320D6E72F4604EB4401134A7D
:10BD0000126852F8210002F07DF8006838600020C7
:10BD1000C9E704EB44000D49096851F8200008B94F
:10BD20000320C0E72F4604EB4401084A126852F88A
:10BD3000210002F067F8808838800020B3E700BF58
:10BD400000BF0120AFE70000502F00204C2F002043
:10BD50002DE9FE4F0446884691461E462F4800783E
:10BD6000844200DA16B90420BDE8FE8F04EB4400DB
:10BD70002B49096851F8200048B104EB44002849D8
:10BD8000096801EB8000407A00F0010008B103204F
:10BD9000EAE7CDF800900196CDF80880012004EB89
:10BDA00044011F4A126802EB8101887204EB4400CF
:10BDB0001B49096851F820506F4628684169284698
:10BDC000884700683968884201D8072004E028685D
:10BDD00039468268284690478246BAF1000F1BD147
:10BDE00007E004EB44010E4A126802EB8101486847
:10BDF000804704EB44000A49096801EB8000807A1F
:10BE00000028EED104EB44000549096801EB8000ED
:10BE1000007A08B90020A7E70120A5E7502F0020ED
:10BE20004C2F0020014607480078814201DB0120A9
:10BE3000704701EB4100044A126802EB8000407A2F
:10BE4000F6E70000502F00204C2F002070B504466C
:10BE500036480078844201DB032070BD04EB4400C7
:10BE60003349096851F8200008B90320F5E704EBCD
:10BE700044002F49096801EB8000407A00F001007E
:10BE800038B104EB44002A49096801EB8000407A8C
:10BE9000E3E704EB4401264A126852F8210000222D
:10BEA000114601F0B6FF00BF04EB440020490968C9
:10BEB00051F820603068416830468847054600BF29
:10BEC000112DF1D08DB907E004EB4401184A126836
:10BED00002EB81014868804704EB4400144909687B
:10BEE00001EB8000807A0028EED104EB4400104979
:10BEF000096801EB8000007A78B904EB44000C4932
:10BF0000096801EB8000407A40F0010004EB440135
:10BF1000074A126802EB8101487204EB44000449AD
:10BF2000096801EB8000407A97E70000502F00205D
:10BF30004C2F00202DE9FE4F0446884691461E46B0
:10BF400035480078844200DA16B90420BDE8FE8F37
:10BF500004EB44003149096851F8200048B104EB72
:10BF600044002E49096801EB8000407A00F001008E
:10BF700008B10320EAE704EB44002849096801EB13
:10BF80008000407A00F0040008B10220DEE7CDF81E
:10BF900000900196CDF80880012104EB44001F4A6F
:10BFA000126802EB8000817204EB44001B490968AF
:10BFB00051F820506F462868416928468847006834
:10BFC0003968884201D8072004E028683946C268E9
:10BFD000284690478246BAF1000F1BD107E004EBD8
:10BFE00044010E4A126802EB81014868804704EB65
:10BFF00044000A49096801EB8000807A0028EED1EC
:10C0000004EB44000549096801EB8000007A08B997
:10C0100000209BE7012099E7502F00204C2F0020A3
:10C02000024A1060024B1970704700004C2F00202C
:10C03000502F002010B50021034801F08BFD04466D
:10C0400084F3100010BD00003479002070B505465F
:10C050000C464FF4803000FA04F1284600F0AAF9AB
:10C0600070BD70B505460C464FF4A07000EB84001F
:10C0700086B23146284600F0B7F970BD2DE9F04789
:10C0800004460D4616461F464FF4803000FA05F868
:10C090004FF4A07000EB85001FFA80F926F07F4670
:10C0A0004146206803F0CBF84146206803F0B8F819
:10C0B0004946206803F0AAF832462946206803F072
:10C0C00095F84146206803F0B1F81FB14146206859
:10C0D00003F0BBF8BDE8F08710B50446206803F014
:10C0E0008AF810BD2DE9F04704460D4617466079E1
:10C0F000324941F820706079314901EBC000007984
:10C1000068B108262F49304A891AC908022242EA32
:10C1100001402EA102F0B6FD3046BDE8F087298827
:10C120002068C0F8081500BF94F90420AB781046C9
:10C130001946002808DB4FEA417C4FEA1C68DFF80B
:10C14000B0C00CF800800BE04FEA417C4FEA1C695C
:10C15000DFF8A0C000F00F08A8F104080CF8089060
:10C1600000BF00BF94F90410084600280DDB00BF93
:10C1700000BF00F01F0301229A4043099B0003F116
:10C18000E023C3F8002100BF00BF00BF00BF0120B3
:10C1900061790B4A02EBC10108716079114641F8DF
:10C1A000304000260749084A891AC908032242EA92
:10C1B000014011A102F066FD3046AEE7B42E00202A
:10C1C000B82E002080590300005903005254432028
:10C1D000696E7374616E636520616C726561647908
:10C1E00020696E697469616C697A65642E0000006B
:10C1F00000E400E018ED00E05254433A20696E6913
:10C200007469616C697A65642E00000010B501469E
:10C2100091F90400002807DB00F01F0301229A4077
:10C22000024B440943F8242000BF10BD00E200E0A7
:10C2300070B505460C4622460221284600F0C6F895
:10C2400070BD10B504464FF48271204600F0CCF862
:10C2500010BD10B504460021206803F001F810BDA0
:10C2600010B504460421206802F0FAFF10BD2DE944
:10C27000F84F04468846154699464FF4803000FA38
:10C2800008FA4FF4A07000EB88001FFA80FB25F03D
:10C290007F455146204600F08DF8206802F0ABFF44
:10C2A00006464146206802F09BFF00903246414618
:10C2B000206802F09BFF5946206802F0A7FF314634
:10C2C000009807F058F9012806D1102003F05CFB14
:10C2D0005946206802F09AFF206802F08CFF06465B
:10C2E0003146284607F047F907465146206802F0D4
:10C2F0009DFF012F0FD16A1C4146206802F076FF96
:10C30000102003F041FB206802F075FFB04225D0F9
:10C310000D20BDE8F88F2A464146206802F066FFEE
:10C32000206802F068FF0646681E314607F023F9D0
:10C3300007466FF07F40A0EB0900B84201D20D2004
:10C34000E7E75FB96A1C4146206802F04FFF2068AA
:10C3500002F051FFB04201D00D20DAE70122514630
:10C36000204600F033F80020D3E7000010B5104855
:10C370000068407E60B106210120FEF775F9044691
:10C3800024B10B480068416903208847002010BD94
:10C39000012007490968087601210846FEF764F97B
:10C3A00004461CB100200249096808762046EEE7E1
:10C3B0005C2F002070B504460D462946206802F027
:10C3C0002FFF2946206802F03AFF70BD70B5044681
:10C3D0000E4615463146206802F028FF1DB1314651
:10C3E000206802F032FF70BD70B505460C46286823
:10C3F000015929B12146286802F008FF012070BDCB
:10C400000020FCE738B50546284600F047FA044608
:10C410003CB96946284607F028FE04460CB90020BE
:10C420002860204638BD2DE9FC47074688469146DE
:10C4300000243E4613E06B46012201A9484600F065
:10C4400040F90098012800D00DE09DF8045000BF8D
:10C4500006F8015B641C0A2D00D104E000BFA8F1BE
:10C460000100A042E7DC00BF0020307014B1384664
:10C47000BDE8FC870020FBE7F7B582B016460398BD
:10C48000019001A800F098FD0546002D02DA0B206E
:10C4900005B0F0BD0E4850F825400CB100202070CA
:10C4A000029810B10020029908700949029841F8D9
:10C4B0002500029808B1012E01D00020E8E70022F3
:10C4C00002A903A800F03AFA07463846E0E7000060
:10C4D000542F00202DE9F74F8EB0044616461CB9A4
:10C4E000092011B0BDE8F08F06F03F06324602A9E0
:10C4F0000FA800F023FA0546002D70D10298039092
:10C5000003A80F9900F0EDFB05462DB99DF8370003
:10C5100000F0800000B1062506F01C00002856D06F
:10C5200045B1042D03D103A8FFF7C0FA054646F034
:10C5300008060AE09DF8120000F0110008B1072576
:10C5400003E006F0040000B10825002D51D106F0EB
:10C55000080000284DD000F0C7FC01900A9901F1B5
:10C560000E00019906F09EFE0A9901F1160001994C
:10C5700006F098FE20200A99C8720A99029800F0E5
:10C5800045FF814600220A99029806F079FE0A9931
:10C5900001F11C00002106F085FE01200299C870FF
:10C5A000B9F1000F25D00298C06A019000224946D7
:10C5B00003A804F0C5FF0546DDB9DDE9011001F06F
:10C5C00013F90546A9F101000299C86011E085B987
:10C5D0009DF8120000F0100010B1042509E05DE0A4
:10C5E00006F0020028B19DF8120000F0010000B131
:10C5F00007254DB906F0080008B146F0400602983C
:10C60000C06A20620A986062002D55D10A9902988A
:10C6100000F0FCFEA0600A9901F11C0000F009FF87
:10C62000E060029820600298C088A08026740020F4
:10C630006074E06160614FF40072002104F1280031
:10C6400001F048F806F0200040B3E06830B3E0683D
:10C650006061029840894FEA402AA768D4F80C80AC
:10C660000CE03946204600F0CFFB0746012F00D8EA
:10C670000225781C00B90125A8EB0A080DB9D045A0
:10C68000EFD8A76155B9C8F3080038B13946029808
:10C69000FEF70AFEB0F1000B01D102250CE00BEB16
:10C6A0005820E061E26902994878012304F12801E9
:10C6B000FFF74EFB00B101250DB100202060284698
:10C6C0000FE72DE9FF4F85B0044615469A46DDF881
:10C6D00018B00020CAF8000003A9204607F0C5FCE6
:10C6E0000490049810B9607C049018B1049809B0C3
:10C6F000BDE8F08F207C00F0010008B90720F6E7C4
:10C700006169E068401A01900198854200D9019D55
:10C71000A0E0A08AC0F3080000287ED103984089D9
:10C72000401E616900EA5129B9F1000F17D1606913
:10C7300010B9A068029004E02046A16900F064FBF3
:10C7400002900298022802D202206074CFE7029879
:10C75000401C10B901206074C9E70298A061A1696A
:10C760000398FEF7A1FD064616B902206074BEE7E5
:10C770004E444FEA5528B8F1000F29D009EB0800C4
:10C7800003994989884203D903984089A0EB090895
:10C7900003994878434632465946FFF7D9FA10B113
:10C7A00001206074A3E7207C00F0800068B1E0699C
:10C7B000801B404509D2E169891B0BEB41204FF4F6
:10C7C000007204F1280100F078FF4FEA482737E0B3
:10C7D000E069B04220D0207C00F0800078B1E269AE
:10C7E00003994878012304F12801FFF7A3FB10B156
:10C7F000012060747BE7207C00F07F0020740399A7
:10C8000048780123324604F12801FFF7A1FA18B154
:10C81000012060746BE700E0E661A08AC0F30800C5
:10C82000C0F50077AF4200D92F46A08AC0F30802B6
:10C8300004F1280011183A46584600F03EFF00BFA8
:10C84000BB44606938446061DAF800003844CAF8D3
:10C850000000ED1B002D7FF45CAF002047E733B5EF
:10C860008BB00D46002269460BA800F067F804461D
:10C870008CB968460B9900F034FA04465CB99DF80F
:10C880002B0000F0800008B1062404E01DB1294609
:10C89000684600F04BFB20460DB030BDF8B50446AD
:10C8A0006946204607F0E1FB0646002E44D1207C75
:10C8B00000F0400000283FD0207C00F0800070B1E4
:10C8C000E26900994878012304F12801FFF732FB5F
:10C8D00008B10120F8BD207C00F07F00207400F03A
:10C8E00003FB0746216A009800F07EFF06461EBB48
:10C8F000656AE87A40F02000E8722946A26820685C
:10C9000006F0BEFC05F11C00E16806F0CBFC3946E0
:10C9100005F1160006F0C6FC002105F1120006F034
:10C92000CDFC01200099C870009806F0B3FD0646C2
:10C93000207C00F0BF0020743046CBE72DE9F74F94
:10C940008AB000210B9801600A9800F035FB08902E
:10C950000898002803DA0B200DB0BDE8F08FB1492C
:10C96000089851F820400CB90C20F5E70B980460AA
:10C970000C9800F0FE000C90207878B16078FFF7FA
:10C9800051FA814609F0010040B90C9820B109F034
:10C99000040008B10A20DFE70020DDE70020207056
:10C9A000089860706078FFF7EDF8814609F00100A3
:10C9B00008B10320D0E70C9820B109F0040008B1B9
:10C9C0000A20C9E7002739462046FEF7F9FB05464D
:10C9D000022D01D02EDA2DE0002614E04FF4DF7096
:10C9E00000EB061104F13000084409900998007921
:10C9F00020B10998083000F01CFD00E0002002A9D9
:10CA000041F82600761C042EE8D3002606B1761ED7
:10CA100000BF02A850F8267027B139462046FEF71D
:10CA2000CFFB00E003200546022D03DB701C064609
:10CA30000428EED3042D01D101208DE7022D01DB66
:10CA40000D2089E704F13B0000F0FFFCB0F5007F0A
:10CA500001D00D2080E704F1460000F0F6FC80468E
:10CA6000B8F1000F04D104F1540000F0E2FC80465C
:10CA7000C4F818804020005DA070A078012804D080
:10CA8000A078022801D00D2066E7A07808FB00F806
:10CA90003D20005D6081608918B16089411E0840B9
:10CAA00008B10D2058E704F1410000F0CEFC2081D0
:10CAB000207A00F00F0008B10D204DE704F143008B
:10CAC00000F0C3FC8246BAF1000F04D104F150001B
:10CAD00000F0AFFC824604F13E0000F0B6FC01908D
:10CAE000019808B90D2037E701984044218900EBEF
:10CAF000111007900798824501D20D202CE7079866
:10CB0000AAEB00006189B0FBF1FBBBF1000F01D182
:10CB10000D2021E703254FF6F570834500D8022547
:10CB200040F6F570834500D801250BF102006061E5
:10CB3000E76101983844206207983844A062032DC9
:10CB400013D104F15A0000F080FC08B10D2003E776
:10CB5000208908B10D20FFE604F15C0000F069FCBB
:10CB6000606260698000069014E0208908B90D2099
:10CB7000F2E6206A40446062022D02D16069400002
:10CB800007E0207D00F00100616901EB410100EB4D
:10CB900051000690A169069800F2FF10B1EB502FEA
:10CBA00001D20D20D8E64FF0FF302061E0608020F8
:10CBB0002071032D2CD104F1600000F046FC012807
:10CBC00026D1791C204600F00FFE08BB0020207102
:10CBD00004F22E2000F039FC4AF65521884217D184
:10CBE00004F1300000F025FC0F49884210D104F513
:10CBF000057000F01EFC0D49884209D104F506704D
:10CC000000F017FC206104F5077000F012FCE060F2
:10CC1000257007480088401C80B205490880E080E4
:10CC2000002099E6542F00205252614172724161F6
:10CC3000582F002010B50446E07FFF2808D0A07FC1
:10CC400018B1E07F01F099FC02E0E07F01F044FDC3
:10CC500000206077207204F10800D4E90021904799
:10CC600010BD70B505460E46144624B1314628461F
:10CC700000F032FF03E03146284600F00FFF70BDA0
:10CC800030B504461088C01C984201D90C2030BD34
:10CC90000220158848551088401C108001201588F6
:10CCA00048551088401C108015884C551088401C31
:10CCB00010800020EBE770B504460D4640F21442A8
:10CCC000115B0122D4F81004FDF77CF9064606B189
:10CCD000357004F13C0204F5826104F1540072DF06
:10CCE00070BD2DE9F34104462646D6F8008002E0E7
:10CCF0000198401C0190019800782F28F8D00198E5
:10CD000000785C28F4D00020B060019800782028DA
:10CD100008D280212B20015500212046FEF7E4FE99
:10CD200005462CE000BF01A92046FEF7A9FC0546F8
:10CD300005B123E02046FEF7FDFD05462B20075DEB
:10CD40003DB1042D04D100BF07F0040000B9052552
:10CD500014E007F0040000B110E0B07900F010001A
:10CD600008B905250AE0208AC0F3080208F130005E
:10CD70001118404600F04AFBB060D4E700BF2846D7
:10CD8000BDE8FC8170B505460C4660880C490988F1
:10CD9000884214D1208840F6772188420FD1A0889C
:10CDA000C01E084908802B886A880749074E891BDE
:10CDB000C908042646EA014005A101F079FF70BDCB
:10CDC0003C2F00203E2F00209859030000590300FB
:10CDD000415454204D54552065786368616E6765F1
:10CDE00020636F6D706C657465642E2063656E746E
:10CDF00072616C202564207065726970686572616B
:10CE00006C202564000000002DE9F04781460C46A7
:10CE1000D9F80050022C02D36869A04202D84FF022
:10CE200001085EE04FF0FF382878012804D002287E
:10CE30002CD0032851D13CE0264606EB5606286A42
:10CE400000EB5621284600F0CFFC00B148E0304608
:10CE5000761CC0F3080105F13000475C286A00EB3E
:10CE60005621284600F0C0FC00B139E0C6F30801A5
:10CE700005F13000405C47EA002704F0010008B1EA
:10CE8000380901E0C7F30B00804629E0286A00EB6F
:10CE90001421284600F0A8FC00B121E040F2FF1167
:10CEA00001EA440205F13001501800F0CEFA804644
:10CEB00016E0286A00EBD411284600F095FC00B17A
:10CEC0000EE040F2FF1101EA840205F13001501832
:10CED00000F0AFFA20F0704802E04FF0010800BF08
:10CEE00000BF4046BDE8F0871CB51F201D21172359
:10CEF0001A46CDE9001001214FF4FD6000F001F861
:10CF00001CBDF0B50446DDE905560020A4F2BC774F
:10CF100040EA47604F1C40EA475040EA024040EA7E
:10CF2000C32040EA451040EA5600F0BD2DE9F04725
:10CF300005460C4600206072A86908B9BDE8F08774
:10CF4000002637461CE03046761CEA6912F800904D
:10CF5000B9F1200F00D113E0B9F1050F01D14FF065
:10CF6000E509092E05D12E2238467F1C04F109015E
:10CF70000A5438467F1C04F1090101F8009000BFF3
:10CF80000B2EE0D3002104F10900C155E869C07AF5
:10CF90002072E96901F11C0000F04BFA2060E96998
:10CFA00001F1160000F045FA8046A4F806804FEA29
:10CFB0001840A08000BFC1E770B502464FF0FF30B7
:10CFC0001568DDB1116800E0491C0D78212D02D3F0
:10CFD0000D783A2DF8D10D783A2D0ED1146814F849
:10CFE000015BA5F130030A2B06D28C4204D11BB998
:10CFF00018464D1C2946156070BD002000BFFBE798
:10D0000070B50B48FFF768F80A4B0CCB841843F156
:10D010000005094903C9201A75EB010004D24FF03D
:10D020008073E41845F100052046294670BD0000D4
:10D03000902E0020A02E0020A82E002038B51F2002
:10D040000090684601F0A6FA044600BFD4F8100527
:10D050000099C84000F0010038BD000002460021E0
:10D060000CE001EB8100074B33F82000904204D123
:10D0700001EB810003EB80007047491C0029F0D0D0
:10D080000020F9E7B85800202DE9FC5F83460E46E2
:10D0900091461F46DDE90C45002E01DA704200E0A2
:10D0A000304682464FF0010803E09AFBF9FA08F196
:10D0B0000108CA45F9DA474500D9B84634B1002E0F
:10D0C00003DB05F00400042800D1641E05F0020013
:10D0D00000B167B105F0010048B944B104E0641E35
:10D0E00020215846FDF7E2FE0CB1A045F7D3002EF3
:10D0F00005DA76422D215846FDF7D8FE07E005F007
:10D100000400042803D12B215846FDF7CFFE05F07B
:10D11000020002280DD105F0010050B94FB944B109
:10D1200004E0641E30215846FDF7C0FE0CB1A04556
:10D13000F7D33B464A4631465846CDE9004506F00E
:10D140005DFEBDE8FC9F30B5024600201378C3F3B6
:10D150008003D3B1137803F00303012B02D0022B19
:10D1600010D107E01388C3F383139B1C0C6823447E
:10D170000B6008E00B680225146805EB9454234407
:10D180000B6000E000BF00BF012030BD70B5054658
:10D190000C464FF48C71284602F042FB38B14FF434
:10D1A0008C71284602F043FB2046FFF743FD70BD1B
:10D1B00070B505460C464FF48871284601F077FF9C
:10D1C00068B14FF48871284601F078FF607900F06B
:10D1D000040020B1206810B10120216888474FF475
:10D1E0008A71284601F063FF68B14FF48A712846BE
:10D1F00001F064FF607900F0080020B1206810B1F0
:10D200000220216888474FF48E71284601F04FFFB5
:10D2100068B14FF48E71284601F050FF607900F03C
:10D22000100020B9206810B10020216888474FF411
:10D230008271284601F03BFF58B14FF482712846B5
:10D2400001F03CFF01202071206810B1032021680B
:10D25000884770BD2DE9F04781460C4616464FF4CD
:10D2600080374FF4A078002520E03946484601F089
:10D27000EFFFA8B14146484601F0DBFF80B13946D7
:10D28000484601F0CAFF3946484601F0D5FF4146FD
:10D29000484601F0B4FFE8B21B4A52F82410884710
:10D2A0007F0008F104001FFA80F86D1CB542DCD342
:10D2B0004FF480780121484601F0CAFF68B1414629
:10D2C000484601F0B6FF40B14146484601F097FF9D
:10D2D0000D4850F82410042088474FF4827802212A
:10D2E000484601F0B5FF68B14146484601F0A1FF4C
:10D2F00040B14146484601F082FF034850F82410EF
:10D3000005208847BDE8F087782E00202DE9F047FA
:10D3100004460E469046002722E0384602F0C2FA44
:10D320000546384602F0C5FA81462046294642584D
:10D330000AB1012200E0002282B14846D4F8041369
:10D34000014009B1012100E0002139B12946204600
:10D3500002F0B4FA2846D6E900219047781CC7B2FB
:10D360004745DADBBDE8F0872DE9F0410446A088A7
:10D3700000EB020CB4F80480904501DD104600E09B
:10D38000A088A8EB0005E088C618B4F80680984588
:10D3900001DD184600E0E088A8EB00074888B4F8F3
:10D3A0000080404504DB4888B4F80280404502DD37
:10D3B0000020BDE8F0818888A84202D388886045B3
:10D3C00001D90020F5E7C888B84202D3C888B04226
:10D3D00001D90020EDE70120EBE70146086808B11C
:10D3E00002680A60704710B50446224602210020F8
:10D3F00001F09CF8002105E054F8210008B101205B
:10D4000010BD491C0229F7D30020F9E770B5054685
:10D410000C4604F11A0000F018F806462878032894
:10D4200005D104F1140000F010F846EA0046304639
:10D4300070BD0146C8788A7842EA00204A7842EAFC
:10D4400000200A7842EA00207047014648780A78AE
:10D4500042EA00207047000010B502F05BFA20B9E4
:10D4600002F07CFA00200149887010BD6459002048
:10D47000F7210180172141800021017141711B2199
:10D480008171C171704770472DE9FF4100272E4817
:10D4900000F038FB2C48001F00F034FB2B4880685C
:10D4A00003902B4805680398284028490C3101EB6C
:10D4B000800800BF03A94046FFF745FE30B103983E
:10D4C000284022490C3101EB800800E000E0F1E740
:10D4D00000BF00240AE00398411C284003911B4927
:10D4E0000C3151F820004DF82400641C022CF2D3BA
:10D4F000009800F0030001280DD0022814D1BDF8D7
:10D5000006700421009801EB9050401E039901EB36
:10D510009000039009E0BDF806700098C0F38310F6
:10D5200003990844039000E000BF00BF0648001FB5
:10D5300000F0E1FA064616B10449039888603846BF
:10D5400004B0BDE8F08100003079002018690020A7
:10D55000E82E002000BF1A4A64213820FCF7F6F8B4
:10D56000044600BF254625B100BF2846FCF71CF83D
:10D5700000BF00BF00BF07F01DF91249124A891A07
:10D58000C908032242EA014010A213A101F084FB62
:10D5900016490A680B490C4BC91AC908032343EA08
:10D5A000014013A101F078FB15A01B4908601B483E
:10D5B0004860084606F094FDFAF73EFA05F004FBD1
:10D5C000B4350020985903000059030030393A342B
:10D5D000393A303200000000636F6D70696C65206D
:10D5E00074696D65203A25730000000080100010FA
:10D5F000435553544F4D4552203A256400000000D6
:10D60000414453313239335F5445535445525F33AB
:10D6100043485F5632000000FC2C0020B103030099
:10D620002DE9F04105460E4614469846A888871C09
:10D630002088801C3844404502D90C20BDE8F08188
:10D64000FE2F01D90C20F9E7781C2188705420881E
:10D65000401C2080FF20218870542088401C20809E
:10D6600022889119288806F0C2FB2188084420806E
:10D67000A88800280DDDA86808B90720DEE7AA8879
:10D6800023889819A968F9F7BCFE2088A98808445E
:10D6900020800020D2E7F0B503461D460C4600204E
:10D6A00000BF15F8017B14F801CBA7EB0C00561E48
:10D6B000321E01D00028F4D0F0BD30B503460C4630
:10D6C0003AB100BF14F8015B03F8015B551E2A1E36
:10D6D000F8D130BD10B5034600BF03F8011B541E3E
:10D6E000221EFAD110BD2DE9FF4F87B004469146A6
:10D6F0001E46A2462546BAF806009AF80510484389
:10D70000001F0690BAF806B0301DB0FBFBF0059084
:10D71000301DB0FBFBF10BFB11000490D9F80000A9
:10D7200081190698814202D90698801B01E0D9F838
:10D7300000000746C9F8007003E02D680598401EF8
:10D74000059005980028F8D103900498ABEB0008E9
:10D75000B84501D9384600E04046804623E00399A9
:10D76000089808440290281D0499084401901498D0
:10D7700028B14246DDE90110F9F743FE04E04246D4
:10D78000DDE90101F9F73DFE002004902D68A7EBCB
:10D790000807039840440390BB4501D9384600E090
:10D7A0005846804600BF002FD9D10BB0BDE8F08F9E
:10D7B00070B503460C469CB101F036FB05460022CD
:10D7C0000AE0084800EB820108881E68B04202D1D6
:10D7D0001A60002070BD521CAA42F2D30520F9E75E
:10D7E0000020F7E70000000070B504460D46002653
:10D7F000E06AA84210D0204605F094FE06465EB9C5
:10D80000607801232A4604F13001FEF7A1FA10B135
:10D810004FF0FF350126E562304670BD2DE9F84F27
:10D8200005460F46144698462878012804D16878A2
:10D8300010B90720BDE8F88F2088801C404508D823
:10D840002878012807D12088801C69780844404541
:10D8500001D90C20EEE72088A8EB0000801E86B2DC
:10D8600000962188891CC81969467DDF814600BF62
:10D87000484600B1DEE700BF2878022804D0687867
:10D88000BDF80010884206DBBDF80000B04202DCA3
:10D890004FF0090A0BE04FF0080A2878012805D15B
:10D8A0006878B04202DC6878009000E00096BDF82D
:10D8B0000000FE2801D90C20BCE7BDF80000401C88
:10D8C000218878542088401C2080208807F800A0F8
:10D8D0002088401C20802088BDF80010084420804B
:10D8E0000020A7E7014604480088814201DA481C6D
:10D8F00000E00020C0B270478C2E0020FEB5044628
:10D900000D46002001900290CDF808D00220ADF81D
:10D9100004000020ADF8060001AA29462046ADDF2C
:10D9200006462EB90298FDF7D2F808B10120FEBDD7
:10D930000020FCE70B4802684FF08050D0F834110B
:10D940000D2A0DD121B1012904D0022906D103E00D
:10D95000012070470120FCE70120FAE70120F8E7E9
:10D960000020F6E7300100100B4802684FF08050AD
:10D97000D0F834110D2A0DD121B1012904D002298A
:10D9800006D103E0002070470020FCE70120FAE701
:10D990000120F8E70020F6E7300100100B4802688C
:10D9A0004FF08050D0F834110D2A0DD121B101294A
:10D9B00004D0022906D103E0012070470120FCE7D2
:10D9C0000120FAE70120F8E70020F6E73001001017
:10D9D0000B4802684FF08050D0F834110D2A0DD159
:10D9E00021B1012904D0022906D103E001207047AA
:10D9F0000120FCE70120FAE70120F8E70020F6E724
:10DA00003001001010B5044609B90E2010BD92FB7C
:10DA1000F3F003FB102008B10920F7E72160002094
:10DA20006060A060A281E38100BFEFE770B50446AB
:10DA30000D4629462046F9F7EFFB18B12A882168E0
:10DA4000881870BD0020FCE770B505460C4620889C
:10DA50006188884204D12846F9F720FC012070BD76
:10DA60000020FCE770B504460D4629462046F9F72C
:10DA7000F8FB18B16A882168881870BD0020FCE79F
:10DA800070B505460C4620886188884204D1284636
:10DA9000F9F7DEFB012070BD0020FCE770B50546FC
:10DAA0000C4604F01F0301229A40D143620905EBA2
:10DAB000820000F039F8064670BD10B502464809EC
:10DAC00052F8200001F01F040123A340184008B1C0
:10DAD000012010BD0020FCE770B505460C4604F09F
:10DAE0001F03012202FA03F1620905EB820000F034
:10DAF0003CF8064670BD10B504460021204600F0F3
:10DB00001EF810BD10B504460121204600F02DF886
:10DB100010BDF8B504460D466A4629462046F9F779
:10DB200012FC06460098F8BDF8B504460D466A4654
:10DB300029462046F9F7EDFB06460098F8BDF8B5F2
:10DB400004460D466A4629462046F9F7E2FB06469A
:10DB50003046F8BDF8B504460D466A4629462046CB
:10DB6000F9F7BEFB06463046F8BDF8B504460D464B
:10DB70006A4629462046F9F7BFFB06460098F8BDDD
:10DB8000F8B504460D466A4629462046F9F7E8FBF3
:10DB900006460098F8BDF8B504460026002000901F
:10DBA0006846FCF76BF8206800686168884215D900
:10DBB00020680068401E226810600178204600F04E
:10DBC00033F80646207A21680978401AC5B22068E1
:10DBD0000079A84201DA2068057100BF9DF80000B5
:10DBE000FCF752F83046F8BD0246D068081A138A8E
:10DBF000B0FBF3F0C0B27047F8B504460D462E46B0
:10DC0000002000906846FCF739F831462046FFF7BF
:10DC1000EBFF21680A68511C2368196010709DF899
:10DC20000000FCF731F8F8BD0246138AD06801FB0A
:10DC30000300704710B5014600BF09B90E2010BDA2
:10DC400000BF087A0B79C01AC2B2D1E9003018605F
:10DC500005E008680368581C0C6820601A70101EE4
:10DC6000A2F10103DAB2F4D10B68187100BFE6E744
:10DC700030B502460B46D40802F00702012090405E
:10DC80001D5D284030BD024600BF0AB90E20704716
:10DC900000BF172901DBF72901DD0720F7E7118015
:10DCA0000020F4E770B504460E4600BF0CB90E2004
:10DCB00070BD00BF2661F720208060801B2020718E
:10DCC000002505E0A11D01EBC500FFF7D1FB6D1C90
:10DCD000002DF7D00020EBE72DE9F04706468846F7
:10DCE0004546B488012C01DBBDE8F0873088242844
:10DCF00020D006DC102809D011280CD0232823D1ED
:10DD00001DE03A280CD055281ED10EE03146284699
:10DD100002F0A6FC19E03146284602F0AEFE14E0FF
:10DD20003146284602F072FF0FE03146284602F0E5
:10DD3000AFFE0AE03146284602F06EFD05E03146AE
:10DD4000284602F011FE00E000BF00BFA81D00EB56
:10DD5000C400007970B3A81D30F834102046A5DF48
:10DD60000746C7B90021A81D00EBC40001710121BD
:10DD7000A81D00EBC4004171A91D31F834201149E0
:10DD8000114BC91AC908042343EA014023460F492D
:10DD900000F08EFF12E0112F10D0384601F074FD14
:10DDA00081460849084A891AC908012242EA014005
:10DDB0004A4600E003E006A100F06EFF00BF00BF8E
:10DDC00092E700000059030000590300CC4F030004
:10DDD00073645F626C655F67617474635F657863C9
:10DDE00068616E67655F6D74755F72657175657387
:10DDF0007428292072657475726E65642025732EEF
:10DE00000000000010B5044620684169204688479C
:10DE100010BD70B504460D461646206832462946A8
:10DE200003692046984770BD01464FF08040405836
:10DE300008B1012070470020FCE708B500224FF030
:10DE400080410A500958009100BF08BD014908608F
:10DE50007047000008030040012291070A507047F4
:10DE60002DE9F04104460CB9BDE8F08100BF4FF444
:10DE70007A7505B904E0054FAE013046B84700BFDA
:10DE8000601E041EF3D100BFEEE7000071490300DD
:10DE900070B540F6F8700068401C18B94FF01020BB
:10DEA000406902E040F6F87000680546681C0028EA
:10DEB0001CD01449144A891AC908032242EA0140B5
:10DEC0002A4612A100F0E8FE284613DF04465CB1A2
:10DED0000C490D4A891AC908012242EA014016A1DB
:10DEE00000F0D0FE204670BD0020FCE70549064A40
:10DEF000891AC908012242EA01401CA100F0C2FEB1
:10DF00000420F0E798590300005903005365747426
:10DF1000696E6720766563746F72207461626C65E8
:10DF200020746F20626F6F746C6F616465723A2049
:10DF300030782530387800004661696C656420725D
:10DF4000756E6E696E672073645F736F6674646567
:10DF5000766963655F766563746F725F7461626C26
:10DF6000655F626173655F73657400004E6F206268
:10DF70006F6F746C6F616465722077617320666F78
:10DF8000756E640010B50E490E4A891AC90803223D
:10DF900042EA01400C4A0DA100F07EFE0A4813DF60
:10DFA00004465CB10649074A891AC908012242EAB7
:10DFB000014011A100F066FE204610BD0020FCE7E4
:10DFC00098590300005903000070020053657474EF
:10DFD000696E6720766563746F72207461626C6528
:10DFE00020746F206D61696E206170703A20307806
:10DFF00025303878000000004661696C6564207245
:10E00000756E6E696E672073645F736F66746465A6
:10E01000766963655F766563746F725F7461626C65
:10E02000655F626173655F736574000010B50024FD
:10E030000F48007808B1852411E000200C49886061
:10E0400048600861C8600B4801F078FC044601F0A4
:10E0500045FB08B901F068FC01200549087001F092
:10E0600059FC10B1012002498870204610BD000003
:10E070006459002081B2020008B500200090684673
:10E08000FBF7FCFD0748C068401E0649C86008460B
:10E09000C06808B9FFF7E0F99DF80000FBF7F4FD50
:10E0A00008BD0000645900202DE9FF4705460C46D5
:10E0B000164698462F781A4840F82760194840F8C5
:10E0C00027804FF00009184B0FCB8DE80F00207808
:10E0D0008DF8000060788DF80100A0788DF80200BE
:10E0E000E0788DF8030020798DF8050060798DF8CF
:10E0F0000600A0680290207B8DF80C00607B8DF8F4
:10E100000D000EB1094800E0002002463B4669467A
:10E11000281D01F0B7FF8146484604B0BDE8F087EE
:10E12000585A0020685A0020084A03003131030081
:10E130002DE9FF4704460D4616461F46DDF83080A0
:10E140004FF00009009501960297CDF80C8000224F
:10E150006946201D02F0E4F88146484604B0BDE857
:10E16000F0872DE9FF4704460D4616461F46DDF8A9
:10E1700030804FF00009009501960297CDF80C8091
:10E1800000226946201D02F0CBF88146484604B0C3
:10E19000BDE8F0870FB438B50446059810B938BC0F
:10E1A0005DF814FB0020009006A800906A46204607
:10E1B000059900F012F80020009000BFEFE770B55D
:10E1C0000446A06800B970BDD4E90403A2682168C0
:10E1D00098470020A06000BFF5E72DE9FC5F82466C
:10E1E0000D4614460DB9BDE8FC9F00BF2E786D1C8E
:10E1F00006B9E1E0252E70D100274FF0010900BFDC
:10E200002E782B2E0CD02D2E02D0302E0CD103E0E8
:10E2100047F001076D1C0AE047F002076D1C06E09D
:10E2200047F004076D1C02E04FF0000900BF00BF7B
:10E23000B9F1000FE4D14FF0000800BF2A2E06D13B
:10E240002168081D2060086880446D1C0DE02E7850
:10E25000302E01DB392E00DD07E06D1CA6F1300009
:10E2600008EB880100EB4108E8E700BF4FF0000B26
:10E270002E782E2E10D16D1C00BF2E78302E01DB93
:10E28000392E00DD07E06D1CA6F130000BEB8B0191
:10E2900000EB410BF1E700BF2E7800BF6C2E01D0E0
:10E2A000682E02D16D1C2E7800E000E0F6E700BF7A
:10E2B000692E21D008DC252E6DD0582E39D0632E42
:10E2C0000CD0642E6CD116E0702E4CD0732E3ED044
:10E2D000752E1FD0782E63D12AE065E02168081DD5
:10E2E0002060D1F8009009F0FF000190504601999C
:10E2F000FCF7DCFD55E000BF2168081D2060D1F867
:10E3000000905B460A2249465046CDE90087FEF759
:10E31000BBFE46E02168081D2060D1F800905B46F6
:10E320000A2249465046CDE9008705F067FD38E0EE
:10E3300000BF2168081D2060D1F800905B461022C4
:10E3400049465046CDE9008705F058FD29E021688F
:10E35000081D2060086801903B46424650460199DE
:10E3600005F05EF81DE02168081D2060D1F80090DE
:10E3700030215046FCF79AFD78215046FCF796FD77
:10E38000002008210B461022CDE9001049465046D6
:10E3900005F034FD05E025215046FCF787FD00E03F
:10E3A00000BF00BF6D1C03E031465046FCF77EFD08
:10E3B000287800287FF41AAF00BF9AF80C0010B13B
:10E3C0005046FFF7FCFE00BF0DE72DE9FF470C4666
:10E3D00015461E46DDE90C78684600F00BF98146CB
:10E3E00044EA450040EA860040EA072040EA084146
:10E3F00009F5E060009A40F82210BDE8FF872DE99A
:10E40000FF470C4615461E46DDE90C78684600F0CD
:10E4100001F9814644EA450040EA860040EA0720C7
:10E4200040EA084109F5E060009A40F82210BDE892
:10E43000FF872DE9FF470C4615461E46DDE90C789F
:10E44000684600F007F9814644EA450040EA860044
:10E4500040EA072040EA084109F5E060009A40F8E8
:10E460002210BDE8FF872DE9F84F05460C4600262F
:10E470003746B046B1460095684600F08BF88246B4
:10E4800046EA470040EA840040EA082040EA0941A1
:10E490000AF5E060009A40F8221000BFBDE8F88F4E
:10E4A0001CB504460020009003460122114601904D
:10E4B0002046FFF7A4FF1CBD2DE9F84F06460D4688
:10E4C00014460027B846B9460096684600F082F820
:10E4D000824647EA480040EA850040EA092040EACF
:10E4E00004410AF5E060009A40F8221000BFBDE840
:10E4F000F88F73B50D46684600F07CF8044604F5C5
:10E50000E060009950F8210020F4403104F5E0600B
:10E51000009A40F82210009950F8210040EA054185
:10E5200004F5E060009A40F822107CBD3CB503463B
:10E530000A4D30CDCDE9004518460BE05DF820408E
:10E54000D4F8204514605DF820501468C5F82045C3
:10E55000121D401C5C188442F0D83CBD9049030059
:10E5600031B5684600F016F804460121009A01FA18
:10E5700002F0C4F80C0500BF38BD31B5684600F0A4
:10E5800049F804460121009A01FA02F0C4F80C058A
:10E5900000BF38BD01460868202802D24FF0A040D5
:10E5A0007047087800F01F0008600148F8E7000095
:10E5B0000003005001460868202802D24FF0A04016
:10E5C0007047087800F01F0008600148F8E7000075
:10E5D0000003005001460868202802D24FF0A040F6
:10E5E0007047087800F01F0008600148F8E7000055
:10E5F0000003005001460868202802D24FF0A040D6
:10E600007047087800F01F0008600148F8E7000034
:10E610000003005001460868202802D24FF0A040B5
:10E620007047087800F01F0008600148F8E7000014
:10E630000003005001460868202802D24FF0A04095
:10E640007047087800F01F0008600148F8E70000F4
:10E650000003005001460868202802D24FF0A04075
:10E660007047087800F01F0008600148F8E70000D4
:10E670000003005001464A09002312B1012A06D1C5
:10E6800002E04FF0FF3302E040F2FF3300BF00BF73
:10E6900001F01F0101208840184008B10120704797
:10E6A0000020FCE731B56846FFF7A4FF044600BF31
:10E6B000D4F810050099C84000F0010038BD31B50C
:10E6C0006846FFF767FF04460121009A01FA02F04D
:10E6D000C4F8080500BF38BD31B56846FFF79AFF9A
:10E6E00004460121009A01FA02F0C4F8080500BFAF
:10E6F00038BD31B56846FFF7ADFF04460121009AE9
:10E7000001FA02F0C4F8080500BF38BDF8B50446A8
:10E710000D466DB900946846FFF75CFF064601217F
:10E72000009A01FA02F0C6F80C0500BF00BF0DE028
:10E7300000946846FFF74EFF06460121009A01FA51
:10E7400002F0C6F8080500BF00BF00BFF8BD00001A
:10E7500001460148084470470060004038B504464F
:10E760002046FFF7F5FF002101602046FFF7F0FF8C
:10E770000068009000BF38BD10B504462046FFF782
:10E78000E7FF0068012800D110BD0020FCE7000071
:10E7900001490860704700000463004070B50446FA
:10E7A0000E46FBF7BFFA0546681C08B9284670BD3F
:10E7B000E8B2E168087100BF0A48006928B9094851
:10E7C00004610020E168086009E006480069C0684B
:10E7D0000068E168086003480069C0680460284672
:10E7E000E5E7000018790020704710B5F9F7B4FF8D
:10E7F00010BD704738B504460D4605484FF4806398
:10E80000044A29460090204600F006F838BD000072
:10E8100081280300F85B00202DE9F04F93B0824679
:10E820000E4617469846DDF87090304600F0F5FB2E
:10E8300018210DA8F8F7FEFD0D97CDF83880CDF81A
:10E84000489000252B46082207A9304600F002FC1C
:10E85000082509980A90BDF82000ADF82C00BDF8F5
:10E860002200ADF82E0000208DF83100079800F04E
:10E87000030001281BD107984FEA902B0798C0F39B
:10E88000C2008DF830000798C0F38314A2002B4615
:10E8900001A9304600F0DEFB05EB84050DA80AABAC
:10E8A000224601A90090584600F0F6FA27E00798A2
:10E8B00000F00300022822D107984FEA905B0798E6
:10E8C000C0F3C2008DF8300000BFBBF1080F01D2C9
:10E8D000584600E0082004462B46224605A930464B
:10E8E00000F0B8FB2544ABEB040B0DAB0AAA2146A4
:10E8F00005A800F017FABBF1000FE6D100BF3046C3
:10E9000000F099FB13B0BDE8F08F000010B502468F
:10E910000B4C04EBC203012906D0022906D00329BF
:10E9200006D0042908D105E0022007E0042005E014
:10E93000187903E0587901E0002000BF00BF10BD46
:10E940000059030010B54FF0FF34FFF74EFF0421CC
:10E950000548FFF723FF044600BF01200249C968AC
:10E96000487100BF10BD0000F05803002DE9F04FC2
:10E970008BB0FCF7B1FA18B100200BB0BDE8F08FF6
:10E980000021B548816100BF00BF00BFBFF34F8FBA
:10E9900000BF00BF00BFA0F5805080680A90AF485C
:10E9A00004680A982040AE4901EB800A0025002641
:10E9B0000020069000BF0AA95046FEF7C4FBB0B184
:10E9C000A548806998B9A6480C3840680A998842D9
:10E9D00007D8A3480C384068A1490C39886000204A
:10E9E000CBE70A9820409E4901EB800A00E000E056
:10E9F000E1E700BF00270AE00A98411C20400A9185
:10EA0000974951F8200007A941F827007F1C022FE1
:10EA1000F2D3079800F0030002287AD10798800DFE
:10EA200005904FF448710798B1EB905F02DD0798AD
:10EA3000800D01E04FF448708146079869F39F50BC
:10EA4000079009F1080004900798C0F3C2000690EF
:10EA50008448049900F084FA0546002D57D02846D2
:10EA600000F0DBFA3346082207A9284600F003FB32
:10EA700008360A982040611C081A4FEA8008C145F0
:10EA800032D9B8F1000F05D00A982040744901EB43
:10EA9000800000E072480390B8F1000F01D04046BA
:10EAA00000E0484600F0FF0BB8F1000F01D06C48C1
:10EAB00000E000200290B8F1000F02D0A9EB08009E
:10EAC00000E00020C0B2019033465A462846039920
:10EAD00000F0D1FA5E44029828B133462846DDE9B9
:10EAE000012100F0C8FA0BE00A9820405C4901EBD4
:10EAF000800B33464A465946284600F0BCFA00BF10
:10EB00000598C01C0A9901EB90000A9000BF43E0F1
:10EB1000FFE7079800F0030001283DD10798C0F3F4
:10EB20008310062803DA0798C0F3831000E006205C
:10EB3000079960F3891107910798C0F3831000F1DA
:10EB400002080798C0F3C20006904FEA88014548C2
:10EB500000F006FA0546F5B1284600F05EFA3346A5
:10EB6000082207A9284600F086FA083600270DE09B
:10EB70000A98421C20400A92394A02EB800133462F
:10EB80000422284600F077FA361D7F1C0798C0F350
:10EB90008310B842ECD800BFDDB32F48D0F8108006
:10EBA000806918B1284600F046FA31E019E04FF0CC
:10EBB000000900BFD8F80C004079012800D1814637
:10EBC000B9F1000F08D000BFD8F80000294602684C
:10EBD0004046904700BF00BFD8F80C00D0F8008036
:10EBE00000BFB8F1000FE2D1284600F024FA00205F
:10EBF000059005A8FBF742F81748806918B918492D
:10EC00000C390A9888609DF81400FBF73DF800BFA6
:10EC10001DE0FFE71048D0F810800AE0C146D9F89F
:10EC2000000081684846884700BFD8F80C00D0F83B
:10EC30000080B8F1000FF1D10B490C4A891AC908BC
:10EC4000022242EA01400AA100F01CF800BFFCF7D2
:10EC500043F980F0010090E618790020E82E0020AA
:10EC600024690020B8590300985903000059030093
:10EC70004261636B656E647320666C75736865646E
:10EC80000000000070B504460D4600231A462946D0
:10EC9000204604F081FB70BDF8B505460E461446CB
:10ECA000009401236A463146284604F075FBF8BDFE
:10ECB0002DE9FC4106460F4614461D460094019579
:10ECC00002236A463946304604F066FBBDE8FC8103
:10ECD0002DE9FE4306460F4614461D46DDF8288002
:10ECE00000940195CDF8088003236A4639463046E2
:10ECF00004F052FBBDE8FE832DE9FF4706460F46B0
:10ED000014461D46DDE90C8900940195CDF8088074
:10ED1000CDF80C9004236A463946304604F03CFB9B
:10ED2000BDE8FF872DE9F05F07460E4690461D4679
:10ED3000082E01D9BDE8F09F95F80C9000202873AB
:10ED40002946404602F07CF900240CE0B44205D28A
:10ED50003A5D1DA12846FFF71DFA03E01CA12846D5
:10ED6000FFF718FA641C082CF0D31AA12846FFF705
:10ED700011FA00241DE0B44216D217F804A0BAF12B
:10ED80007E0F09DCF8F730FB006810F80A0000F08D
:10ED90003E0008B1504600E02E2083465A460EA1A0
:10EDA0002846FFF7F7F903E00CA12846FFF7F2F930
:10EDB000641C082CDFD301222946404602F01CF9CE
:10EDC00085F80C9000BFB5E72025303278000000B0
:10EDD000202020007C0000002563000020000000AF
:10EDE0002DE9F04106460F4600BF00200949087092
:10EDF000094800F01AF9044614B12046BDE8F08134
:10EE0000064800F0DFF906480649401AC508002008
:10EE1000F4E7000018690020B8590300484C0300CB
:10EE2000B85903000059030002480349401AC008BA
:10EE300070470000B85903000059030013B50C4691
:10EE400021466846FEF7B4FC28B90448009A00EB56
:10EE5000C20108681CBD0020FCE700000059030047
:10EE600070B50B48046901200A4908700CE000BF26
:10EE70000120E168487100BF25462868416828469E
:10EE8000884700BFE0680468002CF0D170BD000026
:10EE900018790020186900202DE9FF4707460C4625
:10EEA000164698460C9D95F80C900020287329462C
:10EEB000404602F0C5F8072E47D2DFE806F0040905
:10EEC0000F161F2A370039462846FFF763F93DE041
:10EED000394628462268FFF75DF937E0394628466B
:10EEE000D4E90023FFF756F930E0A06800903946D6
:10EEF0002846D4E90023FFF74DF927E0D4E90201C1
:10EF0000CDE9000139462846D4E90023FFF742F94C
:10EF10001CE0D4E902122069CDE9001202903946C2
:10EF20002846D4E90023FFF735F90FE0D4E902239E
:10EF3000D4E90410CDE90023CDE902103946284672
:10EF4000D4E90023FFF726F900E000BF00BF00224C
:10EF50002946404602F050F885F80C90BDE8FF873E
:10EF60002DE9F84F07468A46388AA0F104080AF1CD
:10EF700004004044401EB0FBF8F0C0B20090384698
:10EF8000FEF709FE044614B90020BDE8F88F002002
:10EF9000207101216171A4F8068025460098A0F136
:10EFA000010B2C462F604FF0000912E03846FEF7A7
:10EFB000F2FD064636B16079401C60712E60376004
:10EFC000354604E0204600F008F80020DDE709F1AE
:10EFD0000109D945EAD32046D7E72DE9F05F044679
:10EFE000274697F805802646A8F1010B002501E089
:10EFF00036686D1C5D45FBD3D6F800A0264600257B
:10F0000007E0D6F8009031465046FEF7F5FD4E4633
:10F010006D1C4545F5D3BDE8F09F70B50446254607
:10F020000121281DFEF775FD70BD10B50446204670
:10F03000FEF700FE10BDF8B5044626460121301D3E
:10F04000FEF79EFD00906D46287810B92046FFF728
:10F05000C4FFF8BD2DE9FC4105460E4614461F4687
:10F06000019401203B4601AA314600902846FEF754
:10F070003AFBBDE8FC812DE9FC4105460E461446ED
:10F080001F46019400203B4601AA314600902846C5
:10F09000FEF729FBBDE8FC8100BF00BF00BFBFF346
:10F0A0005F8F00BF00BF00BF0021016070470246B4
:10F0B000505808B1012070470020FCE708B5002235
:10F0C00042504258009200BF08BDC0F8001370477C
:10F0D000C0F81415704710B5136800F5A46404EB6C
:10F0E0004114236000BF938800F5A46404EB41142D
:10F0F000636000BF936800F5A46404EB4114A3604F
:10F1000000BFD36800F5A46404EB4114E36000BFC2
:10F1100010BDC0F800127047012242507047000035
:10F1200010B500200A49087000BF0A49086000BFF6
:10F1300000BF00BF00BFBFF35F8F00BF00BF00BFB5
:10F1400000BF0549054800F0FCFA002010BD000092
:10F15000C82E0020C42E0020604A0300905B0020CF
:10F1600070B50446144D01212846FEF7F3FC06460F
:10F1700000BF00BF00BF00BFBFF35F8F00BF00BF75
:10F1800000BF0EB9012000E0002000B970BD042CC2
:10F190000BD00A48007818B10748FFF77DFFF5E764
:10F1A0000748047001200549087003F0EDFD02488E
:10F1B000FFF772FF00BFE9E7C42E0020C82E002031
:10F1C000C02E0020002182689160826811618268EF
:10F1D00051618268D16082685160826811607047B5
:10F1E000024602F5A86050F82100704700F5A863B8
:10F1F00043F8212070470146D1F80405704708B54F
:10F20000002242504258009200BF08BD08B50022BB
:10F2100042504258009200BF08BDC0F848137047E2
:10F22000C0F848137047C0F844137047C0F844133F
:10F230007047024650587047C0F808137047C0F82E
:10F2400008137047C0F804137047C0F804137047E0
:10F250000246D2F80403084070470122425070472A
:10F260000122425070470000024A1060121D1160D6
:10F27000704700002C76004001460348085808B14A
:10F28000012070470020FCE70070004008B5002115
:10F29000034A815011464158009100BF08BD00004B
:10F2A000007000400121014A815070470070004009
:10F2B000014609B90E207047024800680860002026
:10F2C000F9E70000D84C0300FEB506460C46204680
:10F2D000FFF7EEFF05460DB12846FEBD0020009069
:10F2E000019002908DF8006001208DF80200062147
:10F2F000ADF8041069462020226869DF054675B123
:10F30000284600F0C1FA07464F49504A891AC908F1
:10F31000012242EA01403A464D49FFF7BDFC002078
:10F3200000900190029001208DF8010000208DF8DE
:10F3300002008DF8030069464020226869DF054617
:10F3400075B1284600F0A0FA07463F493F4A891A9E
:10F35000C908012242EA01403A463E49FFF79CFCB7
:10F3600000200090019002908DF80060F720ADF829
:10F37000020069462320226869DF054675B12846E8
:10F3800000F082FA07463049304A891AC90801223A
:10F3900042EA01403A463049FFF77EFC00200090E7
:10F3A0000190029002208DF8000069460120226839
:10F3B00069DF054675B1284600F066FA074622491E
:10F3C000224A891AC908012242EA01403A462349E1
:10F3D000FFF762FC00200090019002904FF4C8609B
:10F3E00000906946A120226869DF054675B128466C
:10F3F00000F04AFA07461449144A891AC90801223A
:10F4000042EA01403A461649FFF746FC00200090C8
:10F41000019002908DF800006946A020226869DF03
:10F42000054675B1284600F02FFA07460649074AF7
:10F43000891AC908012242EA01403A460949FFF700
:10F440002BFC002049E70000A859030000590300E5
:10F45000545603009C560300E8560300B4550300BD
:10F4600000560300605503002DE9F041044625686D
:10F47000204660DF06462068A84225D91E491F4A5B
:10F48000891AC908022242EA01401DA1FFF7FAFBCE
:10F4900019491A4A891AC908022242EA01402A4631
:10F4A00023A12368FFF704FC01F06CFF2168471AD1
:10F4B0001149124A891AC908022242EA01403A4611
:10F4C00028A1FFF7E9FB00E000BF1EB90120304989
:10F4D00008700EE0304600F0D7F907460649074AA3
:10F4E000891AC908012242EA01403A4629A1FFF7D8
:10F4F000D3FB3046BDE8F081A85903000059030052
:10F50000496E73756666696369656E742052414D14
:10F5100020616C6C6F636174656420666F72207427
:10F52000686520536F66744465766963652E0000D4
:10F530004368616E6765207468652052414D207391
:10F5400074617274206C6F636174696F6E2066728F
:10F550006F6D203078257820746F20307825782ED4
:10F56000000000004D6178696D756D2052414D209D
:10F5700073697A6520666F72206170706C6963616F
:10F5800074696F6E20697320307825782E00000032
:10F590002F2F002073645F626C655F656E61626C23
:10F5A0006528292072657475726E65642025732E36
:10F5B000000000002DE9F041ADF5027D80461848BD
:10F5C000007818B90DF5027DBDE8F0811DE04FF41B
:10F5D000FA70049004A905A861DF044604B115E09F
:10F5E00005AD104901A800F0ACF809E000BF039890
:10F5F0000646376828467168B84701A800F0C2F887
:10F6000000BF03980028F1D100BFE0E700BF052C40
:10F6100004D000BF2046F9F7C7FF00BF00BFD1E705
:10F620002F2F0020CC4C03001CB51B48007808B1DC
:10F6300008201CBD012019490870002003F0ACF817
:10F64000112801D10020F4E7002003F0C3F814488A
:10F6500000680190002000906846FAF70FFB1149FE
:10F6600001A810DF04460CB9012000E000200A497F
:10F6700008709DF80000FAF707FB0CB12046D8E7A8
:10F680000020064908700849087003F0F1FB0120CA
:10F6900003F0A0F80020CCE72C2F00202E2F002014
:10F6A000A84C0300E99402002D2F00203EB50A4922
:10F6B000684600F046F809E0684600F03FF8044666
:10F6C00025686068A847684600F05CF8684600F066
:10F6D00035F80028F0D13EBD9C4C0300014800786D
:10F6E000704700002C2F00202DE9FF41074618E04D
:10F6F00003A84BDF044604B114E00F49684600F04C
:10F7000020F809E000BF029805462E686968039852
:10F71000B047684600F036F800BF02980028F1D1E3
:10F7200000BFE5E700BF052C04D000BF2046F9F775
:10F730003BFF00BFBDE8FF81EC4C03000146886839
:10F74000704770B504460D46256028686060204605
:10F7500000F001F870BD14E0D0E900215268914238
:10F7600002D100218160704741680968426852688F
:10F77000914203D0416809688160F4E7416808312B
:10F780004160E9E710B50446A06800B910BD2168E2
:10F79000A06889680844A060D4E9011049688842DB
:10F7A00005D16068083060602046FFF7D4FF00BFD5
:10F7B000ECE770B505460E466C6806E020683146F9
:10F7C000AA68904700B903E0246820680028F5D1B2
:10F7D00000BF20683060266070BD01464868006840
:10F7E000704701464A6810684A68126822B14A6840
:10F7F000126812684B681A60704710B503460A46D3
:10F800000020596807E00C68944203D114680C602A
:10F81000012003E009680C68002CF4D100BF10BD82
:10F820000246505808B1012070470020FCE708B597
:10F83000002242504258009200BF08BDC0F8081391
:10F84000704701224250704770B502460D4B03F5D8
:10F85000947413E0E61AF01000EBD076761003EB08
:10F86000C6010D68954201D90C4606E0954202D2C8
:10F8700001F1080301E0486870BD00BFA342E9D36D
:10F880000020F9E7804A030030B504462046FFF720
:10F89000DBFF05460DB9024830BD2846FCE70000F5
:10F8A0006C4A030001464FF4A07000EB810080B267
:10F8B000704701464FF480308840704708B50022F9
:10F8C00042504258009200BF08BD0021C0F8001508
:10F8D00070470521C0F8001570470146D1F8C404EF
:10F8E000C1F8C40470470246505808B1012070475F
:10F8F0000020FCE708B5002242504258009200BFA9
:10F9000008BDC0F804137047C0F800127047012208
:10F91000425070470348006808B10120704700203A
:10F92000FCE700000004014010B500F091F901204F
:10F930000149086000BF10BD1805004001460020C5
:10F94000054A12790AB1852004E0034A11600122B8
:10F95000014B1A7170470000582E002010B502208C
:10F96000FEF774FA4FF48270FEF767FA0C20FEF788
:10F9700073FA00BF00BF03480068C0F300400028CE
:10F98000F8D110BD1804004070B5044604B970BD2C
:10F99000024EA5012846B04700BFF8E7314A0300F0
:10F9A0000146080B40B270470146080B40B2704751
:10F9B0000146080B40B270470146080B40B2704741
:10F9C0002DE9F04706460D46304601F081FAF0B1C8
:10F9D0003046FBF70BFBA0F10808404601F004FBA2
:10F9E0000446032C08D13046FEF75CFE08B1032024
:10F9F00000E00220074605E0012C01D1022000E0D2
:10FA00000320074639463046FEF773FD2AE03046AC
:10FA100001F06AFA30B33046FBF7E8FA0446A0007A
:10FA200000F5807087B220460F4951F8201041F050
:10FA300001020D4941F8202000BF3846FEF78EFE36
:10FA40007DB13046FBF7D2FA8146FBF787FA804654
:10FA5000B8F1000F04D0012101FA04F0FEF798FE7E
:10FA600000BF00BFBDE8F087106500402DE9FC47EE
:10FA700006460D4617464FF00008304601F01AFAC8
:10FA800010B14FF0080864E0A878C0F3400239468E
:10FA90003046FBF76BFA0446601C002856D0A87865
:10FAA000C0F3800030BBA87800F0010090B101964F
:10FAB00001A8FEF79FFD814609F5E060019950F825
:10FAC000210020F0020A09F5E060019940F821A028
:10FAD00000BF0CE095F80190002000904B460246D4
:10FAE000014601903046FEF770FC00BF00BF304673
:10FAF00001F0D0F9A878C0F34000D0B128781649B9
:10FB000051F82410154A1140134A42F824101146A6
:10FB100051F824104FF47C5202EA06224FF440338D
:10FB200003EA00431A4311430B4A42F8241000BF72
:10FB30000EE0A4F108000A49085C297840EA811027
:10FB400042B2A4F1080006490A5401E04FF004084B
:10FB500000BF4046BDE8FC8710650040FFC0FCFFC9
:10FB6000D25900202DE9F041304890F8640018B1D6
:10FB700008263046BDE8F081002408E02046FEF764
:10FB800079FD10B1204601F0BFF9601CC4B22A2CE7
:10FB9000F4DB002404E02046FBF7D0F9601CC4B27B
:10FBA0000C2CF8DB21485E30002101608180204868
:10FBB000FFF7FAFE0546062728463946002804DBEB
:10FBC0004A07130E1B4A135408E04A074FEA126C07
:10FBD000194A00F00F031B1F02F803C000BF00BF4B
:10FBE0001348FFF7E1FE0546284600280DDB00BF5D
:10FBF00000BF00F01F02012191404209920002F172
:10FC0000E022C2F8001100BF00BF00BF00BF4FF4E8
:10FC1000BE70FEF7A3FD4FF00040FEF7B9FD0120D6
:10FC2000024981F8640000263046A3E77859002095
:10FC30000060004000E400E018ED00E0014601F043
:10FC40006040B0F1005F01D1012070470020FCE767
:10FC50002DE9F04106254FF08040FFF7A1FE044654
:10FC60002046E21704EBD2625211920002F1E02228
:10FC7000D2F800212146E31704EBD3635B11A4EB18
:10FC800043160123B3401A400AB1012200E00022CA
:10FC900082BB4FF08040FFF783FE04462E4620468D
:10FCA0003146002804DB4A07130E134A135406E0BA
:10FCB0004A07170E114A00F00F031B1FD75400BF4D
:10FCC00000BF4FF08040FFF76BFE0446204600283F
:10FCD0000DDB00BF00BF00F01F020121914042096F
:10FCE000920002F1E022C2F8001100BF00BF00BF85
:10FCF00000BF00BFBDE8F08100E400E018ED00E0C7
:10FD00002DE9F84307460E46384601F0EBF9044664
:10FD1000D4B14FF00008002000906846F9F7AEFF1C
:10FD2000207910B14FF0010802E026600120207117
:10FD30009DF80000F9F7A8FFB8F1000F03D01125D6
:10FD40002846BDE8F88300BF00252846F9E770B5CE
:10FD50000546284601F0C6F9044614B1002020608B
:10FD6000207170BD2DE9F04704460D46914620797B
:10FD70003E4901EBC006307920B14FF008084046FB
:10FD8000BDE8F087C6F8009029462046FBF7B8FA90
:10FD900020680121C0F8001500BF6979AA792B8974
:10FDA0002068C0F80C15C0F80425C0F8083500BF5D
:10FDB000A97AEA7A206841EA0223C0F8103500BF28
:10FDC00000212068FFF7A5F900212068FFF77DF9E1
:10FDD0004FF48E712068FFF771F94FF48871206835
:10FDE000FFF76CF94FF48A712068FFF767F94FF459
:10FDF00082712068FFF762F9306888B32068FFF7E6
:10FE0000DBFD074695F804A038465146002804DB80
:10FE10004A07130E164A135408E04A074FEA126CB9
:10FE2000144A00F00F031B1F02F803C000BF00BFFD
:10FE30002068FFF7C1FD0746384600280DDB00BFEC
:10FE400000BF00F01F02012191404209920002F11F
:10FE5000E022C2F8001100BF00BF00BF00BF00BF1A
:10FE6000012030714FF00008404689E7682E0020DD
:10FE700000E400E018ED00E070B50446207909497F
:10FE800001EBC00500262879022800D001264FF496
:10FE900082712068FFF70BF910B10120287101264B
:10FEA000304670BD682E00202DE9F05F044689467B
:10FEB00015461E4620791C4901EBC00A4A4600211E
:10FEC0002068FFF708F94A4601212068FFF703F987
:10FED00005F00107AB4605EBDB7207EB620291B25E
:10FEE0002068FFF7F5F806F0010010B14FF0100898
:10FEF0000AE006F0020028B10FB1082000E004205B
:10FF0000804601E04FF0000841462068FFF701F904
:10FF10000FB10C2000E008200346F2B25146204603
:10FF200003F0D2F9BDE8F09F682E002070B50446BA
:10FF30000D46002600212068FFF7EBF80421206819
:10FF4000FFF7EAF82046FFF797FF08B1012609E01E
:10FF500000BF2046FFF790FF08B1012601E0002D09
:10FF6000F7D100BF304670BD10B5044600212068AF
:10FF7000FFF773F90220617901EB4101014A505406
:10FF800010BD00007C2E00202DE9F04303461646EC
:10FF900058792D4A42F82060587900EB40002B4AEE
:10FFA000105C18B108242046BDE8F08393F9045092
:10FFB0008F7828463A46002808DB4FEA427C4FEA11
:10FFC0001C68DFF88CC00CF800800BE04FEA427C24
:10FFD0004FEA1C69DFF87CC000F00F08A8F10408A4
:10FFE0000CF8089000BF00BF93F9042010460028C9
:10FFF0000DDB00BF00BF00F01F070125BD40470912
:020000040003F7
:10000000BF0007F1E027C7F8005100BF00BF00BFE5
:1000100000BF0A881868C0F8082500BF08795A7917
:1000200002EB4202094D2A445070C8785A7902EB1B
:1000300042022A44907001205A7902EB4202A854ED
:1000400000242046B0E70000782E00207C2E0020FF
:1000500000E400E018ED00E02DE9F04104460D4613
:100060004FF48076012731462068FFF7C8F83946FB
:100070002068FFF7D8F81DB139462068FFF7E2F88D
:10008000BDE8F0812DE9FF4F83B007460C46387973
:1000900000EBC0006A4901EB8006307F28B14FF0C9
:1000A000080A504607B0BDE8F08F3D683A79654BC5
:1000B00053F822103868FFF723FE18B14FF0110AE9
:1000C0005046EFE70598306006987060207B012865
:1000D00003DC2078FEF751FA02E02078FEF7FCFA04
:1000E000002000900190207800231A460121FEF79D
:1000F00086F96078FF2808D094F801904846FEF70A
:100100003CFA4846FEF7CCF901E04FF0FF39A07801
:10011000FF280ED094F802804FF0010B00200090D1
:100120005B460246014601904046FEF768F900BF73
:1001300001E04FF0FF38A07886F82000E078F077F3
:10014000E078FF280DD0207918B1E078FEF715FA95
:1001500002E0E078FEF7C0FAE078FEF7A1F9207936
:10016000B0772078C5F80805C5F80C95C5F8108556
:1001700000BFA068C5F8240500BF217B627B0AB1DF
:10018000012300E00023184631B1012906D00229DD
:1001900007D0032908D000BF00BF08E040F00200EC
:1001A00005E040F0040002E040F0060000BF00BFA0
:1001B000C5F8540500BFA079C5F8C00500BF00BF51
:1001C0000720C5F8000500BF306888B33868FFF71E
:1001D000EFFB83466179029158460299002804DBBF
:1001E0004A07130E184A135408E04A074FEA126CE4
:1001F000164A00F00F031B1F02F803C000BF00BF28
:100200003868FFF7D5FB8346584600280DDB00BF52
:1002100000BF00F01F02012191404209920002F14B
:10022000E022C2F8001100BF00BF00BF00BF00BF46
:1002300000207077012030774FF0000A504631E7F8
:10024000105A0020E449030000E400E018ED00E04B
:100250002DE9FC410546287900EBC0002D4901EB52
:100260008004206808B32868FFF7A2FB06463046E2
:10027000002817DB00F01F0201219140264A4309A4
:1002800042F8231000BF00BF00BFBFF34F8F00BF75
:1002900000BF00BF00BF00BF00BFBFF36F8F00BF34
:1002A00000BF00BF00BF00BF00BF2F68206898B12B
:1002B0001A493846FFF7C2FA607F68B11421384600
:1002C000FFF7BFFA00BF4FF482713846FFF7A8FA74
:1002D0000028F8D00020607794F82000FF280CD088
:1002E00094F820600020009003460122014601900E
:1002F0003046FEF784F800BF00BF00BF0020C7F8FB
:10030000000500BF2868FFF722FD00202077BDE828
:10031000FC810000105A002080E100E0520108003A
:100320002DE9F04105460E461746287900EBC0003E
:10033000154901EB80044FF00008607F20B14FF0B9
:1003400011084046BDE8F081206820B107F0140094
:1003500008B90120607796E80E10C4E9053CC4E9AD
:100360000312E07FFF2808D0A07F18B1E07FFEF7DE
:10037000B3F902E0E07FFEF700F93B463246214642
:10038000286802F0F5FEDDE7105A002000B50146AE
:100390000248016000F004F800BD000004E50140DF
:1003A00000BF024800680028FBD0704700E401400D
:1003B0002CB51949194A891AC908032242EA014091
:1003C00017A1FEF75FFC1D48002101601C481B4976
:1003D000086000BF1B4804F0A7F80546002D19D09F
:1003E00019A00D490D4A891AC9080322CDE9000553
:1003F00042EA0140CA2320A226A1FEF77DFCFEF7B7
:10040000B5FA00BF00BF24B100BF2046F9F7CCF811
:1004100000BF00BF00BF2CBD985903000059030066
:10042000696E6974207A646174616368616E6E6577
:100430006C2073657276696365000000F82C0020FB
:10044000B9440300643100207A64617461636861B7
:100450006E6E656C5F696E697428266D5F7A68726E
:10046000732C20267A646174616368616E6E6C65BA
:100470005F696E69742900007372635C6164733133
:100480003239335F73696D706C655F746573746561
:10049000722E630025733A2564205A4552524F52FA
:1004A0005F434845434B28257329206661696C3AB0
:1004B0002564000010B1032801D101E000E000BF75
:1004C00000BF704710B50446FCF79AFD014A03C20D
:1004D00010BD0000A82E002010B504460548006895
:1004E00030B10448006803F04BF80020014908606F
:1004F00010BD0000982E0020DCB50646307800289C
:1005000023D13B211148008876DF044600BF2746EF
:10051000002F19D00EA01149114A891AC9080322C7
:10052000CDE9000742EA014073230EA215A1FEF7B0
:10053000E3FBFEF71BFA00BF00BF25B100BF284652
:10054000F9F732F800BF00BF00BFDCBD3C2F002030
:100550006572725F636F6465000000009859030064
:10056000005903002E2E5C6C69627A6E6F726469AA
:10057000635C7372635C7A626C655F6D6F64756CEB
:10058000652E630025733A2564205A4552524F5216
:100590005F434845434B28257329206661696C3ABF
:1005A0002564000070B50546AE883046FCF756FD60
:1005B000044674B14FF6FF7340F2F31205F10801DF
:1005C00004F10A00FCF7D0FE607221463046FAF7CB
:1005D00093FF70BD2DE9F0410546EF7BAE88012FFA
:1005E00001D0BDE8F0814FF6FF70FCF737FD0446FF
:1005F0001CB9042002F026F9F3E700BF2680002092
:1006000020720E480168C4F80A104068C4F80E0051
:1006100000BF4FF6FF7340F2F31205F1100104F131
:100620000A00FCF7A1FE60720548C08918B921468E
:100630003046FAF761FF00BFD3E70000502E0020DC
:10064000CC5800208188014A9180704708800020A2
:10065000CA7B012A02D18A88A0F8242470470000AE
:100660002DE9F04705460F46BE88A81D00EBC604DD
:100670002879A071F87B012802D0022806D102E077
:100680002888208003E06888208000E000BF00BF49
:1006900020886188884236DD22882049204BC91A8B
:1006A000C908042343EA014033461EA1FEF700FBBC
:1006B00021883046A5DF8046B8F1000F02D1012025
:1006C00060711FE0B8F1110F0DD1012020711349A5
:1006D000134A891AC908042242EA014032462149D4
:1006E000FEF7DAFA0EE04046FFF7CEF881460B49F6
:1006F0000B4A891AC908012242EA01404A461AA156
:10070000FEF7CAFA00BFA079E179884203DDA1793A
:100710003046FBF745F8BDE8F087000000590300BC
:100720000059030052657175657374696E672074B2
:100730006F2075706461746520415454204D545588
:1007400020746F202575206279746573206F6E2088
:10075000636F6E6E656374696F6E20307825782ED6
:1007600000000000B850030073645F626C655F674F
:10077000617474635F65786368616E67655F6D74EB
:10078000755F72657175657374282920726574755B
:10079000726E65642025732E0000000030B587B0AE
:1007A00005460020039004900590069002208DF8E5
:1007B0000C00174903C9CDE9000102A80190154AB0
:1007C000518990886A46ADDF044654B902A8FAF709
:1007D00075F930B101218DF812100020ADF810002C
:1007E00003E040F2FD10ADF8100000BF0949888811
:1007F00003A9B0DF0446112CF8D0BDF8100008B1F1
:1008000007B030BD2846F9F7A3FE00BFF8E70000A7
:10081000184D03000880002070B58EB004460E46C7
:100820002C22311D03A8F6F7ECFDBDF80C50BDF8E5
:100830001000C1B2A01D00EBC500C171A11D01EBEC
:10084000C501CA792749284BC91AC908042343EAB4
:1008500001402B4625A1FEF72BFABDF812202149B5
:10086000214BC91AC908042343EA01402BA1FEF712
:1008700013FABDF810201B491B4BC91AC9080423E1
:1008800043EA01402AA1FEF707FABDF816201549F0
:10089000154BC91AC908042343EA014029A1FEF7F0
:1008A000FBF9BDF814200F490F4BC91AC9080423DE
:1008B00043EA014027A1FEF7EFF9206980B12949F9
:1008C00003C9CDE90101ADF80650A01D00EBC5003C
:1008D000C0798DF8080001A920462269904700BF21
:1008E0000EB070BD005903000059030044617461EB
:1008F000206C656E6774682075706461746564202F
:10090000746F202575206F6E20636F6E6E65637443
:10091000696F6E2030782530782E00006D61785F29
:1009200072785F6F63746574733A202575000000F8
:100930006D61785F74785F6F63746574733A2025B6
:10094000750000006D61785F72785F74696D653A5B
:10095000202575006D61785F74785F74696D653A04
:1009600020257500884903002DE9F04705460E460D
:10097000341D2188A81D00EBC10794F8048022884B
:100980000B490C4BC91AC908042343EA01404346EA
:1009900009A1FEF78DF9B879404501DAB87900E090
:1009A0004046814620884946FAF7FAFEBDE8F087BE
:1009B000005903000059030050656572206F6E20D6
:1009C000636F6E6E656374696F6E20307825782072
:1009D000726571756573746564206120646174610A
:1009E000206C656E677468206F66202575206279BB
:1009F0007465732E000000002DE9F0410646B788AB
:100A00003846FCF72BFB05466DB16868F9F713F91A
:100A1000044614B1204601F015FF00BF4FF6FF70E9
:100A2000288000BF00BFBDE8F0810000054989882B
:100A30008288914200D070474FF6FF71014A918041
:100A400000BFF8E70880002070B504460E4600207D
:100A500084F82E04B088B4F8241488420CD120798C
:100A600050B901212046F9F794FB054625B1A06B4A
:100A700010B12846A16B884770BD70B504460D467D
:100A8000AA88A11D01EBC200FCF7F2FC70BD0000BA
:100A90002DE9FC4706460F46BD88B7F80690B01D05
:100AA00000EBC5042B492C4A891AC908042242EAE2
:100AB00001404B462A4629A1FEF7FAF8B9F1170F73
:100AC00001DA172000E0484681462088484501DDCC
:100AD000484600E02088608000202071009523882F
:100AE00062881C49DFF870C0A1EB0C01C9084FF007
:100AF000040C4CEA014028A1FEF7EAF821882846B8
:100B0000B5DF8046B8F1000F0ED04046FEF7BCFEC0
:100B100082461049104A891AC908012242EA014056
:100B200052462DA1FEF7B8F8607908B1BDE8FC8700
:100B3000306968B1344903C9CDE90001ADF802500C
:100B40006088ADF80400694630463269904700BFBE
:100B500000BFEBE7005903000059030050656572C0
:100B6000206F6E20636F6E6E656374696F6E2030E8
:100B70007825782072657175657374656420616E7F
:100B800020415454204D5455206F66202575206215
:100B9000797465732E0000005570646174696E6726
:100BA00020415454204D545520746F2025752062E7
:100BB000797465732028646573697265643A2025C9
:100BC0007529206F6E20636F6E6E656374696F6E3A
:100BD00020307825782E000073645F626C655F6753
:100BE000617474735F65786368616E67655F6D7467
:100BF000755F7265706C7928292072657475726EE4
:100C000065642025732E0000804903002DE9FC4116
:100C100005460E46B788B6F80A80A81D00EBC70443
:100C20002088404501DD404600E0208860806088E3
:100C3000172801DA172000E0608860806288114977
:100C4000114BC91AC908042343EA01403B460FA1CE
:100C5000FEF72EF8286978B1607968B11A4903C99E
:100C6000CDE90001ADF802706088ADF80400694676
:100C700028462A69904700BF002060712071BDE8B6
:100C8000FC81000000590300005903004154542026
:100C90004D5455207570646174656420746F20250F
:100CA00075206279746573206F6E20636F6E6E6558
:100CB0006374696F6E2030782578202872657370B0
:100CC0006F6E7365292E00007849030070B50546E4
:100CD000AE1D30880749C98888420AD10548007E80
:100CE00038B1F9F701FC04461CB102484169022001
:100CF000884770BD088000200548D0E900304FF0DB
:100D000080729A1840F100000149C1E90020704743
:100D1000A02E002070B50546A8880E498988884213
:100D200000D070BDAC1D2078022810D16088094920
:100D3000C98888420BD1207A042808D0207A062856
:100D400005D0207A052802D0A01CFFF727FD00BFA0
:100D5000E7E70000088000202DE9F04104460D4639
:100D60002888262801D0BDE8F081287A012802D001
:100D7000287A02280ED1A078F8F77AFB0746394680
:100D80002046F9F706FA064626B1A06B10B13046A8
:100D9000A16B884700BFE6E72DE9F0410446A51D99
:100DA00028881249C98988421DD1688902281AD128
:100DB000B4F804804046FCF751F9064696B105F1B7
:100DC0000C00F9F784FE20B131464046FAF794FB57
:100DD00008E07068F8F72FFF074617B1384601F0B2
:100DE00031FD00BF00BFBDE8F0810000CC580020FD
:100DF000FEB504460E46B51D0020009001900290FD
:100E00002988208981420FD1688902280CD105F1F7
:100E10000C00F9F75CFE18B1012084F8220029E0EB
:100E2000002084F8220025E02988208B81420FD100
:100E3000688902280CD105F10C00F9F748FE18B1B9
:100E4000012084F8230015E0002084F8230011E03D
:100E50002888A18988420DD1E06958B100208DF819
:100E6000000005F10C0001906989ADF80810684692
:100E7000E1698847FEBD01460868012805D0086879
:100E8000022802D00868042801D101207047002000
:100E9000FCE7000070B5024605490B46D40802F095
:100EA00007021D5D0126964035431D5500BF70BDEC
:100EB000D6590020014605484056012202EBE07059
:100EC00008B1012070470020FCE70000A85900206D
:100ED000014604484056082801DB012070470020E5
:100EE000FCE70000A85900200146064840560028AB
:100EF00005DB04484056082801DA0120704700202D
:100F0000FCE70000A8590020FF2201490A5470475D
:100F1000A85900202DE9F84F814600BF00244FE07A
:100F20002C480057401C00B949E0204600F054F816
:100F3000054649462846FCF79BFE00283ED0204641
:100F400000F052F8064600956846FDF753FB8346CD
:100F50000BF5E060009950F82100C0F30140804695
:100F6000B8F1020F01D1032000E002208246514671
:100F70002846FDF7BEFA00956846FDF73BFB834621
:100F8000012000998840CBF8200500BF2846FAF7D9
:100F90002DF88346F9F7E2FF074677B1032E09D013
:100FA000B8F1020F01D1012E04D0B8F1030F04D122
:100FB000022E02D131462846B84700BF00BF641C4C
:100FC000042CADD34846FCF70EFA0028A6D1BDE8A4
:100FD000F88F0000D259002001460248425C22F0FE
:100FE000C0007047D259002001460248425C900977
:100FF00070470000D259002070B504460D461646D1
:10100000207A05280CD0607A28B10A480AA1026823
:101010002846FDF7BFF809A12846FDF7BBF804E014
:101020001EB106A12846FDF7B5F82846FDF7C7F81A
:1010300070BD0000002F0020257300000D0A000085
:10104000F8B504460D46E08838B116A00090E38854
:1010500016A218A12846FDF79DF8207A05281FD072
:10106000607A58B1217AA088FDF750FC174951F8F1
:101070002060324616A12846FDF78CF828462168E4
:1010800002F05CFBA0880021FDF7D8FE0646207A1E
:10109000104951F8202033460FA12846FDF77AF871
:1010A000F8BD00001B5B306D000000001B5B313B96
:1010B00033316D0025734C6F67732064726F7070ED
:1010C0006564202825642925730D0A00002F00205F
:1010D00025730000EC2E00203C25733E2025733A3A
:1010E0002000000001460348814201D102487047B8
:1010F0000020FCE700200040602E00202DE9F04198
:1011000007460D4616463C48007808B9BDE8F08110
:101110003A4C6520A0700020607003202070C4F855
:10112000037000205AE000EB400115F8213000EB7D
:10113000C001E21D535400EB400135F82110C1F30A
:10114000072300EBC001491C535400EB400155F844
:101150002110C1F3074300EBC001891C535400EB7D
:10116000400105EB81010B7900EBC001C91C535410
:1011700000EB400105EB81018988C1F3072300EBF7
:10118000C001091D535400EB400105EB8101496882
:10119000C1F3074300EBC001491D535400EB40016C
:1011A00005EB81010B7A00EBC001891D535400EB64
:1011B000400105EB81010989C1F3072300EBC00160
:1011C000C91D535400EB400105EB81018968C1F34F
:1011D000074300EBC00108315354401CB042A2DB6E
:1011E00006EBC600C01D1FFA80F84146034803F015
:1011F00094F900BF8AE70000112D00200C51002057
:1012000070B5064C6820A07000206070032020702C
:1012100003252946204603F080F970BD0C510020BB
:101220002DE9F04105460E46074C6920A0700020CC
:10123000607003202070E57026710527394620462E
:1012400003F06BF9BDE8F0810C5100202DE9F04767
:1012500004460D4616464FF00209022D74D360690C
:10126000A84271D92078012804D0022849D0032847
:101270000DD15EE02F4607EB5707206A00EB5721A0
:101280002046FCF7B1FA8146B9F1000F00D075E0B5
:1012900038467F1CC0F3080104F1300001EB000860
:1012A00005F0010028B1F1B298F8000061F31F10B9
:1012B00000E0304688F800000120E070206A00EB72
:1012C00057212046FCF790FA8146B9F1000F00D073
:1012D00054E0C7F3080104F1300001EB000805F009
:1012E000010010B1C6F3071006E098F8000000F006
:1012F000F000C6F30321084388F800000120E070E5
:101300003CE0206A00EB15212046FCF76DFA81468F
:10131000B9F1000F00D031E0B1B240F2FF1202EAA1
:10132000450304F13002981801F0C8FF0120E07075
:1013300024E0206A00EBD5112046FCF755FA8146DF
:10134000B9F1000F01D019E019E040F2FF1101EAF4
:10135000850204F130015018FCF76BF866F31B00AE
:10136000064640F2FF1101EA850204F130015018EF
:10137000314601F097FF0120E07000BF00BF4846F2
:10138000BDE8F08702480068810201F10050704713
:101390000C01001010B586B0694630A0FBF75FFA6B
:1013A0000446304830490860002C4ED1BDF8040096
:1013B000BC2101EB6020A0F5FA602C490870BDF853
:1013C0000400C0F343104870BDF8040000F01F0093
:1013D0008870BDF80600C012C870BDF80600C0F3E2
:1013E00045100871BDF80600C006800E48711E4801
:1013F00000680A680260496841601B4900980968F2
:10140000C86001201849486019491A4A891AC90850
:10141000032242EA014018A1FDF734FC1449154AA1
:10142000891AC908032242EA01400CA215A1FDF75E
:1014300033FC0F490F4BC91AC908032343EA014083
:1014400013A1009AFDF728FC05E000200649096871
:10145000C8600549486006B010BD0000302E6269C2
:101460006E00000004560020802D0020892D0020F1
:10147000985903000059030066696C656C697374C0
:101480003A000000206E616D653A2573000000008F
:101490002073697A653A25640000000010B504469F
:1014A000142C01DB002010BD21460548FCF714FB7D
:1014B00021460348001FFCF70FFB0120F3E7000063
:1014C000F058002070B50546002406E0044901EB01
:1014D00084002946FCF7E2FA641C1E2CF6D370BD8A
:1014E000EC58002010B598B00F488068C0431790A2
:1014F0000D48416817A8FCF717FB179901A8F9F7E1
:1015000073FF2C2201A90CA8F5F77BFF002405E04E
:101510000DA931F81400FFF7D5FF641C0C98A04208
:10152000F6D818B010BD0000E858002010B50446E9
:1015300021460248FCF7B2FA10BD0000F058002026
:101540002DE9F04781460E4617464FF00008D9F8BE
:101550000040022E02D36069B04202D80220BDE8EA
:10156000F08767B100BF4FF0FF3239462046FFF7E2
:101570006DFE8046B8F1000F01D04046EFE700BF96
:1015800031464846FBF740FC054605B922E0012DEF
:1015900001D10220E3E7681C08B90120DFE700223F
:1015A00031462046FFF752FE8046B8F1000F01D0C9
:1015B0004046D4E7D4E90410801E814206D2206957
:1015C000401C2061207940F0010020712E466069A6
:1015D000B042D5D800BF0020C1E70000042804D1E4
:1015E00002490968491C014A11607047302F0020E8
:1015F00010B504462046FAF724FE08B1FFF77CFB3D
:1016000000212046FAF72DFD10B12046FEF764FFB9
:1016100001212046FAF725FD10B12046FEF752FFC2
:10162000204602F01FF8204600F044F810BD0000EC
:101630002DE9F05F834688464FF00D09002088F8B9
:101640000000DBE90267FBF7DBFC341A67EB0105FE
:1016500000210846091BA8411ADAB4F5350F05D355
:10166000F8F768FA11490844002101E0304639468C
:1016700082464FF49603524600210D48FAF7F7FDD3
:101680008146B9F1000F02D10120BDE8F09F03E0CF
:1016900000210748FAF7DAFCB9F10D0F04D15846DA
:1016A00001F06EFF88F800000020EEE7FFFFB400B5
:1016B000902E0020F8B5074655E000BF2B48FEF7F6
:1016C0008CF806460EB1304600E0002004460025A6
:1016D000002C40D06B1ED4E9021059405840014301
:1016E00002D101F0E1FB3EE02148006808B9012584
:1016F00017E01F49D4E902300A68D2E90212591AE8
:1017000090410ED201251A480068D0E90210AA1EA5
:1017100051405040014304D0154801681348FEF77A
:1017200048F8BDB101F0C0FB044669462046FFF70A
:101730007FFF58B10E48006810B93846FAF789FDA6
:101740000B4804609DF8000018B90DE0002008491E
:10175000086007E008E00648006810B93846FAF764
:101760007FFD01E000BFA8E700BFF8BD1C4A0300F1
:10177000982E002070B504460E462546D5E9001087
:10178000884770BD10B504462046F7F7F1FA10B946
:1017900042F2010010BD2046002803DB1F4A125C04
:1017A000520905E01E4A00F00F031B1FD25C5209CC
:1017B0001146082904D20120884000F0EC0008B945
:1017C000002000E0012010B942F20200E2E71548D3
:1017D000806868B16009134951F8200004F01F02C5
:1017E00001219140084361090E4A42F8210012E0AC
:1017F000204600280DDB00BF00BF00F01F020121C2
:1018000091404209920002F1E022C2F8001100BFAB
:1018100000BF00BF00BF0020BCE7000000E400E004
:1018200018ED00E0845B002070B50446F7F7BCFAC1
:10183000054614488068D8B90120124988601248CA
:101840000068124908400F49086010484FF0E02135
:10185000C1F880010C488038D0F8840009494860FC
:101860004FF0FF310848001D01600020207001E0AA
:10187000012020701DB900BF62B600BF00BF00206C
:1018800070BD0000845B002080E100E0FC06FFBD2D
:1018900038B504460D4624B1012C1FD0032C38D195
:1018A00032E00020002817DB00F01F0201219140E8
:1018B000194A430942F8231000BF00BF00BFBFF31D
:1018C0004F8F00BF00BF00BF00BF00BF00BFBFF30E
:1018D0006F8F00BF00BF00BF00BF1BE00020009063
:1018E0006846F8F7CBF90D48007808B9FCF79EFB7D
:1018F0000A48C068401C0949C860012088709DF8EA
:101900000000F8F7C1F905E0FEF70EF8FCF7B4FBAC
:1019100000E000BF00BF38BD80E100E06459002056
:1019200070B501460878821122B1012A1CD0022A22
:1019300026D100E000BF087A8009CE7900EB86004E
:101940008E7906F0030600EB8623487900F00F0439
:10195000887AC0094E7A06F0030600EB4605601946
:10196000C61F581CB04070BD487A0C7A00EB0420AA
:10197000CC7904F03F0400EB0443581C8002F2E7EA
:1019800000BF00BF0020EEE72DE9F04705460E46F8
:1019900090463A4890F8230010B11120BDE8F08736
:1019A00000240121354880F8231005F08000A8B1FB
:1019B00006240221314880F8231077202F4981F82E
:1019C000280000212D4880F8291080F82A1080F87E
:1019D0002B1080F82C10FF2180F82D1005F07F01CE
:1019E000264828300155320E601C244928310A54FB
:1019F000C6F30742A01C0A54C6F30722E01C0A548F
:101A0000201D0E54402D02D0482D04D101E0952711
:101A100003E0872701E0FF2700BF00BF601D1749D3
:101A200028310F54B8F1020F03D0B8F1030F0AD1D7
:101A300004E00521114880F8241009E005210F4831
:101A400080F8241004E001210C4880F8241000BF25
:101A500000BF05F0800008B1012002E0074890F8BF
:101A60002400814609F10E00C3B2044A383206212F
:101A7000A2F1100000F054FE00208FE79C5B0020D4
:101A80002DE9FE43054668784249087042480668D9
:101A9000B469287820B1012834D002286CD14CE0F8
:101AA000687880B1B1464846F9F7E8F8074600BFC4
:101AB000B846B8F1000F04D000BF4046F7F774FDF8
:101AC00000BF00BF00BFF7F727FF006820604FF49A
:101AD00000706060304800688069806888B10020CC
:101AE000009001900290687808B1012000E0002089
:101AF0008DF80100A069029069463046A2689047BF
:101B000000BF43E02448006880698068A0B1234A90
:101B100007CA8DE80700687808B1012000E00020BE
:101B20008DF8010004F10C000190A0690290694653
:101B30003046A268904700BF28E0174800688069D7
:101B40008068C0B1154A0C32D2E900109268CDE924
:101B500001020091687808B1012000E000208DF8B2
:101B6000010004F10C000190A06902906946304622
:101B7000A268904700BF09E000BF032700BF032011
:101B8000F7F712FD00BF00BFBDE8FE8300BF00BF36
:101B9000FAE70000CC2E0020D02E0020C04B03001E
:101BA0002DE9FC5F80468946154698F8006098F854
:101BB0000100000698F8021040EA014098F803106E
:101BC00040EA012098F8041040EA010B0127FE4882
:101BD000808BB0F50E7F7DD010DC40F21322A0EB9D
:101BE0000201904252D004DCD0B1B0F5047F72D132
:101BF0002FE006297AD01329F9D1BAE040F2612208
:101C0000811A904269D006DCA0F24D20002870D0E5
:101C10000628ECD174E10A296CD00F29E7D1FEE146
:101C20002BE2012200214020FFF7AEFE044600BF58
:101C3000A246BAF1000F04D000BF5046F7F7B4FC3B
:101C400000BF00BF00BF00274FF40471DE4881834E
:101C500000BF17B90120BDE8FC9F00BF0122002191
:101C60004020FFF791FE044600BFA246BAF1000FE4
:101C700004D000BF5046F7F797FC00BF00BF00BF7D
:101C8000002740F21321D048818300BF0FB9012003
:101C9000E1E700BF00BF26F0030040B100BF042011
:101CA000287000BF0021C84881830220D3E700BF0D
:101CB00003224FF4D5714820FFF766FE044600BFAB
:101CC000A246BAF1000F04D000BF5046F7F76CFCF3
:101CD00000BF03E089E0D1E108E04BE100BF00BFB5
:101CE000002740F21921B848818300BF1FB90120A5
:101CF000B1E7D7E072E100BF06F00400A0B9B24836
:101D0000807A20F00700C01CAF49887200BF26F01F
:101D1000030040B100BF0420287000BF0021AA4882
:101D20008183022097E700BF0021A7480184807AC1
:101D300000F00700032802D14FF0804000E00020AF
:101D400001900222E9200199FFF71EFE044600BF20
:101D5000A246BAF1000F04D000BF5046F7F724FCAA
:101D600000BF00BF00BF002740F2262196488183B4
:101D700000BF0FB901206EE700BF06F00400B8B342
:101D80009148807A20F00700401C8F49887226F025
:101D9000040600BF8C48008C401C81B28A48018434
:101DA000008CB0F5FA6F08DD00BF0220287000BF7C
:101DB00000218548818302204DE702220021412035
:101DC000FFF7E2FD044600BFA246BAF1000F04D0BF
:101DD00000BF5046F7F7E8FB00BF00BF00BF002779
:101DE0004FF40E717848818300BF17B9012032E7A4
:101DF00013E000BF00BF26F0030040B100BF042085
:101E0000287000BF002170488183022023E700BFB3
:101E100006F001000028BDD18EE000BF26F00300CF
:101E200040B100BF0420287000BF002166488183B4
:101E3000022010E700BF47E06348008C401C81B2DD
:101E400061480184008CB0F5FA6F08DD00BF022004
:101E5000287000BF00215C4881830220FBE65A48BD
:101E6000807A00F00700032802D14FF0804000E0A4
:101E7000002001900222E9200199FFF785FD044628
:101E800000BFA246BAF1000F04D000BF5046F7F7DA
:101E90008BFB00BF00BF00BF002740F24D214A4826
:101EA000818300BF0FB90120D5E600BF00BF26F037
:101EB000030040B100BF0420287000BF0021424849
:101EC00081830220C7E600BF06F001000028B3D1DD
:101ED000022200217A20FFF757FD044600BFA246E8
:101EE000BAF1000F04D000BF5046F7F75DFB00BF0A
:101EF00000BF00BF002740F253213348818300BF59
:101F00000FB90120A7E600BF00BF26F0030040B1D3
:101F100000BF0420287000BF00212B4881830220CD
:101F200099E600BF0BF0804030B12748807A20F05E
:101F300008000830244988722348807A00F007009E
:101F4000032829D0012251025020FFF71DFD04462D
:101F500000BFA246BAF1000F04D000BF5046F7F709
:101F600023FB00BF00BF00BF002740F261211648DD
:101F7000818300BF0FB901206DE600BF00BF26F0CE
:101F8000030040B100BF0420287000BF00210E48AC
:101F9000818302205FE600BF0B4848300A49C860D1
:101FA000012148388182012200214920FFF7ECFC01
:101FB000044600BFA246BAF1000F04D000BF50464D
:101FC000F7F7F2FA00BF01E09C5B002000BF00BF02
:101FD000002740F26B212C48818300BF0FB90120FC
:101FE00039E600BF00BF26F0030040B100BF042067
:101FF000287000BF00212448818302202BE600BF07
:1020000008F10108A9F1010000F0FF0900BF00215B
:102010001D48C18300BF4FF41C71818300BF6B4614
:1020200010224946404600F0B3F8022801DA0020A9
:1020300011E600BF00BF00BF9DF8000048B100BF1F
:102040009DF80000287000BF00210F488183022006
:1020500001E600BF0C484830FFF762FC0A494860BF
:102060004FF400710848018100BF0020287000BFB4
:102070000021054881830220EDE5D2E500270021FB
:10208000014881830320E6E59C5B00202DE9F84FA1
:1020900006460F4614464FF0010A3C48808B38B183
:1020A000B0F5267F22D0A0F2A220002867D156E00A
:1020B00064E096F8008000BF28F0030048B100BF3C
:1020C0000420207000BF0021304881830220BDE839
:1020D000F88F00BF761C781EC7B200BF00212B48C6
:1020E000C18300BF4FF42671818300BF6B464FF45C
:1020F00000723946304600F04BF8022801DA002021
:10210000E5E700BF00BF00BF9DF8000048B100BF79
:102110009DF80000207000BF00211C488183022030
:10212000D5E700BF1948808A01281EDD0122002161
:102130004C20FFF729FC054600BFA946B9F1000F66
:1021400004D000BF4846F7F72FFA00BF00BF00BF1A
:102150004FF0000A40F2A2210C48818300BFBAF17F
:10216000000F01D10120B2E700BF00BF00202070A6
:1021700000BF0021054881830220A8E799E74FF0BE
:10218000000A0021014881830320A0E79C5B002016
:102190002DE9F04704460D4616461F464FF001084C
:1021A0008448C08B40F2D912811A90427AD005DC63
:1021B00048B1A0F2C710002875D16EE0072973D08E
:1021C0001329F9D1DBE0ECE07A48818AC182BDE0D5
:1021D000002178480184FF20764981F828000021F9
:1021E00074480183032180F823105FE07148008C5C
:1021F000401C81B26F480184008C44F62061884203
:1022000009DD00BF0220387000BF00216948C1838A
:102210000220BDE8F08702E0641C681EC5B215B15B
:102220002078FF28F8D045B32078FE281CD1641C04
:10223000681EC5B204225F4880F82320B54201DD44
:10224000304600E028460146002004E0225C594B5D
:10225000DB681A54401C8842F8D356480183C06892
:102260000844544AD06021E000BF0520387000BF08
:1022700000215048C1830220CBE710234D4A383259
:102280000121A2F1100000F04BFA00BF4FF000084E
:1022900040F2C7114748C18300BFB8F1000F04D115
:1022A0000120B6E72CE07DE049E000BF414890F80E
:1022B000230003289AD029E03E48008B301A1FFAE9
:1022C00080F9B9F1F00F01DD4FF0F00909F0FF03DB
:1022D00038480121C268283000F022FA3548C06829
:1022E00048443449C8600846008B484481B23148AC
:1022F000018300BF4FF0000840F2D911C18300BF35
:10230000B8F1000F01D1012083E700BF2948008BFD
:10231000B042D1DB2748C08A401E81B22548C18225
:10232000022300F138020121283000F0F9F900BF42
:102330004FF000084FF4F0711E48C18300BFB8F1A0
:10234000000F01D1012064E700BF00251948C08AB1
:1023500000287FF43DAFFF20164981F828000223B2
:1023600001F138020121A2F1100000F0D9F900BFFB
:102370004FF000084FF4F6710E48C18300BFB8F16A
:10238000000F01D1012044E700BF0021094880F877
:10239000231000BF0020387000BF0648C183022010
:1023A00037E711E74FF0000800210248C1830320FE
:1023B0002FE700009C5B00202DE9F0470646884689
:1023C00014460125D548808BB0F53B7F70D009DCE1
:1023D00088B1A0F2C320002842D010287DD0212847
:1023E00068D1A3E0A0F20A30002879D0162878D06E
:1023F0002628F5D16CE18AE196F800A000BF2AF00A
:10240000030048B100BF0420207000BF0021C34872
:1024100081830220BDE8F08700BFC048807A00F0C9
:102420000700012830D0BD48808A01282CDDBB4838
:10243000012201695920FFF7A7FA074600BFB946F4
:10244000B9F1000F04D000BF4846F7F7ADF800BF60
:1024500000BF00BF002540F2C321B048818300BF08
:102460000DB90120D6E700BF96F800A000BF2AF002
:10247000030040B100BF0420207000BF0021A74826
:1024800081830220C6E700BFA448818AC182D2E0CE
:102490000021A2480183042180F82310FF209F49D6
:1024A00081F828000846808A012804DDFC2103E029
:1024B0005DE012E02CE1FE21984880F8291002230B
:1024C00000F138021946283000F02AF900BF002533
:1024D00040F2D3219148818300BF1DB9012099E7C3
:1024E0008DE0C7E000BF25E08C48008BC0F5007090
:1024F0001FFA80F9B9F1F00F01DD4FF0F009874ABA
:10250000D368128B981809F0FF010123834A3832EF
:1025100000F006F98148008B484481B27F4801836E
:1025200000BF00254FF43971818300BF0DB9012030
:1025300070E700BF7948008BB0F5007FD4DB7748A7
:10254000C06800F500707549C8600321734880F8C1
:102550002310032300F138020121283000F0E0F8B5
:1025600000BF00254FF43B716C48818300BF0DB95B
:1025700001204FE700BF694890F83A0000F01F01C2
:10258000052915D00B2901D00D2908D100BF052040
:10259000207000BF00226148828302203AE700BF1A
:1025A0000420207000BF00225C488283022031E7B3
:1025B00000215A48018433E05848008C401C81B205
:1025C00056480184008C44F62061884208DD00BF33
:1025D0000220207000BF002150488183022019E7AB
:1025E00010234E4A38320121A2F1100000F098F871
:1025F00000BF002540F20A314848818300BF0DB971
:10260000012007E700BF002007E0315C21B1002274
:10261000424981F8232002E0401C4045F5D300BF29
:102620003E4890F823000328C6D03C48C08A401E8C
:1026300081B23A48C1823948C08A00287FF428AF65
:102640003648808A012859DDFF20344981F8280066
:10265000FD21324880F82910032300F138020221BD
:10266000283000F05DF800BF00254FF448712B487A
:10267000818300BF0DB90120CCE600BF00212748AF
:102680000184032180F8231033E02448008C401C8F
:1026900081B222480184008C44F62061884208DD22
:1026A00000BF0220207000BF00211C48818302204F
:1026B000B0E61023194A38320121A2F1100000F0CF
:1026C0002FF800BF00254FF44C711448818300BFE0
:1026D0000DB901209EE600BF002007E0315C21B16A
:1026E00000220E4981F8232002E0401C4045F5D32A
:1026F00000BF0A4890F823000328C6D000BF00207E
:10270000207000BF002105488183022082E673E625
:10271000002500210148818303207BE69C5B00208B
:102720002DE9F84305460E461746984600BF134864
:1027300090F8580000906846FBF78CFF8146012115
:10274000009A01FA02F0C9F80C0500BF00BF00BFF3
:102750003B46324629460A48CDF80080FBF701FD8A
:10276000044600BFA146B9F1000F04D000BF48469F
:10277000F6F71AFF00BF00BFBDE8F8839C5B00209E
:10278000084C030010B501E001F08DFCF7F7B4F838
:102790000028F9D110BD0000FEB505460C49684679
:1027A000FCF7CFFF0DE06846FCF7C8FF044626683B
:1027B00028466168B04708B91120FEBD6846FCF79D
:1027C000E1FF6846FCF7BAFF0028ECD100BFF4E750
:1027D000644C0300FEB505460A496846FCF7B1FFA4
:1027E0000AE06846FCF7AAFF0446266828466168A6
:1027F000B0476846FCF7C6FF6846FCF79FFF002815
:10280000EFD1FEBD804C030070B504460D46A120FB
:102810000B4908700120487008462168C0F8021072
:10282000A188C180A1790172093029680160A98855
:102830008180A97981711021093801F067FE70BD8E
:102840008C32002010B504460348806918B1024854
:1028500081692046884710BDCC58002070B50546D8
:102860000E463146284675DF044624B1112C02D0AD
:102870002046FFF7E7FF0CB9012070BD0020FCE700
:102880002DE9F84F88461546002D35D04FF0000948
:102890000A20009000BF08EB09012A460020F5F746
:1028A0005FFF0446A1442D1BFCB91448007800B911
:1028B00020E0012606B90FE000BF4FF47A7707B990
:1028C00006E0DFF83CA04FEA871B5846D04700BF20
:1028D000701E061EF1D100BF0098401E00900098A7
:1028E00018B900200549087004E001200349087068
:1028F000002DD0D100BF00BFBDE8F88FD42E00203E
:10290000414C03002DE9F04707460E4614469A460F
:10291000B86A10B90720BDE8F0874FF0000836E02C
:1029200008EB4801B86A00EB8105A88800F10209AC
:10293000B9F1FE0F01D90C20EDE709F10100218862
:1029400070542088401C20801620218870542088D4
:10295000401C208022889119288801F048FA21889B
:1029600008442080A88800280DDDA86808B9072041
:10297000D1E7AA8823889819A968F4F742FD20882E
:10298000A9880844208008F1010000F0FF0897F8AA
:102990002C004045C4DC0020BDE70246022082F83E
:1029A000310092F8240010B10720087001E00320E4
:1029B0000870108A88810020C2F8200402F22640A4
:1029C0004860D0688860002070470246012082F885
:1029D00031000020C2F8200402F2264048600020A6
:1029E000886002200870802088810020704770B5C0
:1029F00004460D466069A860208BA88194F82400E5
:102A000018B1062084F83C0002E0012084F83C0064
:102A1000204601F089FA78B1022028750421204669
:102A2000FAF749F9064600BF304600B170BD00BF55
:102A3000052084F8310002E0032084F8310004F519
:102A40008260C4F820040020F0E770B504460D460B
:102A5000E069A860208CA88194F8240018B10620B1
:102A600084F83C0002E0012084F83C00204601F09C
:102A70005BFA78B10220287504212046FAF71BF989
:102A8000064600BF304600B170BD00BF062084F886
:102A9000310002E0042084F8310004F58260C4F8BB
:102AA00020040020F0E7000070B5054611480068DA
:102AB000407E08B1062070BD00BF0F4800F108013C
:102AC000026828469047044600BF24B901200949FE
:102AD000096848760BE00F2C09D10849084A891A81
:102AE000C908012242EA01400649FCF7CBF820461A
:102AF000E1E700005C2F00202480002098590300AB
:102B0000005903003057030000BF0A7822F00F027B
:102B10000A700A7822F0F0020A7000BF062850D22C
:102B2000DFE800F0030E1B28354200BF0A7822F0D0
:102B30000F020A700A7822F0F0020A7000BF40E02B
:102B400000BF0A7822F00F02521C0A700A7822F0A5
:102B5000F00210320A7000BF33E000BF0A7822F0A2
:102B60000F02521C0A700A7822F0F00220320A701A
:102B700000BF26E000BF0A7822F00F02521C0A7044
:102B80000A7822F0F00230320A7000BF19E000BF6C
:102B90000A7822F00F02921C0A700A7822F0F002E2
:102BA00010320A7000BF0CE000BF0A7822F00F025A
:102BB000921C0A700A7822F0F00220320A7000BFDC
:102BC00000BF00BF704700000EB501F0FBFBF5F73A
:102BD0006DFEF5F74BFEF6F7F9F8F5F725FEF4F77D
:102BE000BDFFF5F719F8F4F7C5FF0220F5F7BEF8B9
:102BF0000220F4F7F1FF03211F20FBF734FC03212F
:102C00001F20FBF730FC00BFFCF7ACFF0546002D92
:102C10001AD03DA04149424A891AC9080322CDE988
:102C2000000542EA01404FF4B9733EA244A1FCF70B
:102C300063F8FBF79BFE00BF00BF24B100BF204636
:102C4000F6F7B2FC00BF00BF00BF45480068029025
:102C500003208DF8090002208DF8080000BF414ACA
:102C600002A91F20FCF702FF0546D5B13E482B49BB
:102C70002B4A891AC9080322CDE9000542EA01401E
:102C80004FF4BB7327A22EA1FCF736F8FBF76EFEBC
:102C900000BF00BF24B100BF2046F6F785FC00BF8F
:102CA00000BF00BF01211F20FCF78AFEF6F796FB4C
:102CB00029E0F6F711FDFBF759FEFAF7BFF908B165
:102CC000012000E00020054601F068FD0446274889
:102CD0000068A04216D02548046001F053FD064666
:102CE0000E490F4A891AC908032242EA01402049C5
:102CF00032460B681FA1FBF7DBFFF8F709F900204C
:102D00001B49086000BFD4E76E7266785F67706920
:102D10006F74655F696E6974282900009859030013
:102D2000005903007372635C616473313239335F3D
:102D300073696D706C655F7465737465722E630082
:102D400025733A2564205A4552524F525F434845F5
:102D5000434B28257329206661696C3A256400007D
:102D6000184903001D920200B84D0300082D0020F1
:102D7000E02C00202564206368616E6765636F75D1
:102D80006E743A25640A000010B50CE000BF2C48B0
:102D9000806804462B4800782168884700B910BD38
:102DA0002748FCF7EFFC00BF254880680028EDD1DC
:102DB00000BFFCF755F800BF00BFFBF7D7FD0028A8
:102DC000FBD100BF00BF1F480078032803D01D4877
:102DD000007802281DD100BF00BF00BF00BF00BFA8
:102DE000BFF34F8F00BF00BF00BF1748006800F45B
:102DF000E06016490843001D1349086000BF00BF8A
:102E000000BFBFF34F8F00BF00BF00BF00BF00BFB8
:102E1000FDE7FCF763FC10B133DF044600BF00BFE1
:102E200001200B49086000BF00BF00BF00BFBFF317
:102E30004F8F00BF00BF00BF00E020BFFDE70000D4
:102E4000905B0020C02E00200CED00E00000FA0591
:102E50000005004070B504460D462CB90120034919
:102E600048700020F8F7F4F970BD000064590020A4
:102E700070B51620FEF786FC044600BF254625B136
:102E800000BF2846F6F790FB00BF00BF70BD10B52D
:102E900000BF00F009F818B14FF0FF328260C26045
:102EA0000028F6D110BD000010B50448FCF799FCCD
:102EB00004460CB1204610BD0020FCE71C4A03006C
:102EC0002DE9FE4306468846F468357C9648C08A5C
:102ED00030B900BF944991F85800FBF70AFC00BFD5
:102EE000914890F82300022804D08F4890F82300DE
:102EF00001287DD1A81FC5B2A41D706800784C2898
:102F000003D115B1681EC5B2641C02E0681EC5B2CB
:102F1000641C15B12078FF28F8D045B97068007896
:102F20004C2803D1681CC5B2641E00E00024002CAC
:102F300049D17D4890F82200012844D001208DF825
:102F40000100794890F82200012806D0022805D017
:102F5000042816D005281CD117E000BF00208DF8EA
:102F600000000321704880F8221000BFF6F762FDD0
:102F7000074627B100BF3846F6F716FB00BF00BF73
:102F800010E001208DF800000CE002208DF8000018
:102F900008E000BF032700BF0320F6F705FB00BFD2
:102FA00000BF00BF00BF00BF5F4991F85800FBF7AA
:102FB000A0FB00BF03215C4880F82210016868462E
:102FC0008847BDE8FE83584890F82300022817D1AF
:102FD0000121554880F82310277827F0010070B9A7
:102FE000514890F824000E30C3B24F4A383200E006
:102FF0000AE00621A2F10A00FFF792FBE1E700BF19
:103000000021494880F8231006200290464890F895
:103010002200012806D002280BD0042830D0052831
:1030200075D150E00221404880F8221000218183B0
:1030300000BF02AA29462046FEF7B2FD02281EDB89
:1030400000208DF804009DF808008DF8050003218C
:10305000354880F8221000BF014691F85800FBF770
:1030600048FB00BF00BF314A4FF080415068C0F8B4
:10307000241500BF00BF2C48016801A888474FE015
:1030800002AA29462046FFF701F802281ADB012090
:103090008DF804009DF808008DF8050003212248F2
:1030A00080F8221000218182C18280F8231000BFA5
:1030B000014691F85800FBF71CFB00BF1A48016855
:1030C00001A888472CE002AA29462046FFF774F998
:1030D00002281ADB02208DF804009DF808008DF804
:1030E00005000321104880F82210002180F82310E9
:1030F0008182C18200BF014691F85800FBF7F9FABE
:1031000000BF0948016801A8884709E0FFE700BF40
:10311000032700BF0320F6F747FA00BF00BF00BF38
:1031200000BF00BF4DE700009C5B0020084C03007F
:1031300070B586B004460D462E4620788DF8040002
:1031400060680290217A8DF80C10E1680491217C6E
:103150008DF81410044850F82610044850F8262022
:1031600001A8904706B070BD685A0020585A002048
:103170002DE9F04704460E4615461F46286818B14B
:103180002868FCF75BFD28B1A86850B1A868FCF777
:1031900055FD30B9002070774FF010084046BDE86B
:1031A000F087D5E90001C4F844054FF4A962115134
:1031B00000BFD5E90201C4F834054FF4A7621151EC
:1031C00000BF4FF48C712046FCF731FB2046394696
:1031D00001F0010232B100BF01234FF4AA62135083
:1031E00000BF06E000BF00234FF4AA62135000BFE7
:1031F00000BF01F0020232B100BF01234FF4A86208
:10320000135000BF06E000BF00234FF4A862135024
:1032100000BF00BF00BF07F0080018B9102120460A
:10322000FCF70FFB3068A0B900BF4FF48C7120464B
:10323000FCF7F6FA0028F8D0F07FFF281CD0B07F0A
:1032400018B1F07FFBF799F916E0F07FFBF744FA2D
:1032500012E0A146012020EA970ABAF1000F04D13A
:1032600040214846FCF7EAFA04E04020C9F804038C
:1032700000BF00BF00BF00BF4FF0000840468EE710
:1032800070B506460C461546A9B204F11A0000F0C6
:1032900015F83078032804D1290C04F1140000F04B
:1032A0000DF870BD00F8011B090A00F8011B090A9E
:1032B00000F8011B090A00F8011B704700F8011B08
:1032C000091200F8011B70472DE9F04105460F4631
:1032D00014461E46022038717C713868A8B14FF040
:1032E000820804F0040008B148F0100804F0080057
:1032F00008B148F0200804F0100008B128F0800858
:1033000041462868FBF7E1FE00BF4FF48271286850
:10331000FBF7D4FE04F0800028B12868821911461A
:103320000846BDE8F08131462868FBF7F5FE00202D
:10333000F7E700002DE9F05F05460E4690461F4670
:10334000DDF828904FEA154AF8F774FE83464AEAFA
:103350000B42781C00EA09000E4941F8202007EAD8
:10336000090001EB8004206865F3C5002060206837
:1033700068F389102060206866F39F202060206831
:1033800020F00300401C2060206820F00400206032
:10339000BDE8F09F246900202DE9FC47804689465E
:1033A00016461C461C480768012201A92046F7F76B
:1033B00009FDC0B1019800F1020A002509E056F8A4
:1033C000252050460AF1010A3840144941F82020CE
:1033D0006D1CA542F3D30097224649464046019B07
:1033E000FFF7A8FF00BF0D480C38007880B100201F
:1033F00000906846F6F742FC00BF00BFFBF7B6FA44
:103400000028FBD100BF9DF80000F6F73DFC00BF8F
:10341000FAF739F8BDE8FC87E82E0020246900207F
:103420002DE9F04781460C4615469846002608F0DF
:103430000100A0B105E0641C761C39464846F7F748
:1034400035FD2778002FF6D104E06D1E2021484677
:10345000F7F72CFDB5421BD9002DF6D118E01CB1B1
:103460002046F3F7F2FF064604E06D1E2021484691
:10347000F7F71CFDB54201D9002DF6D105E0641C1B
:10348000761C39464846F7F711FD2778002FF6D10C
:10349000BDE8F08770B50446204600F043F80546C5
:1034A000002D38D1207803282ED1207901282BD166
:1034B0004202002104F13000FAF70CF94AF65521D6
:1034C00004F22E20FFF7FAFE144904F13000FFF752
:1034D000E9FE134904F50570FFF7E4FE04F50670F4
:1034E0002169FFF7DFFE04F50770E168FFF7DAFEF8
:1034F000E069401CE0626078012304F13001E26A77
:10350000F8F718FD00202071607800221146F8F7C6
:10351000C1FB00B10125284670BD00005252614137
:10352000727241612DE9F04104460027E078F8B15C
:10353000E56A607801232A4604F13001F8F7FAFCC5
:1035400008B1012714E00020E070206A281AA16960
:1035500088420DD2A67809E0A0690544607801236D
:103560002A4604F13001F8F7E5FC761E022EF3D26C
:103570003846BDE8F0810246501A20F07F4070477F
:103580002DE9FE4304464FF0000833480078012837
:103590005ED1002C5CD0F9F733FDD4E90232C01AB9
:1035A000914147D3002000906846F6F767FB2069F9
:1035B00018B94FF0FF31A160E1609DF80000F6F707
:1035C00063FB60690190A0690290244A082101A868
:1035D000F6F726F8054600BF2F4627B100BF38464C
:1035E000F5F7E2FF00BF00BF002000906846F6F745
:1035F00045FB206988B14FF0FF33D4E902105940F0
:103600005840014309D0D4E902302169591840F1EA
:103610000000C4E90210012600E000269DF8000029
:10362000F6F732FB2EB121460D48FCF7C2F84FF0F9
:1036300001080DE04FF0FF33D4E902105940584023
:10364000014305D021460648FCF7B3F84FF00108C6
:103650004046BDE8FE8300009C2E00207517030045
:103660001C4A0300F8B50646694620480068FAF788
:10367000F9F9044637E0207820B1012810D002285B
:1036800024D11DE06068D0E902104FF0FF335940AB
:103690005840014303D016486168FCF78AF816E0E9
:1036A000144960680968884203D100201149086004
:1036B00005E00F486168FCF7A0F8054600BF06E08A
:1036C000FFF7E5FB01200C49087000E000BF00BFD8
:1036D000694606480068FAF7B7F969460348006882
:1036E000FAF7C0F90446002CC5D1F8BD184A03000A
:1036F0001C4A0300982E00209C2E0020F8B5054699
:103700000E4669460B480068FAF790F904467CB10A
:1037100025706660694607480068FAF7B1F928B174
:1037200000BF0548F8F772FD00BF00BF0020F8BDDC
:103730000420FCE7184A0300902E00207047000088
:1037400010B531493148F5F725FD2F490C31304886
:10375000F5F720FD00F0ACFF38B1F4F701FB0128CC
:103760000AD00120F4F702FB06E0F4F7F9FA022888
:1037700002D00220F4F7FAFAA2202649264A12685B
:1037800001EB0211087002202249234A126801EB62
:10379000021148701C4800681E491F4A126801EB5C
:1037A0000211C1F802001848C1681A481A4A126882
:1037B00000EB0210C0F80610134801691548164ABC
:1037C000126800EB0210C0F80A1002211148124AD8
:1037D000126800EB02108173A2200E490E4A126893
:1037E00001EB0211C8730C480068401C0A490860CC
:1037F00008460068082806D18021064800F086FEA9
:1038000000200549086010BDF44E0020B82B0020B0
:10381000C02B00200C330020DC2C00202DE9F043CD
:10382000A3B005460E4690461F4600203880012270
:1038300029462448F8F74EFE8146B9F1000F0DD015
:103840002149224A891AC908012242EA01402A462E
:103850001FA1FBF721FA23B0BDE8F0830024194A29
:10386000802103A8F8F7DFFD11E001AB02AA1CA13B
:1038700003A8F3F707FE029806F8140006EB4401CC
:1038800001984870641C444500DB07E000BF0D4A06
:10389000802103A8F8F7C7FD0028E6D100BF3C80CF
:1038A00009490A4A891AC908032242EA0140234603
:1038B0002A460DA1FBF7FCF90248F8F7A3FD00BF6B
:1038C000C9E700008C330020985903000059030019
:1038D0006F70656E202573206661696C65640A00EF
:1038E00025782C25780000006C6F616420257320FA
:1038F0006366672073697A653A25640A00000000F0
:1039000070B586B006460C462146304600F051F9A7
:1039100008B106B070BD94F82F0018BB207B0228B8
:1039200002D0207B03281DD1616AA069814219D190
:10393000E06960626069A06294F82000C0F3401002
:1039400084F82C00002084F82D00207B032804D16B
:103950002146304600F0C4F93DE02146304600F0F3
:103960008DF838E0142204F10C0101A8F3F749FDA9
:1039700094F82F00E0B13046FBF7AFFF054605F0A5
:10398000020018B101208DF8000010E005F00400DD
:1039900018B102208DF8000009E005F0010018B10F
:1039A00003208DF8000002E004208DF8000002E002
:1039B00000208DF80000002084F8300094F82000EA
:1039C00000F0040010B194F82F0018B16846D4E953
:1039D0000021904700BF00BF9BE70146032001F094
:1039E00001020AB14FF4024001F002020AB148F2AA
:1039F000012001F004020AB148F20220704770B5BC
:103A000005460C46A16A606B884235D200BFD5F8E6
:103A10001805C0B2626B616A8854606B401C6063B9
:103A2000A06A401E616B814209D194F8200000F029
:103A3000400020B902212846FBF766FF18E0A16A82
:103A4000606B884206D194F8200000F0400008B96D
:103A5000012070BDA16A606B884209D194F82000F2
:103A600000F0400020B1022084F82D000020F0E793
:103A700020212846FBF74BFF0120EAE7F8B5064670
:103A80000C460027344800904FF482713046FBF713
:103A900031FF4FF492713046FBF72CFF4FF48E71DB
:103AA0003046FBF727FF4FF484713046FBF722FFC7
:103AB0000020606384F82F00A06A012809D194F8DF
:103AC000200000F0400020B902213046FBF71CFF27
:103AD00003E001213046FBF717FF20213046FBF7BA
:103AE00016FF94F82D00022803D000213046FBF782
:103AF0000EFF206838B140F28620A060A1683046F1
:103B0000FBF7FFFE25E002E00098401E00900098C1
:103B1000002805DD2146304600F04BF80028F3D19F
:103B200094F82F0058B13046FBF7D7FE054625B173
:103B30002846FFF752FF074600E0032700BF009822
:103B4000002806DC3046FBF7C0FE3046FBF7C1FE1E
:103B500003273846F8BD0000A086010070B5054671
:103B60000C46A16A606B884206D2626B616A885C0F
:103B7000C5F81C0500BF1AE094F82C0028B11C21E0
:103B80002846FBF7C4FE002070BD94F8200000F02A
:103B9000400040B11C212846FBF7B9FE012084F803
:103BA0002D000020F0E714212846FBF7B0FE01208D
:103BB000EAE770B505460C4600264FF482712846A8
:103BC000FBF791FE28B14FF482712846FBF792FE75
:103BD000012694F82F0078B14FF492712846FBF734
:103BE00089FE4FF48E712846FBF784FE4FF48471F2
:103BF0002846FBF77FFE5FE04FF492712846FBF703
:103C000072FE60B14FF492712846FBF773FE1421E7
:103C10002846FBF77CFE012084F82F004CE04FF48F
:103C20008E712846FBF75FFE08B34FF48E7128466D
:103C3000FBF760FE606B401C60634FF49271284696
:103C4000FBF751FE60B14FF492712846FBF752FE2C
:103C500014212846FBF75BFE012084F82F002BE09F
:103C600021462846FFF77AFF30BB002070BD4FF495
:103C700084712846FBF737FEF0B14FF48471284673
:103C8000FBF738FE4FF492712846FBF72CFE60B12B
:103C90004FF492712846FBF72DFE14212846FBF7BE
:103CA00036FE012084F82F0006E021462846FFF763
:103CB000A6FE08B90020D9E77EB1002084F82D00C7
:103CC00094F82F0038B92146284600F0F1F980F029
:103CD000010084F82F000020C8E70120C6E700009B
:103CE000F8B506460C4600272F4800904FF4827125
:103CF0003046FBF7FFFD4FF492713046FBF7FAFDBB
:103D00004FF48E713046FBF7F5FD4FF48471304669
:103D1000FBF7F0FD00213046FBF7F6FD0020606365
:103D200084F82F0020213046FBF7F1FD94F82D0098
:103D3000012803D008213046FBF7E9FD2146304633
:103D4000FFF70CFF206838B140F28620A060A16820
:103D50003046FBF7D6FD25E002E00098401E0090BB
:103D60000098002805DD21463046FFF722FF002895
:103D7000F3D194F82F0058B13046FBF7AEFD05465D
:103D800025B12846FFF729FE074600E0032700BFBC
:103D90000098002806DC3046FBF797FD3046FBF71D
:103DA00098FD03273846F8BDA086010030B50446CB
:103DB0001088C01C984201D90C2030BD0220158803
:103DC00048551088401C10800A20158848551088D6
:103DD000401C108015884C551088401C1080002015
:103DE000EBE7014608784A7840EA0220704702462D
:103DF0000A70100A48700220704700002DE9FF4F3A
:103E000081B0884616461F46DDE90E4B45464FF009
:103E1000010A03E0B5FBF6F50AF1010AB542F9D251
:103E2000574500D9BA460BF0010098B994B10BF090
:103E30000200022803D117B93020009001E02020B1
:103E4000009004E0641EDDE90010F7F72FF80CB1D4
:103E5000A245F7D3012509E0012F01D97F1E04E017
:103E6000B8FBF5F9B14500D201E07543F4E700BFB6
:103E700000BFB8FBF5F909FB15880D4810F80910CB
:103E80000198F7F713F8B5FBF6F5002DF1D10BF01B
:103E9000010048B144B104E0641E20210198F7F705
:103EA00005F80CB1A245F7D305B0BDE8F08F0000CE
:103EB000364A0300F8B506463546A8B2F9F7CEF8FB
:103EC00004466CB3207A1749097B88420ADAA8B203
:103ED00004F10A01FEF7C2FC074617B1207A401C24
:103EE00020721DE0002020720E48007C50B1A8B264
:103EF0003B2176DF074627B1082F02D03846FEF770
:103F0000A1FC00BF0748406950B100208DF80000B7
:103F1000A8B2ADF80200034841696846884700BF6F
:103F2000F8BD0000CC58002010B50446607940B1BF
:103F300094F82E0428B9204600F0B6F808B1012004
:103F400010BD0020FCE72DE9FC4780468946154658
:103F50009A46DDE90A675346022249464046CDE9C2
:103F6000006700F017F8044600BF204608B1BDE81E
:103F7000FC8700BF5346102229464046CDE9006722
:103F800000F008F8044600BF204600B1EFE700BF8C
:103F90000020ECE72DE9FF5F07468B4696461D465D
:103FA0000E9C4FF0000920880390C84647E07868CF
:103FB00000EB880000680190002202A901A864DFDC
:103FC000064600BF304610B104B0BDE8F09F00BF08
:103FD0009DF80800704530D1B9F1000F01D00020E4
:103FE00000E00220009020889DF80810014400980D
:103FF00001440F98814201DD0C20E5E7B9F1000F83
:104000000AD12088401C2080208805F800B0208834
:10401000401C20804FF001092088421902A901A804
:1040200064DF064600BF304600B1CDE700BF2188FF
:104030009DF808000844208000BF08F10108388876
:104040004045B4DCB9F1000F0DD021880398401C25
:10405000081A1FFA80FABAF1FF0F01DD0C20B3E74E
:10406000039805F800A00020AEE770B504460D46A1
:1040700084B1206870B12068007858B12068C08889
:10408000A188884206D121684878F7F7CBFE00F076
:10409000010018B100202860092602E0206828608D
:1040A0000026304670BD7047014691F830047047D5
:1040B00070B505460C46A16A606B884207D0284659
:1040C000FBF703FC2846FBF704FC002070BD012031
:1040D000FCE7000001480088704700003E2F0020E8
:1040E000F0B5ADB0054600BF9DF8A80020F00F0068
:1040F000401C2A909DF8A80020F0F00010302A9073
:1041000000BF2868F3F7A1F986B232462AA82968C9
:104110007CDF044600BF2746002F1AD08DA09049AF
:10412000904A891AC9080322CDE9000742EA0140F2
:1041300040F231138CA294A1FAF7DEFDFAF716FCD7
:1041400000BF00BF26B100BF3046F5F72DFA00BF13
:1041500000BF00BF00202B902C901020ADF8AC00C9
:104160003C20ADF8AE000020ADF8B0004FF4C870B0
:10417000ADF8B2002BA87ADF044600BF2746002F17
:104180001AD074A07649774A891AC9080322CDE962
:10419000000742EA014040F23B1373A27AA1FAF70A
:1041A000ABFDFAF7E3FB00BF00BF26B100BF30460E
:1041B000F5F7FAF900BF00BF00BF7B497B48F9F76C
:1041C00071FD044600BF2746002F1AD061A0644944
:1041D000644A891AC9080322CDE9000742EA01406E
:1041E00040F2451360A268A1FAF786FDFAF7BEFB1C
:1041F00000BF00BF26B100BF3046F5F7D5F900BFBC
:1042000000BF00BFF7216948F9F73DFD044600BF34
:104210002746D7B14FA05249524A891AC9080322EA
:10422000CDE9000742EA01404FF4A4734EA256A123
:10423000FAF762FDFAF79AFB00BF00BF26B100BF94
:104240003046F5F7B1F900BF00BF00BF686808B19C
:1042500068688047AC2102A8F3F7ECF802208DF8DB
:10426000080000208DF80A0006208DF80B000121BF
:10427000ADF854104E49169101218DF8841040215B
:104280002491002125914B482B9002A94A48F5F72B
:10429000DEFE064600BF3746D7B12EA03049314A70
:1042A000891AC9080322CDE9000742EA01404FF408
:1042B000B8732DA234A1FAF71FFDFAF757FB00BF20
:1042C00000BF24B100BF2046F5F76EF900BF00BF64
:1042D00000BF01213848F5F7B7FE1C2126A8F3F7E7
:1042E000A9F8002026904FF4A03027904FF4F0203A
:1042F000289003208DF8A4000020ADF8A6008DF8CA
:10430000A8002E482B902E482C9026A8F5F7FCFFED
:10431000064600BF3746D7B10EA01149114A891A87
:10432000C9080322CDE9000742EA014040F28713A1
:104330000DA215A1FAF7E0FCFAF718FB00BF00BFC9
:1043400024B100BF2046F5F72FF900BF00BF00BF22
:104350002DB0F0BD6572725F636F64650000000090
:1043600098590300005903002E2E5C6C69627A6E26
:104370006F726469635C7372635C7A626C655F6DB3
:104380006F64756C652E630025733A2564205A4569
:1043900052524F525F434845434B282573292066AC
:1043A00061696C3A2564000085CD0200F47F00202D
:1043B000382F0020B5040300C07B0020F90403005F
:1043C000E7B402007CB503211148F5F7E2FE05468B
:1043D00000BF2E46002E19D00EA01149114A891A8D
:1043E000C9080322CDE9000642EA014087230EA254
:1043F00015A1FAF781FCFAF7B9FA00BF00BF24B1A2
:1044000000BF2046F5F7D0F800BF00BF00BF7CBD5D
:10441000C07B00206572725F636F646500000000FE
:1044200098590300005903002E2E5C6C69627A6E65
:104430006F726469635C7372635C7A626C655F6DF2
:104440006F64756C652E630025733A2564205A45A8
:1044500052524F525F434845434B282573292066EB
:1044600061696C3A256400007FB505460C46114829
:10447000006890F8230010B9082004B070BD2088AF
:10448000F42801DD0720F8E7002000900190029059
:10449000039008480068808AADF8000003950294F4
:1044A00001208DF8020003490968098C88B2694629
:1044B000AEDFE2E7482F0020704700007FB50546D9
:1044C0000C461148006890F8220010B9082004B08A
:1044D00070BD2088F42801DD0720F8E70020009057
:1044E000019002900390084800688088ADF80000B1
:1044F0000395029401208DF8020003490968098C94
:1045000088B26946AEDFE2E7482F002013B50446C3
:1045100001A92046FFF7D2FF1CBD13B5044601A92F
:104520002046FFF7CBFF1CBDF0B58DB004460E460C
:104530005D4804604FF0FF305B49096808845B4BBD
:104540000FCB08AD0FC500BF14B90E200DB0F0BDE4
:1045500000BF00BF0EB90E20F8E700BF3068E06171
:10456000214608A862DF054600BF284600B1EDE7F6
:1045700000BF20788DF832000120ADF83000A21C79
:104580000CA9A8DF054600BF284600B1DEE700BF42
:1045900020216846F2F74EFF0220ADF80000207897
:1045A0008DF80200F420ADF804000120ADF80600FB
:1045B0008DF80C009DF80D0020F0080008308DF8F3
:1045C0000D009DF80D0020F00400001D8DF80D0079
:1045D00000208DF8110001208DF8120000BF6088C6
:1045E00004F10C026946F6F707FD07460FB138469D
:1045F000ACE700BF20216846F2F71CFF0320ADF8AE
:10460000000020788DF80200F420ADF804000120AD
:10461000ADF806008DF80C009DF80D0020F010009C
:1046200010308DF80D0001208DF811008DF812006A
:104630008DF8130000BF6088221D6946F6F7DCFC88
:1046400007460FB1384681E700BF20216846F2F7E0
:10465000F1FE0420ADF8000020788DF80200F4206F
:10466000ADF804000120ADF806008DF80C009DF8AF
:104670000D0020F0100010308DF80D0001208DF895
:1046800011008DF812008DF8130000BF608804F14E
:1046900014026946F6F7B0FC07460FB1384655E7F5
:1046A00000BF002052E70000482F0020084D030003
:1046B00004480068B0F92000401C08B10120704790
:1046C0000020FCE7482F002070B505460E4606B1D5
:1046D00005B970BD34462888102804D011281CD094
:1046E00050282DD127E01849184A891AC9080322F1
:1046F00042EA014016A1FAF7C5FAA88800B2208460
:104700002189A888F9F7FAF884F822002189A88875
:10471000F9F7F4F884F8230013E00B490B4A891ADF
:10472000C908032242EA01400FA1FAF7ABFA4FF0A1
:10473000FF30208405E029462046FCF759FB00E0C5
:1047400000BF00BF00BFC4E7985903000059030031
:10475000424C455F4741505F4556545F434F4E4E74
:104760004543544544000000424C455F4741505F7B
:104770004556545F444953434F4E4E454354454478
:104780000000000072B60449096801EB4102C2EB67
:10479000C11062B670470000302F002000B572B61D
:1047A000FFF7F0FF4FF47A71B0FBF1F362B61846F1
:1047B00000BD00007CB54FF480410020FAF710FBEB
:1047C000044600BF254625B100BF2846F4F7ECFE9D
:1047D00000BF00BFFAF7B6F8F5F720FE044600BFA9
:1047E000254625B100BF2846F4F7DEFE00BF00BF16
:1047F000F5F7BCF9044600BF254625B100BF2846A1
:10480000F4F7D2FE00BF00BFFAF78AFC044600BFEF
:10481000254625B100BF2846F4F7C6FE00BF00BFFD
:10482000FAF702FF044600BF254625B100BF28461F
:10483000F4F7BAFE00BF00BF0020019001A90120DB
:10484000FAF742FD044600BF254625B100BF2846C1
:10485000F4F7AAFE00BF00BF01A8FAF705FE044660
:1048600000BF254625B100BF2846F4F79DFE00BFD6
:1048700000BF0F4903C9CDE9000140F6FF70ADF854
:1048800000000C4A69460C48FBF77EFB044600BF5B
:10489000254625B100BF2846F4F786FE00BF00BFBD
:1048A00001210548FBF7D8FB0348FBF75DFB7CBD06
:1048B000004D0300DD150300F84C03002DE9F04323
:1048C0000246104601231C460D460026374600BF0F
:1048D000202802D24FF0A04803E000F01F00DFF8CC
:1048E0002480C44643EA440848EA850848EA062882
:1048F00048EA07490CF5E06848F8209000BFBDE899
:10490000F08300000003005002000000003002406D
:10491000010000000100000003000000182D00202D
:10492000382D0020D82D0020002E0020040000008B
:10493000000000000000000080FFFFFF07070000EC
:104940002E000200182E00200000000000000000D1
:10495000A84B0300C44F0300C04F0300B84F03002F
:1049600000020000110B04056C580020000000003C
:104970000338FDD870470000770A000000000000EF
:10498000770A0000000000007ADA00000000000052
:1049900000000050000300506E7266785F67706917
:1049A0006F74655F696E6974006E7266785F6770B8
:1049B000696F74655F6F75745F696E6974006E729C
:1049C00066785F6770696F74655F696E5F696E694D
:1049D000740000006E7266785F7370696D5F696E57
:1049E00069740000E58702000D8802007370696D2C
:1049F0005F78666572006E7266785F7370696D5F6E
:104A00007866657200000000FFFFFFFF0006FF00F0
:104A10000000004000000000745B00200000000067
:104A2000B02E0020C3B2020001000600000000000A
:104A30000338FDD8704730313233343536373839A2
:104A40004142434445460000CC590300D05903007D
:104A50000000000000000000000000000000000056
:104A6000484A0300604A030004000000556E6B6E64
:104A70006F776E206572726F7220636F64650000DD
:104A800000000000845403000100000030530300C4
:104A9000020000002451030003000000A45303009F
:104AA00004000000F853030005000000D852030082
:104AB000060000007452030007000000E0530300EA
:104AC00008000000EC5203000900000050530300EE
:104AD0000A0000006C5403000B0000000C5103009E
:104AE0000C000000045303000D000000D454030028
:104AF0000E000000D05303000F0000000C54030010
:104B0000100000004054030011000000E8540300AE
:104B100012000000BC5403001300000058540300AE
:104B2000800000008C52030081000000C851030087
:104B300082000000885103008300000068510300D8
:104B400084000000A451030085000000B05203005F
:104B500086000000B8530300900000005452030088
:104B60009100000048510300920000001853030018
:104B70000082000020540300018200006C530300F7
:104B8000028200008853030000840000E451030007
:104B90000184000090540300028400002C520300A2
:104BA000038400000852030035AB02007DAC020014
:104BB000F1AB0200DDAC0200BDAB02002DAB020088
:104BC00002000000000000000000000003000000E0
:104BD00000000000000000000001000000000000D4
:104BE00000000000010000000000000000000000C4
:104BF00002010000000000000000000002010000AF
:104C00000000000000000000000000000030004034
:104C10000000000001000000000000FF06FF00008F
:104C20000000000400000000000000000000000080
:104C3000F5E70200F3E70200E9E7020000000000E8
:104C40000338FDD87047000000670020FF01000016
:104C500000690020000000000000000000000000CB
:104C600000000000544C0300644C030008000000E6
:104C7000385A0300485A03000000000000000000FA
:104C8000704C0300804C030008000000285A030009
:104C9000385A030000000000000000008C4C0300A4
:104CA0009C4C03000800000000100201D0590300D2
:104CB000D8590300D8590300F8590300F8590300E4
:104CC000105A0300105A0300185A0300AC4C03009A
:104CD000CC4C030008000000B82B0020185A030039
:104CE000205A0300205A0300285A0300DC4C03001A
:104CF000EC4C0300080000000040024024000400C7
:104D000000000641000000009ECADC240EE5A9E078
:104D100093F3A3B50000406E020000000000000005
:104D200050EADA308883B89F604F15F30000C98ECF
:104D300000404040404040404040414141414140AE
:104D40004040404040404040404040404040404063
:104D500040050202020202020202020202020202F2
:104D600002202020202020202020200202020202F7
:104D7000020290909090909010101010101010104F
:104D8000101010101010101010101010020202025B
:104D9000020288888888888808080808080808089F
:104DA000080808080808080808080808020202029B
:104DB00040000000314D03006E7266785F677069D5
:104DC0006F74655F696E5F696E6974284144533121
:104DD0003239335F52454144595F50494E2C2026A9
:104DE000696E436F6E6669672C2061647331323976
:104DF000335F72656164795F70696E5F6972712992
:104E0000000000006170705F74696D65725F6372AD
:104E10006561746528266D5F7265636F72645F7586
:104E2000706C6F61645F746D722C204150505F54E0
:104E3000494D45525F4D4F44455F524550454154A1
:104E400045442C205265636F726455706C6F6164C9
:104E50005F746D725F636229000000006170705FB3
:104E600074696D65725F63726561746528266D5F34
:104E70007265636F72645F75706C6F61645F6669A1
:104E80006E6973685F7061636B65745F7265706F84
:104E900072745F746D722C204150505F54494D45BF
:104EA000525F4D4F44455F53494E474C455F534811
:104EB0004F542C205265636F726455706C6F61643F
:104EC0005F66696E6973685F7061636B65745F725A
:104ED00065706F72745F746D725F636229000000A9
:104EE0006170705F74696D65725F7374617274284C
:104EF0006D5F7265636F72645F75706C6F61645F24
:104F000066696E6973685F7061636B65745F726513
:104F1000706F72745F746D722C204150505F5449F1
:104F20004D45525F5449434B53283330292C202898
:104F3000766F69642A296D5F7265706F72745F6441
:104F40006174615F73756D636865636B636F6465DE
:104F5000290000006170705F74696D65725F637233
:104F60006561746528266D5F677265656E5F6C6943
:104F70006768745F6566666563745F746D722C2024
:104F80004150505F54494D45525F4D4F44455F522B
:104F9000455045415445442C20426F6172644C6930
:104FA0006768745F6566666563745F746D725F6879
:104FB000616E646C65722900312E30300000000093
:104FC0005344430049464C59544F50005265717543
:104FD000657374696E6720746F20757064617465A1
:104FE00020415454204D545520746F202575206263
:104FF00079746573206F6E20636F6E6E656374697C
:105000006F6E203078257820287265747279292E89
:105010000000000073645F626C655F6761705F64CD
:105020006174615F6C656E6774685F7570646174EC
:1050300065282920287265717565737429206F6E43
:1050400020636F6E6E656374696F6E2030782578AB
:105050002072657475726E65642025732E000000E1
:105060005468652072657175657374656420636F3B
:105070006D62696E6174696F6E206F66205458208E
:10508000616E64205258207061636B6574206C659A
:105090006E6774687320697320746F6F206C6F6E15
:1050A00067206279202575206D6963726F7365636F
:1050B0006F6E64732E00000073645F626C655F67DF
:1050C000617474635F65786368616E67655F6D7452
:1050D000755F726571756573742829206F6E206322
:1050E0006F6E6E656374696F6E20307825782072FC
:1050F000657475726E656420627573792C207769AA
:105100006C6C2072657472792E0000004E52465FFE
:105110004552524F525F494E56414C49445F4441BB
:10512000544100004E52465F4552524F525F534F1A
:1051300046544445564943455F4E4F545F454E41A2
:10514000424C4544000000004E52465F4552524FCB
:10515000525F464541545552455F4E4F545F454E50
:1051600041424C45440000004E52465F4552524F6A
:10517000525F4D555445585F554E4C4F434B5F461B
:1051800041494C45440000004E52465F4552524F43
:10519000525F4D555445585F4C4F434B5F46414914
:1051A0004C4544004E52465F4552524F525F4D555A
:1051B0005445585F434F4E445F494E49545F464102
:1051C000494C4544000000004E52465F4552524F44
:1051D000525F4D555445585F494E49545F464149C9
:1051E0004C4544004E52465F4552524F525F424C2E
:1051F000455F495053505F52585F504B545F545273
:10520000554E4341544544004E52465F4552524F1D
:10521000525F424C455F495053505F504545525F85
:1052200052454A4543544544000000004E52465FF3
:105230004552524F525F424C455F495053505F4C6C
:10524000494E4B5F444953434F4E4E4543544544AA
:10525000000000004E52465F4552524F525F41508F
:10526000495F4E4F545F494D504C454D454E544556
:10527000440000004E52465F4552524F525F4E4F1F
:10528000545F535550504F52544544004E52465F60
:105290004552524F525F4D4F44554C455F4E4F540F
:1052A0005F494E495449414C495A45440000000069
:1052B0004E52465F4552524F525F4D4F44554C45FA
:1052C0005F414C52454144595F494E495449414C14
:1052D000495A4544000000004E52465F4552524F25
:1052E000525F4E4F545F464F554E44004E52465FFC
:1052F0004552524F525F494E56414C49445F5354B8
:10530000415445004E52465F4552524F525F444110
:1053100054415F53495A45004E52465F4552524FE1
:10532000525F494F5F50454E44494E4700000000D0
:105330004E52465F4552524F525F5356435F48416B
:105340004E444C45525F4D495353494E470000006F
:105350004E52465F4552524F525F494E56414C495C
:10536000445F4C454E475448000000004E52465F93
:105370004552524F525F4452565F5457495F45520F
:10538000525F414E41434B004E52465F4552524F91
:10539000525F4452565F5457495F4552525F444EE4
:1053A00041434B004E52465F4552524F525F494E69
:1053B0005445524E414C00004E52465F4552524FAA
:1053C000525F53544F524147455F46554C4C000085
:1053D0004E52465F4552524F525F4E554C4C000064
:1053E0004E52465F4552524F525F494E56414C49CC
:1053F000445F504152414D004E52465F4552524F1C
:10540000525F4E4F5F4D454D000000004E52465FCB
:105410004552524F525F464F5242494444454E0016
:105420004E52465F4552524F525F4452565F545758
:10543000495F4552525F4F56455252554E0000004B
:105440004E52465F4552524F525F494E56414C496B
:10545000445F4144445200004E52465F4552524F11
:10546000525F5245534F5552434553004E52465F8B
:105470004552524F525F494E56414C49445F464C4B
:10548000414753004E52465F5355434345535300E3
:105490004E52465F4552524F525F424C455F495013
:1054A00053505F4348414E4E454C5F414C5245413D
:1054B00044595F4558495354530000004E52465FCB
:1054C0004552524F525F434F4E4E5F434F554E54DD
:1054D000000000004E52465F4552524F525F544901
:1054E0004D454F55540000004E52465F4552524FB5
:1054F000525F4255535900007761726E696E6700C2
:1055000064656275670000001B5B313B33306D00E2
:105510001B5B306D000000001B5B313B33316D00C5
:105520001B5B313B33326D001B5B313B33336D0012
:105530001B5B313B33346D001B5B313B33356D00FE
:105540001B5B313B33366D001B5B313B33376D00EA
:10555000696E666F000000006572726F7200000075
:1055600073645F626C655F6366675F736574282947
:105570002072657475726E65642025732077686586
:105580006E20617474656D7074696E6720746F202D
:1055900073657420424C455F47415454535F434602
:1055A000475F534552564943455F4348414E47453F
:1055B000442E000073645F626C655F6366675F73AF
:1055C000657428292072657475726E656420257370
:1055D000207768656E20617474656D7074696E679C
:1055E00020746F2073657420424C455F434F4D4DCE
:1055F0004F4E5F4346475F56535F555549442E0013
:1056000073645F626C655F6366675F7365742829A6
:105610002072657475726E656420257320776865E5
:105620006E20617474656D7074696E6720746F208C
:1056300073657420424C455F47415454535F434661
:10564000475F415454525F5441425F53495A452E7B
:105650000000000073645F626C655F6366675F7380
:10566000657428292072657475726E6564202573CF
:10567000207768656E20617474656D7074696E67FB
:1056800020746F2073657420424C455F434F4E4E2B
:105690005F4346475F4741502E00000073645F62DE
:1056A0006C655F6366675F73657428292072657433
:1056B00075726E6564202573207768656E2061744D
:1056C00074656D7074696E6720746F2073657420E3
:1056D000424C455F4741505F4346475F524F4C4500
:1056E0005F434F554E542E0073645F626C655F6379
:1056F00066675F73657428292072657475726E65BC
:1057000064202573207768656E20617474656D7000
:1057100074696E6720746F2073657420424C455F16
:10572000434F4E4E5F4346475F474154542E00005F
:1057300054686520626F6F746C6F61646572206875
:1057400061732077726974652070726F7465637419
:105750006564206974732073657474696E6773205F
:10576000706167652E20546869732070726F686974
:10577000626974732073657474696E6720746865F8
:10578000206164766572746973696E67206E616DFD
:10579000652E2054686520626F6F746C6F6164655C
:1057A00072206D75737420626520636F6D70696C13
:1057B00065642077697468204E52465F424C5F539F
:1057C000455454494E47535F504147455F50524FEF
:1057D000544543543D3020746F20616C6C6F7720CA
:1057E00073657474696E672074686520616476659A
:1057F00072746973696E67206E616D652E000000BA
:105800006E72665F626C655F6761747400000000B1
:10581000626C655F6E757300636C6F636B00000094
:10582000434C4F434B0000004750494F5445000044
:1058300050525300554152540000000055415254FB
:105840004500000053414144430000005350494D7E
:10585000000000005457490050574D005744540071
:105860005254430054494D45520000006170705F2E
:10587000627574746F6E00006170705F74696D653D
:10588000720000007077725F6D676D740000000039
:10589000736F72746C697374000000007274745FCB
:1058A0006C6F675F6261636B656E6400617070004E
:1058B0006E72665F736468006E72665F7364685FC1
:1058C000626C65006E72665F7364685F736F63001D
:1058D000485A0300B82B0020AC030000E079020016
:1058E000705B0300642F0020EC600000628D0200FA
:1058F000304C0300000000009C580300D82E00200C
:1059000000580300000004041058030000000000C9
:105910001858030000000000205803000000000099
:105920002858030000000000305803000000000069
:1059300034580300000000003C5803000000000041
:1059400044580300000000004C5803000000000011
:1059500054580300000000005858030000000000E5
:105960005C580300000000006058030000000000C5
:1059700064580300000000006C58030000000000A1
:105980007858030000000000845803000000000065
:105990009058030000000000AC580300000004040D
:1059A000B058030000000303B858030000000303CD
:1059B000C458030000000303E02E0020F85F00201D
:1059C00020600020206000202C000000919A02003E
:1059D00085A7020000000000CDA602000000000024
:1059E00045A702000000000057A10200C07B002074
:1059F000D9DC0200F47F0020C94603006431002096
:105A0000C94603000C52002005A5020008800020B2
:105A10003DA8020000000000552E03000000000019
:105A2000DDA5020000000000B5F502000000000046
:105A3000E9F60200000000009118030000000000D9
:105A4000F1AE020000000000011210080119022E40
:105A500003160412051406080712081209100A0A90
:105A6000170B070C740D010E160F031005111612FB
:105A700005133F1412151216141705181219121ACD
:105A8000121B121C121D100A210122202320242087
:105A9000251226162708280829122A122B122C1242
:105AA0002D162E332F70301231123212331234125F
:105AB000351236123712381239123A123B123C1292
:105AC0003D123E123F1440FF5012602A6282150CB4
:105AD0000214033982111D070F08FF821119821366
:105AE000780D1982111B10048208081507133B1446
:105AF000241504825A0282BA40820A283082011A8E
:105B00001AFF015306FF022C4029382901093620CB
:105B100001400922800933400C3EC001408064509E
:105B20004903024B011510014011024504A9B55A61
:105B3000FFAB1458550314F854031A5008111904F4
:105B40001A10041A08041A18041A20041A28041A2D
:105B500030041A38041A40042A4828F1128014929A
:105B6000650112020422FFFF14040090D00300001C
:040000050002720182
:00000001FF
